:020000040802F0
:10000000D8F40020A9010208A5AC0208059F020847
:10001000C9AA0208D5180208C1050308000000009B
:10002000000000000000000000000000E5C402081D
:10003000C31D02080000000011B20208ADDC020876
:10004000C3010208C3010208C3010208C301020878
:10005000C3010208C3010208E1420208F742020894
:10006000C3010208C3010208C3010208C301020858
:10007000C3010208C3010208C3010208C301020848
:10008000491C0208591C0208C301020800000000B4
:100090000000000000000000000000000143020812
:1000A000C3010208C3010208C3010208C301020818
:1000B000C3010208BDDF0208C3010208C301020830
:1000C000C3010208C3010208C3010208C3010208F8
:1000D000C301020899F60208A9F602080000000010
:1000E000EB420208C3010208C3010208000000003D
:1000F000000000000000000000000000C301020832
:1001000000000000C3010208C3010208C301020885
:1001100000000000000000000000000000000000DF
:10012000691C0208791C0208891C0208C301020824
:10013000C3010208000000000000000000000000F1
:10014000000000000000000000000000C3010208E1
:10015000C3010208991C0208A91C0208B9F602088A
:10016000C3010208C30102080000000000000000F3
:10017000000000000000000000000000000000007F
:1001800000000000C30102080000000000000000A1
:10019000C3010208DFF80CD000F06AFC00480047F9
:1001A000051E0308D8F4002006488047064800478B
:1001B000FEE7FEE7FEE7FEE7FEE7FEE7FEE7FEE717
:1001C000FEE7FEE79DDD0208950102082DE9F05FDC
:1001D0000546002092469B468846064681464024B6
:1001E0001BE0284641464746224600F020F8534689
:1001F0005A46C01A914110D311461846224600F0C3
:10020000E3FA2D1A67EB01084F4622460120002130
:1002100000F0DAFA17EB00094E41201EA4F10104A8
:10022000DFDC484631462A464346BDE8F09F202A97
:1002300004DB203A21FA02F00021704721FA02F390
:10024000D040C2F12002914008431946704740EA6D
:1002500001039B0703D009E008C9121F08C0042A44
:10026000FAD203E011F8013B00F8013B521EF9D22B
:100270007047D2B201E000F8012B491EFBD2704753
:100280000022F6E710B513460A4604461946FFF762
:10029000F0FF204610BD421E12F8013F002BFBD19B
:1002A00011F8013B02F8013B002BF9D1704730B542
:1002B00005462A460B4612F8010B13F8014B08B10C
:1002C000A042F8D01CB1002802D06D1CF1E72846EE
:1002D00030BDCAB2401E10F8011F8A4202D0002968
:1002E000F9D100207047421C10F8011B0029FBD1F6
:1002F000801A704710B5002200E0521C835C8C5CB1
:10030000A34201D1002BF8D1D8B2E1B2401A10BDFE
:1003100030B504460020034600E05B1C934203D244
:10032000E05CCD5C401BF8D030BD034611F8012BDA
:1003300000F8012B002AF9D11846704730B5054660
:100340000020034600E05B1C934205D2EC5CC85CD5
:10035000201A01D1002CF6D130BD70B5064610F040
:100360009BFA046805460A220021304600F09CFAF8
:100370002C6070BD2DE9FE4F804681EA0300C00F5E
:100380000C46009021F0004123F00045B8EB02003C
:10039000A94105D24046214690461C460B460246DE
:1003A00023F00040104347D0270DC7F30A00C3F3E2
:1003B0000A510290401A019040286BDAC3F31300EF
:1003C00040F4801B0098924620B10023D2EB030A30
:1003D00063EB0B0B01985946C0F14002504600F008
:1003E000F3F906460D4650465946019A00F0FBF9CE
:1003F00010EB08006141002487EA115284EAE77398
:100400001A4340D0009A62B3019A012A4FEA075278
:1004100015DC001B61EB02014FF0004202EA0752BB
:10042000CDE90042001C41F5801132462B4600F018
:10043000B9FA03B0BDE8F08F40462146F9E7001B4A
:1004400061EB0201001C41F5801300185B4120188C
:10045000A2F5001747EB030140EAD570B6196D41CC
:1004600011E06D084FEA360645EAC0754FEA0752BB
:10047000001B61EB0201001C41F5801149084FEAA5
:1004800030000019514132462B4603B0BDE8F04F11
:1004900000F079BA0098012240000023D0EB02025C
:1004A00063EBE073009821464FEAE074B8EB00007C
:1004B00061EB0401E9E783F000435BE781F0004171
:1004C00058E72DE9FE4F81EA030404F0004421F0CF
:1004D000004100944FF0000B23F0004350EA010468
:1004E0005ED052EA03045BD0C3F30A54C1F30A5549
:1004F0002C44A4F2F3340194A0FB0254C1F3130181
:1005000041F48011C3F3130343F4801301FB02444D
:1005100000FB034E840A970A44EA815447EA835752
:10052000A4FB076802958D0A05FB07854FEA932C0B
:1005300004FB0C542705029D4FEA065847EA16377C
:10054000B5EB08056EEB070C870E920E47EA811794
:1005500042EA8312A7FB0201B6EB0B0164EB000435
:100560002B0D43EA0C335E1844EB1C50DA4651461F
:10057000E7FB0201C5F313044FEA0B3343EA1453BC
:100580004FEA0432019C43EA0603A4F10C040294EE
:10059000009CCDE900B400F005FA03B0BDE8F08F8F
:1005A00000200146F9E72DE9F04D81EA030404F04B
:1005B000004B21F0004514464FF0000A23F00041A3
:1005C00050EA050220D054EA01021DD0C5F30A57B3
:1005D0000246C5F31303C1F31300C1F30A5640F4F6
:1005E000801543F48013A7EB0608101BD64608F2CB
:1005F000FD3873EB050002D308F1010801E0921801
:100600005B41B8F1000F03DA00200146BDE8F08D30
:1006100000204FF48011064684460EE0171B73EB52
:10062000050705D3121B63EB050306434CEA010CD7
:1006300049084FEA300092185B4150EA0107EDD1BA
:1006400052EA030012D082EA040083EA050108435B
:1006500005D0101BAB4106D20122002306E0002288
:100660004FF0004302E06FF0010253101AEB060056
:100670004CEB085110EB0A0041EB0B01BDE8F04DCB
:1006800000F081B90EB540F2334102910021CDE96D
:1006900000110A460B4600F085F903B000BD70B5A5
:1006A000C1F30A5201F000450024C1F3130140F2E6
:1006B000FF3341F480119A4201DA002070BD40F20C
:1006C00033439A42A2F2334203DC5242FFF7AFFDBA
:1006D00000E090402C43F1D0404270BD00F0004259
:1006E00030F000400AD0C10D01F56071C0F3160072
:1006F00042EA0151C20840071143704700200146F9
:100700007047000030B5041E71F1000404DB4FF0A7
:100710000044404264EB0101141E73F1000405DB48
:100720001C464FF00043524263EB04038B4208BF68
:10073000824230BD30B5041E71F1000404DB4FF07D
:100740000044404264EB0101141E73F1000405DB18
:100750001C464FF00043524263EB0403994208BF2A
:10076000904230BD01F0004330B421F0004150EA26
:10077000010206D00A0DA2F56072C1F31301002A2E
:1007800002DC30BC00207047440F44EAC104C100C1
:10079000E01830BC00EBC25000F0BEB830B50B46DC
:1007A000014600202022012409E021FA02F59D42A1
:1007B00005D303FA02F5491B04FA02F52844151E75
:1007C000A2F10102F1DC30BD202A04DB203A00FA5C
:1007D00002F1002070479140C2F1200320FA03F398
:1007E000194390407047202A06DBCB17203A41FA84
:1007F00002F043EAE07306E041FA02F3D040C2F1AE
:100800002002914008431946704700000FB40023AE
:1008100000B589B00CA900910B996FF00042CB6034
:100820001E4B06931E4B07930423CDE901321D4A4C
:10083000089202466B46002000F0CEF909B05DF840
:1008400014FB70B586B006464FF0FF300091CDE93D
:100850000101002015460C4604903246694604A862
:10086000FFF7D4FF02460498211825B108B10846C5
:1008700000E020462860049800280DD0002A02DD00
:100880000098884208D0081B0094CDE90104324644
:10089000694604A8FFF7BAFF06B070BD110E020842
:1008A0002F0E02089D0A02082DE9F04791460F46D7
:1008B00080460446002614F8015B2DB100F0EAF8EA
:1008C0000068405DC007F6D12B2D02D02D2D18D029
:1008D000641E4A463946204600F0BAFA27B1396804
:1008E000A14201D1C7F8008071054FF002040BD579
:1008F0004042002803DD0FF0CFFF0460A007BDE8F1
:10090000F08746F48066E4E70028F8DA0FF0C4FFC9
:1009100004606FF00040F2E70029A8BF7047401C58
:10092000490008BF20F00100704710B4B0FA80FC05
:1009300000FA0CF050EA010404BF10BC704749B142
:10094000CCF1200421FA04F411FA0CF118BF0121B2
:1009500021430843A3EB0C01CB1D4FEA00614FEA92
:10096000102042BF002010BC704700EBC350104461
:100970000029A4BF10BC7047401C490008BF20F0EC
:10098000010010BC704710B5141E73F1000408DAA2
:10099000401C41F1000192185B411A4301D120F043
:1009A000010010BD2DE9F04D92469B4611B1B1FA00
:1009B00081F202E0B0FA80F220329046FFF704FFA5
:1009C00004460F4640EA0A0041EA0B0153465A46E4
:1009D000084313D0114653EA010019D0C8F1400270
:1009E0005046FFF724FC05460E46504659464246FF
:1009F000FFF7EAFE084305D0012004E0204639460F
:100A0000BDE8F08D0020054346EAE0762C433743ED
:100A10000A986305E40AA0EB08000022FD0A44EAF4
:100A200047540A3002D500200146E9E701051019B4
:100A30006941DDE9084500196941BDE8F04DA2E7CB
:100A4000C1F30A52C1F3130140F2FF3341F48011A4
:100A50009A4202DA00200146704740F233439A423C
:100A6000A2F2334202DC5242FFF7E1BBFFF7ACBE19
:100A7000064C074D06E0E06840F0010394E80700EB
:100A800098471034AC42F6D3FFF788FB20390308AF
:100A90004039030800487047802B030810B504460E
:100AA000FFF7F8FF0068005D00F0010010BD0000D6
:100AB0002DE9FF4F087883B09946FF2805D0491CDF
:100AC0002D2804D00024002008E000200BE00124A1
:100AD000F9E700EB800003EB4000491C0B78FF2B8B
:100AE000F7D104B1404200230293147819461D4601
:100AF0002D2C01D02B2C04D1521C2D2C13D00024D2
:100B00000294AA461478FF2C0FD00A25A3FB05787F
:100B100001FB05814FF0000C03FB0C11521CE31983
:100B20004AEB0101EEE70124EAE7814453EA0100C0
:100B300002D019F5C87F06DA03980021C0E9001138
:100B400007B0BDE8F08F0025AE4E2F46DFF8B88223
:100B5000184600F0DAF9CDE90001B9F1000002DA37
:100B6000C9F1000400E004460023A74A1AEB030B76
:100B700042EB045A12E0E00707D02A4633463846D3
:100B80004146FFF79EFC074688462A4633461046F4
:100B90001946FFF796FC05460E466410002CEAD174
:100BA000DDE90001B9F1000F5A46534606DAFFF7B6
:100BB000FAFC3A464346FFF7F6FC05E0FFF781FCF6
:100BC0003A464346FFF77DFC029A0AB181F00041A4
:100BD000039AC2E90001B3E72DE9FF4F1F468DB02C
:100BE000D7E901464FF0FF382E2045464FF0000967
:100BF0000B90B9696D1C0E988847396A8246884700
:100C00000028F6D1BAF1FF3F0AD024F4D064002EB8
:100C100011DDBAF12B0F08D0BAF12D0F0BD102E084
:100C2000404611B08DE744F48064B9696D1C0E989C
:100C300088478246761E6946600501D52D2000E072
:100C40002B208DF8000001F1010B0DF1200809E0C7
:100C5000B9696D1C0E98884782460F9844F4007459
:100C6000761E0560002E02DDBAF1300FF0D00B9930
:100C70008A453ED144F0800406E00F99681CA9F132
:100C8000010944F400740860B9696D1C761E0E9861
:100C9000884782463028F0D02BE00B998A4505D151
:100CA000200603D444F08004761E18E050460FF06E
:100CB000C9FF08B30DF11301761E44F400748B458F
:100CC00008D2AAF130000BF8010B200607D5A9F1D4
:100CD000010003E0200602D409F101008146A005CD
:100CE00002D50F99681C0860B9696D1C0E98884779
:100CF0008246002ED1DC53E0002E51DDBAF1650FA3
:100D000002D0BAF1450F4BD1A00549D5B9696D1C88
:100D100024F44074761E0E9888478246002E0CDD1F
:100D20002B2804D0BAF12D0F07D144F48074B9698F
:100D30006D1C0E9888478246761EE00501D52D2150
:100D400000E02B2108F8011BCDF82C8021E00DF1EB
:100D50002901761E44F4007488450CD2AAF13000B3
:100D600010F0FF0088F8000002D10B99884509D9DE
:100D700008F1010806E0E00501D5244801E042F24F
:100D80000F708146B9696D1C0E98884782460F988E
:100D90000560002E04DD50460FF054FF0028D6D128
:100DA000F9690E988847FF208BF8000088F800004A
:100DB0000020069007904B466A4608A906A8FFF750
:100DC00077FEA00502D46FF001002AE714F0240F8B
:100DD0000AD0E00714D1DDE906123868031D3B6034
:100DE0000068C0E900120BE0DDE90601FFF7BAFC7C
:100DF0000146E00704D13868021D3A6000680160CE
:100E000028460EE7000014400000F03FF1D8FFFF35
:100E1000426842B1016811F8013B23B1521EC0E99A
:100E20000012184670470121C160881E7047426851
:100E30005AB1C368016843B983688B4205D0491E23
:100E4000521CC0E90012002070474FF0FF3070477D
:100E50002DE9F05F82460078002715468B460AF19F
:100E60000104B946302801D09DB113E014F8010BFC
:100E70000127782803D0582801D045B10AE00DB1E8
:100E8000102D07D10027102514F8010B02E00825CA
:100E900000E00A250026B0460EE005FB080005FB31
:100EA00006F1012701EB10461FFA80F8B6F5803FE6
:100EB00000D3B94614F8010B294600F018F80028B1
:100EC000EBDABBF1000F05D00FB1641E00E0544611
:100ED000CBF80040B9F1000F06D00FF0DDFC022185
:100EE0000160C81EBDE8F09F48EA0640FAE73A28CC
:100EF00000D2303820F02002412A01D3A2F137007D
:100F0000884201D34FF0FF3070470EB540F23342B4
:100F100002920022CDE900221346FFF743FD03B001
:100F200000BD70B58C1810F8015B15F0070301D1F6
:100F300010F8013B2A1106D110F8012B03E010F83C
:100F4000016B01F8016B5B1EF9D12B0705D400235F
:100F5000521E0DD401F8013BFAE710F8013BCB1A01
:100F6000921C03E013F8015B01F8015B521EF9D5F6
:100F7000A142D8D3002070BD70B50546AC6B206C83
:100F800000F0500050BB206C40F4007020642068DA
:100F9000806800F04050E8B9A069D8B92068C06AFC
:100FA00000F4700020B12068806800F4806088B987
:100FB0002068406820F0200021684860206C20F400
:100FC00080702064206C00F4805018B9206C40F0D0
:100FD00001002064204604F005F903E0A06BC16C19
:100FE0002846884770BD70B50546AC6B402020642C
:100FF000606C40F004006064204604F0F5F870BDB9
:1010000070B50446A56B284604F0EDF870BD0000ED
:10101000014600220023022901DB00207047002244
:1010200006E0064800EB820030F811000344521C31
:10103000642AF6D36420B3FBF0F0EFE7F4E200207B
:1010400010B5C82202490348006804F061F910BDD8
:10105000F4E200204006002054494A6822F440325D
:101060004A604A6843681A434A600268526822F438
:10107000807203685A6002685368026943EA022278
:1010800003685A600268526822F0407203685A602E
:101090000268526883681A4303685A60026892685B
:1010A00022F4006203689A6002689268C3681A4377
:1010B00003689A603E4B826A9A4218D0026892682E
:1010C00022F0706203689A6002689268836A1A4329
:1010D00003689A600268926822F0405203689A603E
:1010E00002689268C36A1A4303689A600BE0026858
:1010F000926822F0706203689A600268926822F037
:10110000405203689A600268926822F00202036803
:101110009A6002689368826943EA420203689A60AF
:10112000026AA2B10268526842F4006203685A601F
:101130000268526822F4604203685A600268536889
:10114000426A521E43EA423203685A6005E002686E
:10115000526822F4006203685A600268D26A22F47C
:1011600070020368DA620268D36A828B521E43EA15
:1011700002520368DA620268926822F4007203681D
:101180009A6002689368026B43EA422203689A609D
:101190000268926822F4806203689A600268936829
:1011A000426943EA822203689A6070470023014043
:1011B0000100000F01490860704700004006002050
:1011C00010B500200E49088000F050FC09F088F8A6
:1011D00008F0F8F906F092FF09F08CF803F096FC9D
:1011E0000EF06CF90748B0F85600012801D10CF058
:1011F00049FE0AF037F80AF00DF80FF0C1FA10BDF9
:101200001E0000209824002008B500200AF082FE6D
:1012100010F0BEFF0AF0DAFA00F0F0FB0BF018FC59
:10122000FFF70EFF00F054F809F040F81248B0F84C
:101230005600012802D10CF013FE08E00E48B0F869
:101240005600022803D109F019FE09F02DFD03F024
:10125000A5FA0EF025F911F097F8084808F07CF986
:101260000020074B4FF47A72012100900348006878
:1012700008F0FEF908BD00009824002000000020BE
:10128000ADB1020810B5FFF79BFF0E4800780E497C
:10129000097888420ED00C4800780A490870084640
:1012A000007810B10EF03AFA04E000200749086017
:1012B00010F002FA0348007808B111F083F808F042
:1012C000B7FF10BD2E0000202D0000206406002076
:1012D00010B5012010F063FE0D4908700846007833
:1012E000132802D110F094FE10E00A4809F04EF8DD
:1012F000084800780649087008460078332802D16B
:1013000009F012F802E000200349C88710BD000070
:10131000540600205506002098240020F8B500212E
:101320000F2010F027FB7F49086000217E4810F055
:10133000BBFB7C48008800F4804000287ED04FF43E
:10134000804200210F2010F0B0FC0021102010F08E
:1013500011FB76490870084600787549087000222C
:1013600072480178734810F059FB73487149B1F81D
:101370000110018071486F49B1F8051001806D4876
:1013800000786F49097888427ED16A48407A2028DF
:10139000FAD16848C0786B490870664800796A4994
:1013A00008706448807A6949087064486149B1F8F6
:1013B000051001806548007842005E490B316448A1
:1013C000FEF745FF61480078420060480078400021
:1013D0000B30584BC1185F48FEF739FF5B48007867
:1013E0000B2101EB8000534901445B4809880180CF
:1013F00000205A490880022059490870002519E048
:10140000534830F8150057490968884210D15648AA
:1014100090ED000B51EC100BFFF741F940B2464242
:101420004C4830F915103246444800880AF004FC54
:10143000681CC5B245480078854200E060E0DFDB0B
:101440003E48008800F09EFA4849088048480088D5
:10145000B0F5967F1CDB084600884549098888421C
:1014600013D14348008841490880344802884048E5
:1014700001880088401C3E4B18803E4820F811200F
:1014800001203D49087003E039E000203A49087026
:101490002E4800783949097888420BDD2B480078BE
:1014A0003649087029480078420022490B313448F7
:1014B000FEF7CDFE002414E00B2000EB44001D4994
:1014C000084400880090BDF8000026490968884259
:1014D00005D100202B490870204600F057F8601C09
:1014E000C4B21A4800788442E6DB18480078844287
:1014F0000BD1012023490870204600F047F804E092
:10150000214A00210F2010F0D0FB10F0EDF801214E
:10151000054810F0C9FA002010F00CFB002010F074
:1015200091FAF8BD5002002000D023245C02002074
:101530005D020020104400206402002066020020AA
:10154000D70100206E0200206F02002071020020EF
:10155000EC490020444C0020740200200A000020C6
:101560001A020020CC010020E802002078020020AE
:10157000760200209C4E00205F02002072020020B4
:101580003C450020600200200090272410B504464E
:101590006E4800686E4908806E4804706E486F4956
:1015A0000988A0F801106E490988C1816849098835
:1015B00001826C4800786849C87108466A49098800
:1015C000A0F8051010F008FC684A03C268480078CB
:1015D000A04223D107F0F0FF642190FBF1F201FB60
:1015E0001200644908806248007800EB8000098896
:1015F00001EB800000F29E2004EBC40101EB04111A
:1016000000EB01100004C117584B0CCB8018594156
:10161000000A40EA01605849086018E05448007820
:1016200000EB800040F29E2101EB800004EBC4013E
:1016300001EB041100EB01100004C1174B4B0CCB64
:1016400080185941000A40EA01604B4908604A4845
:10165000006810F021FA46490978491C091B01EB82
:10166000C10202EB01110A2202EB011010F047FA4D
:101670004148006820F001000021090241EA1061A0
:1016800000023E4A03C239480CC833481A3010F0F1
:1016900027FE3A480CC830481E3010F021FE0020CA
:1016A000374988812C48898941843648007878B147
:1016B00035483649364A128841F8220008463449EE
:1016C000098800EB810124480968C0F80A1008E085
:1016D0002E482F49098800EB81011F480968C0F88E
:1016E0000A102C4800781C4908702B480078887430
:1016F000212048720846C574C07C00F00F00C874F1
:1017000000223C2010F01DFB00213C2010F02CFB9F
:10171000012010F04DFA214908700020204908707E
:101720001E48007880B904E01D480078052800DDD7
:1017300009E000210F2010F01DF91A49086000F09F
:1017400080000028F0D000BF10BD0000240400403D
:101750007A0200206B020020A6440020CC01002069
:101760001C000020EA010020660200208002002008
:101770007102002042030020540200204002002099
:10178000982400205F020020FFFF01004C5300203E
:1017900078020020D70100206802002061020020AA
:1017A00020060020500200200148008870470000F9
:1017B000A405002010B500F003F8002010BD0000C3
:1017C00010B52648FFF7F6FC254900200AF01AFE5E
:1017D000002108460AF0F8FC2023224A002108468E
:1017E0000AF05CFC2023204A032100200AF056FC6A
:1017F00040231D4A012100200AF050FC80231A4A90
:10180000022100200AF04AFC184900200EF056FC84
:10181000174901200EF052FC164902200EF04EFC32
:101820004FF480620F49002001F0F4F801220D49C5
:10183000022001F0EFF84FF480520A49012001F034
:10184000E9F840220C49002003F056F94FF4805289
:101850000549012003F050F9002010BDC0E400202C
:1018600068E50020000402400000024038E6002045
:10187000B8E6002078E600200008024010B51148C4
:101880000088002802DD01200F4908800E480088EA
:10189000B8B10C48008800280CDD0A480088401EBA
:1018A000084908800120094908700C21084805F002
:1018B000DBFD06E00020054908700C21044805F016
:1018C000F3FD10BD040000200600002009000020E8
:1018D000C0E5002000BFFEE710B504460021024825
:1018E00009F004F910BD000091D5020810B50246B8
:1018F0000B460020002103E0545C0444A0B2491CC4
:101900009942F9D3C443A0B210BD00002DE9F041C3
:1019100004460D4616460748006838B10648324668
:10192000294603682046034F3F68B8470020BDE8BA
:10193000F0810000680500206C05002010B5002033
:10194000074908700749086009F0DEFD00224FF4DE
:101950008051054804F03EFA00F008F810BD000080
:1019600016020020680600200000024010B5002189
:10197000034810F099F80FF0B7FE0FF09DFE10BD70
:1019800000D0232431B500240AE00A4800EB4401CA
:1019900002226846FEF7BCFC00B905E0601C84B278
:1019A000054800888442F0DB00BF00200349085549
:1019B000204638BD9C4E0020760200202052002098
:1019C0000EB50021084A0948CDE901210090A0F296
:1019D000E220B0F8A01200F2C22300F2A22200F529
:1019E000207009F0EBF90EBD11AD02087A27002036
:1019F00001480078704700007D03002000B587B0E3
:101A00001C216846FEF73CFC00208DF801000220F6
:101A10008DF800000F4801904FF480700290C000D4
:101A2000049040200590694600200EF0E7F80A482F
:101A30000A49C1F890050A48C1F89C050948C1F84F
:101A400098050948C1F89405084607F063FC07B0FB
:101A500000BD0000F46D0020CB1B0208546800207C
:101A6000BD1B0208051C0208191C02081CB5FFF763
:101A7000BFFF10B907F0C0FB97E0FFF7B9FF0128DF
:101A80002FD1002001900090694602200EF0A2F8AC
:101A900020E09DF80400032812D14448006850B1AA
:101AA00007F08AFD41490968401AC8280BD900206F
:101AB00000F0C2F807E007F07FFD3C49086002E053
:101AC00000203A4908604FF47A73012201A9009876
:101AD00006F029F901A900200DF0BEFF0028D8D09A
:101AE00063E0FFF785FF02282FD1002001900090CE
:101AF000694602200EF06EF820E09DF804000328ED
:101B000015D12B48006868B107F056FD28490968CF
:101B1000401AC8280ED9012026490870002000F07C
:101B20008BF807E007F048FD2149086002E000203B
:101B30001F4908609DF804000EF044FD01A9002033
:101B40000DF08AFF0028D8D02FE0FFF751FF0328BF
:101B50002BD100200190002420E09DF804000328F0
:101B600015D11548006868B107F026FD12490968CB
:101B7000401AC8280ED901200E490870002000F034
:101B80005BF807E007F018FD0B49086002E0002051
:101B9000094908609DF804000EF014FD01A9002019
:101BA0000DF05AFF0028D8D000BF1CBD80030020D4
:101BB000840300207E0300208803002010B5044623
:101BC000214600200DF048FF10BD0FB410B5ADF553
:101BD000027D85A881904FF4007101A8819B849AB1
:101BE0000EF044FE0020819001A8FEF77CFB044625
:101BF000224601A900200EF01BFB0DF5027D10BC52
:101C00005DF814FB31B500240122694600200EF076
:101C10000FFB0446204638BD70B50446002520461B
:101C2000FEF761FB06463246214600200EF000FB1F
:101C30000546284670BD000001460248017000209C
:101C4000704700007D03002010B5024803F04AFCF5
:101C500010BD0000B8E7002010B5024803F042FCB8
:101C600010BD000018E8002010B5024803F03AFC4F
:101C700010BD000008E5002010B5024803F032FC5A
:101C800010BD000078E8002010B5024803F02AFCDF
:101C900010BD0000F8E6002010B5024803F022FC59
:101CA00010BD0000D8E8002010B5024803F01AFC6F
:101CB00010BD000058E700200146087810381823AE
:101CC000B0FBF3F20848805CC865032A05D90868B0
:101CD0006FF30900001D886503E008686FF30900D1
:101CE0008865886D70470000DE2A030801460020E1
:101CF0008A6A8B69CBB932B1012A0DD0022A03D08E
:101D0000032A10D10EE000BFCB6A03F08073B3F159
:101D1000807F00D1012007E0CB6AB3F1C07F00D102
:101D2000012001E000E000BF34E08B69B3F5005F03
:101D30001AD132B1012A07D0022A03D0032A11D1C5
:101D40000AE000BF01200EE0CB6A03F08073B3F11C
:101D5000807F00D1012006E0CB6AB3F1C07F00D1C3
:101D6000012000E000BF15E032B1012A05D0022AAF
:101D700004D0032A0CD103E000BF00BF012008E01B
:101D8000CB6A03F08073B3F1807F00D1012000E0C3
:101D900000BF00BF704730B50468246824F4802475
:101DA00005682C60046863608468402C04D1046872
:101DB000A2600468E16003E00468A1600468E26076
:101DC00030BD704701201A494872022019494872F3
:101DD00003201949487204201849487214481849C8
:101DE000097801701448164909780170114814499E
:101DF000097801700E4813490988A0F805100E48AB
:101E000010490988A0F805100A480E490988A0F869
:101E100001100A480B490988A0F801100A4809492D
:101E20000988A0F8011007490988A0F80510704733
:101E300084090020E2090020A6090020980900205A
:101E4000D7010020CC010020F809002010B509F0CE
:101E500095FF38200BF01CFF01200FF06DFC0820CF
:101E60000BF016FF0FF0A2FD0F4908600F48007835
:101E700018B10F480FF0E6FA02E00E480FF0E2FA50
:101E800001210D480FF010FE48F283000FF049FECB
:101E900000200FF085FE4FF47A700FF04BFE00200B
:101EA0000FF0D0FD10BD0000C4000020770100201D
:101EB000440000203900002000D023242DE9F04305
:101EC00091B007460D4614463C22934902A8FEF7FE
:101ED000BEF9D7F80880D8F83400D0F8009028462A
:101EE000362D73D013DC04283FD007DCC0B10128A5
:101EF00032D0022837D0032869D135E00E2867D0C8
:101F00000F2867D0152876D03528F5D1C6E03738A8
:101F100008285CD2DFE800F0C4C5C6C7C8C9CACB70
:101F200000207E4908607E4908607C48006800EB1C
:101F3000400002AB53F820207848006800EB4000D6
:101F400003EB80004168404606F020F874480068C2
:101F5000401C73490860DBE0404606F039F848460B
:101F600007F0E4FAD4E000BF00BF042D37D16B487E
:101F7000006800EB400002A901EB8000007A00F04D
:101F8000040030B300206649086064480068401CC3
:101F90006249086008460068052805D300226149A7
:101FA000384606F023FC10E05C48006800EB400077
:101FB00002AB53F820205948006800EB400003EBC7
:101FC00080004168404605F0E1FFA1E067E09DE048
:101FD00052E000E08EE0012011B0BDE8F0834F48F0
:101FE000006800EB400002A901EB80008068022D30
:101FF00002D1012101E06EE00221084018B3002067
:102000004749086045480068401C44490860084644
:102010000068052805D300224249384606F0E6FB51
:1020200029E03E48006800EB400002AB53F8202056
:102030003A48006800EB400003EB800041684046EE
:1020400005F0A4FF17E036480068401C34490860DA
:1020500008460068032805D300223349384606F0B5
:10206000C5FB08E00E203B4642F2107200210090B2
:10207000484606F09FFB4BE02848006800EB400014
:1020800002AB53F820202548006800EB400003EB2A
:1020900080004168404605F079FF39E000BF00BF8D
:1020A00000BF00BF00BF00BF00BF00BF00BF26468B
:1020B0001A48006810B101280AD104E0D6E90001ED
:1020C00008F096FD05E0D6E9000108F0A9FD00E062
:1020D00000BF00BF1CE026466B4614A2D6E90001F3
:1020E00007F0FCFB012800D012E0DDE9000108F058
:1020F0006DFD0DE0002008F009FD012805D100224A
:102100000D490E4806F072FB02E001E0012063E792
:1021100000BF002060E70000A42903080C05002090
:102120001005002044290308E42803082B434349F1
:10213000443A2025700D0A00D42803088CC30020DF
:102140002DE9F84304460D469046A668706B076873
:10215000032D78D005DC5DB1012D23D0022D6FD188
:1021600027E0042D70D00E2D6CD00F2DF7D1B3E0E9
:102170004FF46120614908600846016801200DF0B4
:10218000C1FE00205E4908705E4908605E49086033
:102190000E2023464FF47A7200210090384606F054
:1021A00009FBA8E0304605F013FF384607F0BEF9FA
:1021B000A1E053480078012812D14FF461204F4923
:1021C00008600846016801200DF09CFE0E202346A1
:1021D0004FF47A7200210090384606F0EBFA8AE05C
:1021E00000204949086047480068401C454908608C
:1021F00008460068032818D340480068B0F5E13F5E
:1022000009D101203E49087040A241F28831304690
:1022100005F0BCFE12E00321002008F08BFC002238
:102220003F49204606F0E2FA08E00E2023464FF42C
:102230007A7200210090384606F0BCFA5BE002E0BA
:1022400056E001E033E056E02F480068401C2E497C
:10225000086000202B4908602B480068052812D12F
:102260004FF4E130254908600846016801200DF06F
:1022700049FE0E2023464FF47A7200210090384622
:1022800006F098FA12E0204800680A2805D90022D2
:102290002449204606F0AAFA08E00E2023464FF40F
:1022A0007A7200210090384606F084FA23E0144840
:1022B0000078012809D10321002008F03BFC00220E
:1022C0001749204606F092FA15E017A241F288312C
:1022D000304605F05BFE0EE0002008F017FC0128F8
:1022E00005D100221249134806F080FA03E002E00B
:1022F0000120BDE8F88300BF0020FAE700050020B8
:1023000004050020F8040020FC04002041542B495F
:1023100050523D3932313630303B26570D0A0000DD
:1023200014290308E4280308415445300D0A00002D
:10233000D42803088CC300202DE9F04105460E4641
:102340001446AF6836B1012E16D0022E18D0032ED7
:102350001ED116E0A046FFF727FA10490880104961
:10236000D8F8040008600D4803880EA241F28831B5
:10237000384605F00BFE0EE0384605F029FE0AE06F
:1023800000BF002206480168284606F02FFA02E046
:102390000120BDE8F08100BF0020FAE7AC05002075
:1023A0001006002041542B434C564C3D25750D0A18
:1023B000000000002DE9F84305460E461446AF68BC
:1023C00036B1012E1ED0022E20D0032E26D11EE0C3
:1023D000A0460120144908701449D8F80400086088
:1023E00013480068006800901148006811A241F28B
:1023F00088314368384605F0C9FD0D4800680BF088
:1024000093FF0EE0384605F0E3FD0AE000BF00222E
:1024100006480168284606F0E9F902E00120BDE817
:10242000F88300BF0020FAE7AA0500201406002068
:10243000B405002041542B514C544F4E453D312C96
:10244000252E2A730D0A00002DE9F04105460E469F
:102450001446AF6836B1012E14D0022E1BD0032EC5
:1024600021D119E0A0461349D8F80400086012A24F
:1024700041F28831384605F089FD4FF48020124939
:10248000086013E0002011490870114908703846AF
:1024900005F09EFD0AE000BF0022064801682846BC
:1024A00006F0A4F902E00120BDE8F08100BF0020A1
:1024B000FAE700001806002041542B514C544F4EAF
:1024C000453D300D0A000000180C0240AA0500200E
:1024D000AB0500202DE9F84305460E461446AF68CB
:1024E00036B1012E1ED0022E20D0032E26D11EE0A2
:1024F000A0460120144908701449D8F80400086067
:1025000013480068006800901148006811A241F269
:1025100088314368384605F039FD0D4800680BF0F6
:1025200057FF0EE0384605F053FD0AE000BF0022D9
:1025300006480168284606F059F902E00120BDE886
:10254000F88300BF0020FAE7A80500200806002055
:10255000B005002041542B515454533D322C2225B8
:102560002E2A73220D0A00002DE9F04105460E4681
:102570001446AF6836B1012E14D0022E1BD0032EA4
:1025800021D119E0A0461349D8F80400086012A22E
:1025900041F28831384605F0F9FC4FF480201149AA
:1025A000086013E000201049087010490870384690
:1025B00005F00EFD0AE000BF00220648016828462B
:1025C00006F014F902E00120BDE8F08100BF002010
:1025D000FAE700000C06002041542B515454533D9F
:1025E000300D0A00180C0240A8050020A9050020A3
:1025F00010B50446FFF7D8F81D490988884204D071
:10260000204600F043F8002010BD1A48007858B961
:102610000BF09AFE184908600846006868B1204629
:1026200000F086F80020EFE714480078012804D174
:10263000204600F093F80020E6E71148007858B9EA
:102640000BF038FE0F4908600846006868B1204664
:1026500000F03AF80020D7E70B480078012804D1B1
:10266000204600F047F80020CEE74FF0FF30CBE7E0
:10267000AC050020A8050020B0050020A905002019
:10268000AA050020B4050020AB0500201CB50446B7
:1026900000200090E06B40680190E06B406840686B
:1026A00004494860002088606A46E06B06F09EF8A6
:1026B00000201CBDD8050020012002490870002020
:1026C00070470000AB0500201CB5044600200090B8
:1026D000E06B40680190E06B4068406804494860E6
:1026E000002088606A46E06B06F080F800201CBD80
:1026F000E80500201CB5044600200090E06B40680F
:102700000190E06B406840680449486000208860A0
:102710006A46E06B06F06AF800201CBDF805002050
:10272000012002490870002070470000A905002020
:102730001CB5044600200090E06B40680190E06BFF
:102740004068406804494860002088606A46E06B41
:1027500006F04CF800201CBDB80500201CB504464E
:1027600000200090E06B40680190E06B406840689A
:1027700004494860002088606A46E06B06F036F83D
:1027800000201CBDC80500202DE9F84305460E4673
:102790001446D5F80880022E18D003DC3EB1012E75
:1027A0002CD10FE0032E12D00A2E27D116E0274697
:1027B00015497868086015A241F28831404605F055
:1027C000E5FB1EE0404605F003FC1AE000BF0022D6
:1027D0000D480168284606F009F812E00020009034
:1027E00027466B460CA2D7E9000107F077F80228CC
:1027F00000D006E0009808F03FFA02E00120BDE8B2
:10280000F88300BF0020FAE77804002041542B43EE
:1028100053510D0A000000002B4353513A20256408
:102820002C252A0D0A0000001CB50446002000904B
:10283000E06B40680190E06B406840680449486084
:10284000002088606A46E06B05F0D0FF00201CBDC8
:102850006804002010B5044608F006FA012802D1E9
:102860002046FFF7E1FF4FF0FF3010BD2DE9F041AA
:1028700004460D461746A66835B1012D0BD0022D32
:102880000DD0032D16D10BE00DA241F28831304658
:1028900005F07CFB11E0304605F09AFB0DE000BF2F
:1028A0000221084608F046F900220849204605F0B2
:1028B0009DFF02E00120BDE8F08100BF0020FAE7A3
:1028C00041542B4346554E3D300D0A003429030830
:1028D0007FB5E0B005460E46144622464FF4C0715F
:1028E0006846639B0DF0C2FF684605F0CDFD0020F1
:1028F00064B070BD00B595B000208DF8390002209D
:102900008DF8380025480F904FF42060109024482F
:10291000119004201290102013900EA901200DF0A8
:102920006DF918B14FF0FF3015B000BD1D4806F02D
:1029300013FE10B14FF0FF30F6E71B4803901B4821
:102940000490382005901A4806901A4807901A48B3
:1029500008901A4809904FF4C0600A9018480B90EC
:102960004FF4C0600C900F480D9003A9154805F076
:102970005BFB10B14FF0FF30D6E701201149124B3D
:1029800012A2CDE900101349074805F0D1FE124903
:10299000054805F007FF0020C6E70000F4AC002062
:1029A0007C040020800400208CC30020F82503084C
:1029B000AD3D02088D3F0208253E0208F4B6002016
:1029C000F4BC0020F4C20020B82703084543363089
:1029D00030530000B4280308D128020810B5054878
:1029E000006928B1034A918A1069012203F0F2F9C3
:1029F000002010BD74C3002010B50548006928B13F
:102A0000034A918A1069002203F0E4F9002010BD06
:102A100074C300200346044840F8331000EBC300A1
:102A2000828000207047000074C3002010B5054864
:102A3000006828B1034A91881068002203F0CAF99F
:102A4000002010BD74C3002010B50548006828B1EF
:102A5000034A91881068012203F0BCF9002010BDE0
:102A600074C300202DE9F04105460E461446D5F802
:102A7000088036B1012E0ED0022E10D0092E26D19C
:102A80001DE000201549086015A241F2883140463A
:102A900005F07CFA1EE0404605F09AFA1AE00F486D
:102AA0000068012805D100221049284605F09EFE45
:102AB00004E000220E49284605F098FE0AE0274669
:102AC000064B0CA2D7E9000106F008FF02E0012046
:102AD000BDE8F08100BF0020FAE7000030050020CB
:102AE00041542B43474154543F0D0A0084290308A5
:102AF000442903082B43474154543A2025640000DD
:102B00002DE9F04393B005460C469146002720215D
:102B10000BA8FDF7B5FBAE68706BD0F800802422DF
:102B20008D4902A8FDF793FB07F0D8FF0746052261
:102B30008AA13846FDF702FC28B1052289A1384652
:102B4000FDF7FCFB28B989A220210BA806F0B9FFEC
:102B500022E0052287A13846FDF7F0FB28B987A2BD
:102B600020210BA806F0ADFF16E0052285A138460E
:102B7000FDF7E4FB28B97DA220210BA806F0A1FFF8
:102B80000AE0052281A13846FDF7D8FB20B981A2D1
:102B900020210BA806F095FF032C31D005DC5CB199
:102BA000012C25D0022C7DD129E0042C29D00E2C1B
:102BB00079D00F2CF7D1C8E0002078490860784917
:102BC00008607648006800EB400002AB53F8202014
:102BD0007248006800EB400003EB8000416830461B
:102BE00005F0D4F96E480068401C6D490860AFE0FC
:102BF000304605F0EDF9404606F098FCA8E000BF2D
:102C000000BF042C33D16548006800EB400002A9E6
:102C100001EB8000007A00F0040020B3002060493E
:102C200008605E480068401C5C490860084600680F
:102C3000032805D300225B49284605F0D7FD11E0A3
:102C40005648006800EB400002AB53F82020534880
:102C5000006800EB400003EB80000BAB416830469E
:102C600005F094F974E0012013B0BDE8F083022C64
:102C70000AD14A48006800EB400002A901EB80003D
:102C8000007A00F0010060B9032C32D1434800689B
:102C900000EB400002A901EB8000007A00F0020086
:102CA00038B301E052E03DE000203D4908603B4878
:102CB0000068401C3949086008460068032805D3AD
:102CC00000223849284605F091FD2AE03348006883
:102CD00000EB400002AB53F820203048006800EBC6
:102CE000400003EB80000BAB4168304605F04EF925
:102CF00017E02B480068401C294908600846006816
:102D0000032805D300222849284605F06FFD08E076
:102D10000E202B4642F2107200210090404605F032
:102D200049FD15E01D48006800EB400002AB53F878
:102D300020201A48006800EB400003EB80000BAB3A
:102D40004168304605F022F902E001E001208BE7FE
:102D500000BF002088E70000E02903083436303047
:102D6000300000003436303032000000434D4E4514
:102D7000540000003436303031000000554E494ECA
:102D800045540000343630303600000034363030E0
:102D90003300000043544E45540000002805002035
:102DA0002C05002074290308B42803082DE9F041FC
:102DB00004460D461746A66825B1012D03D00F2DF8
:102DC00015D101E016E015E00C480078012808D183
:102DD00000200A49087000220949204605F006FD36
:102DE00008E0304601F06CF800B903E002E0012091
:102DF000BDE8F08100BF0020FAE700009804002041
:102E000044290308F8B507460D4614460F2D0FD088
:102E100005DC4DB1012D08D0042D24D109E01A2D77
:102E20000DD0272D1FD11AE01FE00AF065FC1CE031
:102E30001BE000220E49384605F0D8FC15E0264676
:102E4000002000906B460BA2D6E9000106F046FD7B
:102E5000012800D009E000980AF072FD05E0012089
:102E60000A49087001E00120F8BD00BF0020FBE71F
:102E7000C42803082B51495552433A2022636C6FF2
:102E8000736564222C25640D0A000000980400205C
:102E90002DE9F04104460D461746A66825B1012DDF
:102EA00003D00F2D06D101E007E006E0304600F028
:102EB000E3FF02E00120BDE8F08100BF0020FAE757
:102EC00070B505460C46164624B1012C03D0042CDF
:102ED00008D101E008E007E000220549284605F096
:102EE00085FC01E0012070BD00BF0020FBE7000071
:102EF000C42803082DE9F04104460D461746A6688C
:102F000035B1012D0BD0022D0DD0032D16D10BE0C4
:102F10000DA241F28831304605F038F811E0304614
:102F200005F056F80DE000BF0321022007F002FE75
:102F300000220849204605F059FC02E00120BDE8C6
:102F4000F08100BF0020FAE741542B4346554E3D27
:102F5000310D0A004429030870B505460C46164693
:102F600024B1012C09D00F2C1CD107E0FFF75EFD26
:102F70000221002007F0DEFD16E015E0002007F03A
:102F8000C5FD012803D10221002007F0D3FD002058
:102F900007F0C6FD012804D100220549284605F0A6
:102FA00025FC01E0012070BD00BF0020FBE7000010
:102FB000E42803082DE9F84305460E469046AC6820
:102FC000606B076826B1012E1AD00E2E60D11BE06F
:102FD0000020E06200BF2046216988470028FAD01F
:102FE0000020E0622D490870FFF720FD0E202B46DF
:102FF00040F6B83200210090384605F0DBFB4AE08D
:10300000384606F093FA46E02448007830B10128AB
:1030100013D0022825D0032838D131E001201F49E0
:103020000870FFF711FD0E202B464FF47A72002135
:103030000090384605F0BEFB28E0022017490870D2
:10304000FFF7CCFC4FF4612101200CF05BFF0E2058
:103050002B464FF47A7200210090384605F0AAFB07
:1030600014E003200D490870FFF7C6FC0E202B4624
:103070004FF4487200210090384605F09BFB05E0B4
:1030800000220749284605F0B1FB00BF00BF02E05F
:103090000120BDE8F88300BF0020FAE7DC0400202F
:1030A000F4280308F8B507460D461446142D13D02E
:1030B00005DC4DB1012D08D0042D31D106E0332DB2
:1030C0001AD0342D2CD121E02CE02BE0002217491E
:1030D000384605F08BFB25E02646002000906B4625
:1030E00013A2D6E9000106F0F9FB012800D019E08F
:1030F00000980AF0FFFB15E0264612A13068FDF7A4
:10310000F9F800B10EE0FFF70BFB0BE0264610A12B
:103110003068FDF7EFF800B104E0FFF7CDFA01E009
:103120000120F8BD00BF0020FBE70000C428030811
:103130002B51495552433A202272656376222C2541
:10314000640000002B515454533A20300D0A000003
:103150002B514C544F4E453A20300D0A00000000D0
:10316000034611B1012902D100E002E001E0012093
:10317000704700BF0020FBE72DE9F04105460C46F3
:103180001646AF68052C1FD2DFE804F0030E1213B9
:10319000140007F0A7FC804643460EA241F2883196
:1031A000384604F0F3FE12E0384604F011FF0EE05A
:1031B00000BF00BF304607F005FD08480022416807
:1031C000284605F013FB02E00120BDE8F08100BFB6
:1031D0000020FAE725730D0A00000000A00400207B
:1031E0002DE9F84304460E461546A768786BD0F8DB
:1031F0000090072E74D005DC5EB1012E1AD0022E8D
:103200006FD11EE0082E6DD00E2E6CD00F2EF7D190
:10321000C5E000206849087068490860684908608E
:1032200001206849087068A241F28831384604F0EC
:10323000ADFEBEE0384604F0CBFE484606F076F917
:10324000B7E05D480078A8BB00205E4908705C4884
:103250000068012803D05A480068052811D10120D0
:1032600055490870002055490860554908600120FB
:103270005449087057A241F28831384604F086FE5E
:103280004EE04E480068401C4C4908600846006803
:10329000642805D900225249204605F0A7FA88E0A3
:1032A0000E2023464FF4FA6200210090484605F0B4
:1032B00081FA35E0FFE740480078012830D100204E
:1032C000404908703E480068012803D03C48006827
:1032D000052809D143480068401C424908600BE0BA
:1032E0001FE063E02BE039E000203E4908603348EE
:1032F0000068401C314908603A480068032805D33B
:1033000000223949204605F071FA08E00E202346D4
:103310004FF4FA6200210090484605F04BFA00BFD6
:1033200047E0A8462448007840B9254B2FA2D8E9A9
:10333000000106F0D3FA022800D03AE039E0A846AE
:103340001D480078012808D11D4B2CA2D8E90001A6
:1033500006F0C4FA022800D02BE02AE016480078D4
:1033600060B900201649086001201649087027A29C
:1033700041F28831384604F009FE0FE00E4800782B
:1033800001280BD100200E49086001200D4908706A
:1033900010A241F28831384604F0F8FD09E00948EE
:1033A000007810B9384600F067FD02E00120BDE862
:1033B000F88300BF0020FAE7140500201C05002058
:1033C000180500202405002041542B434552454751
:1033D0003F0D0A0041542B43475245473F0D0A0019
:1033E000C428030820050020642903082B43455204
:1033F00045473A20252A2C25640000002B434752DC
:1034000045473A20252A2C256400000041542B43CF
:103410005245473F0D0A00002DE9F04104460D4694
:103420001646A76835B1012D0ED0022D11D0032DFF
:1034300019D10DE00F4806600FA243F698210368EA
:10344000384604F0A3FD11E0384604F0C1FD0DE05C
:1034500000BF084800680AF073FA00220B492046B2
:1034600005F0C4F902E00120BDE8F08100BF0020B2
:10347000FAE700004005002041542B5149434C4FCE
:1034800053453D25642C31300D0A00008429030882
:103490002DE9FE4F05460E461446AF68786BD0F80E
:1034A0000090032E3CD005DC4EB1012E30D0022E10
:1034B00074D134E00E2E72D0162EF9D14BE046486E
:1034C000046000680AF0C6F98046434800680AF0C4
:1034D000AFF98246404800680AF0ECF9012801D1B2
:1034E0003EA000E03EA08346CDE901A800903A4806
:1034F0003CA241F288310368384604F047FD0E20B3
:103500002B46414A00210090484605F053F95FE000
:10351000384604F05DFD484606F008F858E057E0EC
:103520002D4800680AF030FA38480068401C3749D6
:10353000086008460068032807D3002008600022BE
:103540003349284605F052F904E000223149284663
:1035500005F04CF93CE0A04600200290019001A843
:10356000009002AB2CA2D8E9000106F0B7F90228BE
:1035700000D02DE018480068029988421ED10198B9
:1035800070B9002021490860134800680AF01AFA4F
:1035900000222049284605F029F90FE015E00EE049
:1035A0000D4800680AF0F0F918480068401C1749F7
:1035B000086000221749284605F018F908E00022A3
:1035C0001449284605F012F902E00120BDE8FE8FFB
:1035D00000BF0020FAE700003805002054435000E7
:1035E0005544500041542B51494F50454E3D312CCC
:1035F00025642C222573222C222573222C25752C40
:10360000302C300D0A00000020BF02003C050020D5
:10361000B4280308842903082B51494F50454E3ADA
:103620002025642C25640D0A000000002DE9FC41D2
:1036300006460F461446D6F80880022F25D003DC34
:103640003FB1012F57D10EE0032F10D01B2F52D1C5
:1036500021E02C4804602CA241F2883103684046E6
:1036600004F094FC4AE0404604F0B2FC46E02548F1
:1036700000680AF053F9234800680AF061F9002253
:103680002649304605F0B2F838E00022234930469A
:1036900005F0ACF832E0002001902546009001AB27
:1036A0001FA2D5E9000106F019F9012804D0154838
:1036B00000680AF033F921E0019820B91148006848
:1036C0000AF02CF91AE06B4618A2D5E9000106F0C1
:1036D00005F9022804D00B4800680AF01FF90DE034
:1036E0000848DDE9001200680AF018FA0548006889
:1036F0000AF0A2F902E00120BDE8FC8100BF002031
:10370000FAE700004405002041542B514952443D42
:1037100025642C313032340D0A000000842903085E
:103720002B514952443A2025640D0A002B5149522D
:10373000443A20252A0D0A25650000002DE9F043B2
:1037400085B005460E461446AF68786BD0F80090F9
:10375000032E50D005DC4EB1012E1CD0022E74D1A8
:1037600020E00E2E7DD0172EF9D153E0454804609D
:1037700000204549087005F01FFF4449414A12687E
:1037800041F822003F4842A241F28831036838469E
:1037900004F0FCFB72E0384604F01AFC484605F0E1
:1037A000C5FE6BE03848007801280AD100203D4969
:1037B000344A1268885400223B49284605F016F81E
:1037C00018E005F0F9FE39492E4A126851F8221026
:1037D000401A3749884208D32A4800680AF0B0F8EE
:1037E00000203049274A1268885400222E49284672
:1037F00004F0FCFF42E000202A49224A1268885463
:10380000204800680AF09CF800222749284604F066
:10381000EDFF33E00020049003900290A04602A840
:1038200003A9CDE9001004AB22A2D8E9000106F0FB
:1038300055F803280BD0134800680AF081F80022DD
:103840001949284604F0D2FF18E013E009E0029875
:1038500018B901200C49087002E000200A490870DC
:103860000CE008480AA241F288310368384604F0A7
:103870008DFB03E0012005B0BDE8F08300BF002010
:10388000F9E700005005002054050020BCC30020CB
:1038900041542B514953454E443D25642C300D0A6B
:1038A000000000003405002084290308C8C300205C
:1038B000905F01002B514953454E443A2025642C1A
:1038C00025642C25640D0A002DE9F84305460E46B3
:1038D0001746D5F808800024032E33D005DC5EB1EE
:1038E000012E27D0022E77D12BE0102E34D0182EA7
:1038F0004AD0192E7BD170E040480760006809F07B
:10390000B9FF044604B975E0204606F07CF93C494D
:1039100008600846006800B96CE0394800684068F3
:103920000090364837A241F288310368404604F0DF
:103930002DFB5FE0002032490860404604F048FB60
:1039400058E057E02D48006809F0FAFF002232499C
:10395000284604F04BFF4DE004F0C0FB012807D1DE
:10396000274A12685168264A1268106804F032FE2D
:103970002348006843682248006844F620610268D2
:10398000404604F02DFB35E01C48006809F072FF4A
:10399000044604B92EE01A480168204606F00BF9E7
:1039A00001211E48154A1268815405F005FE1C4984
:1039B000124A126841F8220008461049096850F876
:1039C000210018490D4A126841F8220000221249CC
:1039D000284604F00BFF0DE009E00848006809F0F4
:1039E000AFFF00220C49284604F000FF02E001204E
:1039F000BDE8F88300BF0020FAE70000480500207A
:103A00004C05002041542B514953454E443D2564FB
:103A10002C25750D0A0000008429030834050020B8
:103A2000BCC30020C8C300202DE9F0410446002695
:103A30000025002705F0C0FD804600BF35E0284680
:103A400009F028FF03280BD1042128460AF00EF9BB
:103A50002A462D49E06B04F0C9FE0020BDE8F08144
:103A6000284609F017FF042806D12A462749E06BAB
:103A700004F0BCFE0020F1E7284609F00BFF052802
:103A800006D12A462049E06B04F0B0FE0020E5E7AD
:103A9000284609F01FFF012806D12A461C49E06B81
:103AA00004F0A4FE0020D9E76D1C032DC7DB1948E4
:103AB0000068401C032190FBF1F201FB1205002677
:103AC0001DE0284609F0E6FE062811D1284609F037
:103AD000D1FE074667B1384606F095F840B10D486B
:103AE00005602A460C49E06B04F080FE0020B5E733
:103AF000681C032190FBF1F201FB1205761C032EDA
:103B0000DFDB4FF0FF30A9E7142A0308042A03087B
:103B1000242A030858050020342A03082DE9F0431D
:103B20002DED028B91B004460D469146A668706B50
:103B300007689FED370AB0EE408A042D58D005DCA7
:103B40004DB1012D11D0022D58D14FE00E2D4ED088
:103B5000322D53D110E00E20234642F21072002184
:103B60000090384604F026FE4EE0304604F030FA6D
:103B7000384605F0DBFC47E007F0D2FCBCEEC00A9B
:103B8000244880ED000A24488088000B4FF47A71A5
:103B900010FB01F020498988C1F3032101EBC10228
:103BA00002EB011100EB81001B490979C1F30311FC
:103BB00001EB810100EB41001749097901F00F0188
:103BC00008441649086013480368084614A10268AF
:103BD00002A80CF037FE1949086002A8FCF783FB25
:103BE0008046414602A80AF0C5FB0DE000BF00BFB9
:103BF00000221349204604F0F9FD05E0012011B030
:103C0000BDEC028BBDE8F08300BF0020F7E70000A9
:103C100000000000E404002098240020F0040020AC
:103C2000C9E8B1B8B1E0BAC52564CAA3D3E0B5E725
:103C3000C1BFB0D9B7D6D6AE25640000EC040020D1
:103C4000042903082DE9F84304460D469046A6686A
:103C5000706B0768102D6FD2DFE805F008141B2584
:103C60002F6E6E6E6E6E6E6E5D6E3D61002035491C
:103C700008703549086035A241F28831304604F0B9
:103C800085F95BE0304604F0A3F9384605F04EFCB8
:103C900054E00E20234640F6B8320021009038460A
:103CA00004F088FD4AE00E2023464FF47A7200218A
:103CB0000090384604F07EFD40E02248007801285C
:103CC00005D100222449204604F090FD02E00120A5
:103CD000BDE8F88332E01B480078012805D10022B6
:103CE0001D49204604F082FD14E0174800680A28A8
:103CF0000BD215480068401C1349086013A241F21A
:103D00008831304604F042F904E00022134920468D
:103D100004F06CFD12E001200A4908700EE000205A
:103D200006F0F4FE012805D100220D490D4804F0EB
:103D30005DFD03E002E0FFE70120C9E700BF0020CE
:103D4000C6E70000050500200805002041542B436C
:103D500050494E3F0D0A0000242903083429030866
:103D6000D42803088CC3002010B50446022006F0B6
:103D7000CDFE012812D100200A490860E06B40689E
:103D80004860E06B406840680749486000208860F0
:103D90000022E06B04F02AFD002010BD4FF0FF3040
:103DA000FBE70000A0040020BC04002070B505461D
:103DB0000C46214601200BF04FFE70BD06484168BD
:103DC00005E00648814201D1012070474968002979
:103DD000F7D10020F9E700008CC300207429030804
:103DE00010B50446022006F09BFE012812D10020E7
:103DF0000A490860E06B40684860E06B40684068D2
:103E000007494860002088600022E06B04F0EEFC67
:103E1000002010BD4FF0FF30FBE70000A0040020A1
:103E2000CC04002070B506460D461446285D68B9DE
:103E300044B1601E285C0A2804D1294606A004F07B
:103E40006BFB03E0294608A004F066FB22462946E6
:103E500001200CF0EDF970BD5B41542053656E6498
:103E60005D202573000000005B41542053656E64A3
:103E70005D2025730D0A000010B50446204600F0B1
:103E800067F808B9002010BD2046FEF7B1FB08B95D
:103E90000020F8E7204600F003FA08B90020F2E716
:103EA0002046FFF761FF08B90020ECE72046FFF746
:103EB00097FF08B90020E6E74FF0FF30E3E7000086
:103EC00070B5054605F078FB0446284600F040F83A
:103ED00008B9002070BD2846FEF78AFB08B900200B
:103EE000F8E72846FFF7A0FD08B90020F2E72846CA
:103EF000FEF7B0FC08B90020ECE712480068201A71
:103F000042F21071884208D90E48046000220E491E
:103F10000E4804F06BFC0020DCE7284600F0C0F9F6
:103F200008B90020D6E72846FFF71EFF08B9002091
:103F3000D0E72846FFF754FF08B90020CAE74FF042
:103F4000FF30C7E79C040020942903088CC300209D
:103F500010B50446002006F0E3FD012803D103213B
:103F6000002006F0E7FD002006F0D0FD012806D174
:103F700000220449044804F039FC002010BD4FF031
:103F8000FF30FBE7D42803088CC300207FB504462C
:103F9000002003902CB1E06818B1606A08B1A06AF3
:103FA00018B94FF0FF3004B070BD14E103A92046EA
:103FB000E268904710B14FF0FF30F4E79DF80C1025
:103FC000E26A501CE062606A81540020E26A616A21
:103FD0008854E06A07280CD1072290A0616AFCF798
:103FE00097F930B901208F49087001F0F9FE8E4928
:103FF0000860E06A07280CD107228CA0616AFCF7F0
:1040000087F930B902208749087001F0E9FE864936
:104010000860E06A0A280CD10A2286A0616AFCF7CF
:1040200077F930B903207F49087001F0D9FE7E4945
:1040300008607C480078012807D07A480078022878
:1040400003D078480078032809D101F0C9FE7649E9
:104050000968401A40F2DC51884200D9C1E0714839
:10406000007801281FD176A1606AFCF720F9054687
:10407000C5B10020029002AB72A2E16A606A05F04D
:104080002DFC012800D0ACE0029800B9A9E0606ADC
:10409000281A801C029908446D4908600A20614969
:1040A000087000BF97E05F480078022829D164A11A
:1040B000606AFCF7FCF8054615B366480068B0F185
:1040C000FF3F0ED10020029002AB63A2E16A606A5A
:1040D00005F004FC012800D083E05E4902980860E6
:1040E00000BF5C48006800B97BE0606A281A801C49
:1040F000584909680844564908600A204949087027
:1041000069E048480078032825D1002002904CA19E
:10411000606AFCF7CCF801900198D8B101A8009032
:1041200002AB50A2E16A606A05F0D8FB052800D016
:1041300057E0606A0199081A001D02990844444931
:1041400008600A20374908704149E06A09688842D6
:1041500000D146E03FE0334800780A2805D13C49C9
:10416000E06A0968884236D13BE09DF80C000D28D2
:1041700003D1012084F830000AE09DF80C000A28E1
:1041800006D194F83000012802D1022084F83000D2
:1041900094F83000022816D1E06A022804D10020E9
:1041A000E06284F830000EE0002084F830001D4802
:1041B00000780A2806D100201A490870E06284F8C5
:1041C000300000E00DE0E06A012804D1606A007868
:1041D0003E2800D105E0D4E90A01401E8142FFF4E7
:1041E000E5AE00BFE16A606A05F05EFB012810D110
:1041F000E06A50B1E06A401E616A085C0A2804D196
:104200001FA0616A04F088F903E021A0616A04F04C
:1042100083F900200349087000BFC4E62B514952BE
:10422000443A20008C04002094040020434F4E4E5A
:10423000454354002B514D54524543563A200000FB
:104240000D0A00002B514952443A20256400000019
:104250009004002088040020434F4E4E45435420D4
:10426000256400002B514D54524543563A20252ACF
:104270002C252A2C252A2C25752C256500000000CC
:104280005B415420526563765D2025730000000079
:104290005B415420526563765D2025730D0A000052
:1042A00010B5044606F086FC012812D100200A4908
:1042B0000860E06B40684860E06B40684068074910
:1042C0004860002088600022E06B04F08FFA002034
:1042D00010BD4FF0FF30FBE7A0040020AC0400202D
:1042E00010B5012001F076FC10BD10B54FF48050E0
:1042F00001F070FC10BD10B5022001F06BFC10BD88
:1043000010B54FF4007001F065FC10BD70B586B0BB
:1043100004460D46002000900190022005900120E7
:104320000290204606F088F803906119481E06F0B6
:1043300083F80646204606F07FF8301A401C0490A9
:10434000694601A801F0C8FA18B14FF0FF3006B075
:1043500070BD0020FBE7000010B5002201B909E0A4
:10436000012901D10A0205E0022901D10A0201E076
:104370004FF440720E4B1B6823F440730C4C2360C7
:1043800023461B681343236023461B6823F0F8036E
:10439000236023461B68022444EAC0042343044CE0
:1043A000236023461B6843F48033236010BD000064
:1043B000103C02401C48006800F40070B0B11A487C
:1043C000006820F400701849086000BF08460068C3
:1043D00040F4006008600846006820F4006008604F
:1043E00000BF0846006840F4007008600E4800688E
:1043F00000F48060B0B10C48006820F480600A4985
:10440000086000BF0846006840F480500860084615
:10441000006820F48050086000BF0846006840F43F
:104420008060086070470000003C02400A4A126841
:1044300022F44072084B1A601A46126842F00402D5
:104440001A601A4612684FF4803343EA00231A4375
:10445000014B1A6070470000103C0240074A126886
:1044600022F44072054B1A601A4612681A601A4606
:10447000126842F001021A6001707047103C02405D
:1044800010B50949096821F44071074C21602146A3
:10449000096841F4407121602146096841F0010139
:1044A00021600260436010BD103C0240084A12685F
:1044B00022F44072064B1A601A46126842F4807267
:1044C0001A601A46126842F001021A6001807047B1
:1044D000103C0240084A126822F44072064B1A60EF
:1044E0001A46126842F400721A601A46126842F0C4
:1044F00001021A6001607047103C02402A480068BF
:1045000000F0100040B12948C06940F01000274970
:10451000C8611020244908602348006800F020008A
:1045200040B12248C06940F008002049C8612020FD
:104530001D4908601C48006800F0400040B11B485D
:10454000C06940F004001949C8614020164908605C
:104550001548006800F0800040B11448C06940F080
:1045600002001249C86180200F4908600E480068A7
:1045700000F4807048B10D48C06940F001000B495B
:10458000C8614FF48070084908600748006800F06F
:10459000020040B10548C06940F020000349C861ED
:1045A00002200149086070470C3C024038E90020B5
:1045B00070B50446002500201449C86101F010FCC4
:1045C000054609E0601C38B124B101F009FC401B2C
:1045D000A04201D9032070BD0D48006800F480306E
:1045E0000028EFD10A48006800F0010010B1012056
:1045F000074908600648006800F4F97018B1FFF731
:104600007DFF0120E7E70020E5E7000038E9002012
:104610000C3C02402DE9F84307460D46144600269F
:10462000B0460020009024E0042C0CD24FF0FF3064
:104630000090002603E0A85D0DF80600761CA64257
:10464000F9D3A04603E0286800904FF00408F32057
:104650000A490860002339460220009A01F092F9C5
:1046600018B14FF0FF30BDE8F88347444544A4EB50
:104670000804002CD8D10020F5E700000C3C0240D3
:104680000FB4F8B504460D4600261CB9701EF8BCE0
:104690005DF814FBE06A08B90020F8E709A800906B
:1046A000E76A29462046009B089AB847064600203C
:1046B00000903046EBE7F0B504460D461E4600215B
:1046C00000270023214600BF10E042F8331002EB20
:1046D000C300476002EBC3075B1C6868D1F804C0E5
:1046E000604502D137600020F0BD49680029ECD157
:1046F000481EF9E72DE9F0410546002700264FF650
:10470000FF7000EA1547AEB20848046809E0208847
:10471000B84205D100223146204603F0A3FF02E053
:104720006469002CF3D100BFBDE8F081C806002009
:104730002DE9F04186B006460F464FF000080025EF
:10474000002402A804AB12A239460090304605F0BE
:10475000C5F8022803D0601E06B0BDE8F081DDE98F
:10476000020105F052F800F0FF08049805780124D2
:1047700003E00498005D4540641C0598A042F8D809
:10478000454502D04FF0FF30E6E70020E4E70000A7
:104790002425702A25700D0A0000000010B588B08D
:1047A00000F016FA00F0C6FB00208DF805008DF829
:1047B0000400224802904FF4806003902048049047
:1047C0004FF4206005900220069001A90BF016FA24
:1047D000B0211C4804F0F8FF1BA20A211948401C14
:1047E00005F06FF91749086219A20A2115480B3024
:1047F00005F067F91349486217A20A2111481530DC
:1048000005F05FF90F4988620120154908701548C5
:10481000B0F854001349B1F8521040EA0124B4F53D
:10482000612F02D8B4F5165F01D24FF4E13421466E
:1048300002200BF067FB08B010BD0000F46E0020F2
:10484000F4720020047D002024474E4747410000B9
:104850002447504753560000244742475356000010
:10486000920300209824002030B58FB004460D46F6
:10487000282104A8FBF704FD29462046FFF758FF2E
:1048800018B14FF0FF300FB030BD1D481D491E4A12
:104890001E4BCDE9002102901DA22946204605F0BD
:1048A0001DF80F2802D04FF0FF30ECE714490868DC
:1048B000FBF753FD224908701249086800210BF0EC
:1048C000FBFF204880ED000B0F49086800210BF02A
:1048D000F3FF1D4880ED000B09490868FBF73DFD1B
:1048E000174908700948016818480A6802608988F1
:1048F000818013480078164908600020C3E7000053
:104900001C040020040400200C04002024040020C7
:1049100024252A2C25702C25702C252A2C25702C3A
:10492000252A2C25702C252A2C252A2C252A2C25B5
:104930002A2C252A2C252A2C252A2C252A2A000037
:1049400090030020F0030020F8030020B47D002035
:104950000004002070B596B004460D4628210CA82E
:10496000FBF78EFC0AA808A906AA04ABCDE9002132
:1049700002903D4A2946204604F0B0FF15281AD17E
:104980003A480088001D394908800498FBF7E5FC87
:1049900006460698FBF7E1FC06440898FBF7DDFCA9
:1049A00006440A98FBF7D9FC304431490988084489
:1049B0002F49088054E008A806A904AB2DA2CDE930
:1049C00000102946204604F089FF112816D12748F7
:1049D0000088C01C254908800498FBF7BEFC0646E9
:1049E0000698FBF7BAFC06440898FBF7B6FC30447F
:1049F0001F49098808441E49088031E006A804AB15
:104A00002AA229460090204604F068FF0D2812D102
:104A100016480088801C154908800498FBF79DFC07
:104A200006460698FBF799FC30441149098808446A
:104A30000F49088014E004AB27A22946204604F061
:104A40004DFF09280CD109480088401C07490880FF
:104A50000498FBF782FC0649098808440449088049
:104A6000002016B070BD0000082D03082E040020A1
:104A70002C04002024252A2C252A2C252A2C252A02
:104A80002C252A2C252A2C252A2C25702C252A2C4D
:104A9000252A2C252A2C25702C252A2C252A2C2544
:104AA0002A2C25702C252A2A0000000024252A2CD7
:104AB000252A2C252A2C252A2C252A2C252A2C256A
:104AC0002A2C25702C252A2C252A2C252A2C2570C9
:104AD0002C252A2A0000000024252A2C252A2C25F2
:104AE0002A2C252A2C252A2C252A2C252A2C2570EF
:104AF0002C252A2A00000000034B43F8301003EB5A
:104B0000C0039A8070470000F47C00200EB500209E
:104B100002900190009069460BF05CF82DE0FCF7E4
:104B200067FF012803D0FCF763FF022806D14FF48A
:104B30007A73012201A9009803F0F5F89DF80400AA
:104B400000F09AF89DF80410194802680068401CAB
:104B5000174B18601748815418460068B0F5007F5D
:104B600007D318460168134806F0C6F8002010491C
:104B7000086004F021FD1049086001A902200AF034
:104B80006BFF02900028CAD00948006870B104F099
:104B900013FD09490968401A322807D904480168F9
:104BA000044806F0A9F80020014908600EBD000085
:104BB00038040020C87D00203C04002010B5034AC2
:104BC00091899068002201F005F910BDF47C002065
:104BD00010B5034A91899068012201F0FBF810BDDD
:104BE000F47C002010B504461D480470012C06D04A
:104BF000022C0FD0052C18D00A2C2CD120E00E222C
:104C0000184902200BF014FB1522174902200BF063
:104C10000FFB21E00E22154902200BF009FB1522A3
:104C2000114902200BF004FB16E00E22104902206D
:104C30000BF0FEFA15220C4902200BF0F9FA0BE0FA
:104C40000E220C4902200BF0F3FA1522064902202D
:104C50000BF0EEFA00E000BF00BF002010BD000026
:104C600091030020B10300209C030020BF0300201B
:104C7000CD030020DB03002030B589B004469F4AF5
:104C8000D2E900109268CDE9070206919B4A0C32E6
:104C900007CA03AB07C3994A183207CA8DE8070051
:104CA0009748007830B1012819D0022851D0032844
:104CB0007DD169E0242C11D1012091490870002098
:104CC000C1F8AC000846D0F8AC10D0F8AC00401CDD
:104CD0008B4AC2F8AC0002F12C0044540AE1884827
:104CE000D0F8AC10D0F8AC00401C854AC2F8AC003B
:104CF00002F12C0044542C38D0F8AC001146096A5B
:104D0000884225D31046411C026A2C30FBF700FB79
:104D100018B902207A4908701AE0794800F10B01AD
:104D2000426A2C30FBF7F4FA18B902207449087073
:104D30000EE0734800F11501826A2C30FBF7E8FAA7
:104D400018B902206E49087002E000206C49087012
:104D5000D0E06B48D0F8AC10D0F8AC00401C684AEA
:104D6000C2F8AC0002F12C0044542C38D0F8AC004E
:104D70007F2803D3002011460870BBE00D2C02D120
:104D800003205F490870B5E05D48D0F8AC10D0F85A
:104D9000AC00401C5A4AC2F8AC0002F12C0044544A
:104DA0000A2C6FD15748007840B9574800E0A0E07E
:104DB000B0F8700055490978884207D00020514961
:104DC0000870514991F87000FFF70CFF4C4800F152
:104DD0001501826A2C30FBF79BFA28B94848D0F8B5
:104DE000AC102C30FFF7B6FD4548411C026A2C3050
:104DF000FBF78EFA00286CD14148D0F8AC102C306B
:104E0000FFF732FD00223E48D0F8AC00801E3C493E
:104E10002C310A543E48007878B100203C49087093
:104E20003C4908603C4803683C4802680846016801
:104E30003B48006807F0D8FB4BE00120344908707C
:104E4000384800683849097888420DD036480078DB
:104E5000042808D103A8FBF746FA0546294603A80B
:104E600009F088FA00BF00BF2F48007806281CD23E
:104E7000DFE800F003090D1B12174FF40840254925
:104E8000086017E031E088202249086012E04FF006
:104E90008810204908600DE04FF408001D490860A3
:104EA00008E022481B49086004E02048883019497E
:104EB000086000BF00BF184803681848026815481A
:104EC00001681748006807F08FFB174800781549FC
:104ED000086004F071FB16490968401AB0F57A7F42
:104EE00003D304F069FB12490860002004490870EC
:104EF00000E000BF00BF09B030BD0000C4250308BA
:104F0000047D0020920300209824002091030020BB
:104F10003404002068060020700600206C06002083
:104F200064060020300400209003002000888800E0
:104F30009403002010B50C4A91881068012200F0FB
:104F400049FF0A2000F0B4FC074A9188106800224B
:104F500000F040FF0A2000F0ABFC034A9188106883
:104F6000012200F037FF10BDF47C00202DE9F04F46
:104F700095B0044688461546994600200090824622
:104F80002E46CB4600271CB1B8F1000F00D025B942
:104F90004FF0FF3015B0BDE8F08F4AE000203870C8
:104FA000142301AA3B21304604F0A2FD0090009892
:104FB000122838D926A10198FBF79CF900B138E0F6
:104FC000BAF1000F14D1B24620212046029A04F013
:104FD00078FD202104F12000039A04F072FD0C9862
:104FE000FBF7BBF908B1012000E0002084F8400085
:104FF00041460398FBF77EF9A8B920212046029A82
:1050000004F05FFD202104F12000049A04F059FD12
:105010000C98FBF7A2F908B1012000E0002084F809
:1050200040000020B6E7B81C801BABEB000BBE1C99
:1050300000BF5A4607A1304604F09DFD071EADD1C2
:10504000BAF1000F01D1401EA4E70020A2E7000042
:10505000535452000D0A000038B50246002000905B
:1050600000BF92F83C00012801D1022038BD012088
:1050700082F83C0000BF0868092816D91068C0688B
:105080000C780A3C04EB44050724AC40A0431468A8
:10509000E0600C780A3C04EB44048868A040146883
:1050A000E46820431468E06013E0106800690C783D
:1050B00004EB44050724AC40A043146820610C783D
:1050C00004EB44048868A0401468246920431468F1
:1050D00020614868072817D21068406B0C79641E5D
:1050E00004EB84051F24AC40A04314686063088867
:1050F00080B20C79641E04EB8404A0401468646BD5
:1051000020431468606331E048680D2817D21068A6
:10511000006B0C79E41F04EB84051F24AC40A04312
:1051200014682063088880B20C79E41F04EB8404BF
:10513000A0401468246B20431468206316E01068B4
:10514000C06A0C790D3C04EB84051F24AC40A043DD
:105150001468E062088880B20C790D3C04EB84048A
:10516000A0401468E46A20431468E062194B1A4CAA
:105170001068A04206D10868122803D1586840F48C
:1051800080005860144C1068A0421CD10868102898
:1051900002D00868112816D1586840F40000586001
:1051A000086810280FD10D4800680D4CB0FBF4F0D2
:1051B00000EB80004000009002E00098401E00904C
:1051C00000980028F9D100BF002082F83C0000BF01
:1051D00000BF4BE70023014000200140C40600202F
:1051E00040420F00704770477047000070B504469A
:1051F00000250CB9012070BD1549A06A884200D075
:1052000000BF206C30B90020606484F83C00204668
:1052100000F020F8206C00F0100088B9206C20F419
:10522000885040F0020020642046FBF715FF002064
:105230006064206C20F0020040F00100206400E077
:10524000012500BF002084F83C0000BF2846D2E7BB
:105250000100000F10B586B004462149206888423D
:105260003CD100BF002000901E48006840F48070D0
:105270001C4908600846006800F48070009000BF78
:1052800000BF02200190032002900020039001A99A
:10529000154800F0ADFC154815490860002048602D
:1052A000002113488160C1604FF4806101614900B1
:1052B0004161890081614911C1614FF4403101624E
:1052C0000021416200F02EFA18B17E2109A00BF0F6
:1052D0008FFA00BF0648A063846300BF06B010BD0C
:1052E00000200140443802400000024010640240A7
:1052F00008E500202E2E2F5372632F73746D333206
:10530000663478785F68616C5F6D73702E6300003F
:10531000F8B504460D4616460020009000BF94F8EC
:105320003C00012801D10220F8BD012084F83C0096
:1053300000BF2068806800F00100A0B92068806884
:1053400040F00100216888603C4800683C49B0FB9F
:10535000F1F000EB4000009002E00098401E009049
:1053600000980028F9D12068806800F0010000282A
:1053700062D0206C40F20161884340F48070206468
:105380002068406800F4806028B1206C20F4005050
:1053900040F480502064206C00F4805020B1606C98
:1053A00020F00600606401E00020606400BF00207F
:1053B00084F83C0000BF234F2348A16BC8632348F7
:1053C000A16B08642248A16BC8646FF022002168B9
:1053D00008602068406840F080602168486020686C
:1053E000806840F4807021688860226802F14C0176
:1053F00033462A46A06B00F00BFA786800F01F00D5
:1054000058B92068806800F0405028B9206880684A
:1054100040F08040216888600EE00E492068884294
:105420000AD12068806800F0405028B92068806860
:1054300040F0804021688860002075E7C4060020A5
:1054400040420F0000230140790F020801100208BA
:10545000E70F020800200140014691F835000228BC
:1054600003D08020486501207047052081F8350071
:105470000868006820F001000A6810600020F3E767
:1054800070B504460CB9012070BD94F835000228AF
:1054900000D1F9E72068006820F001002168086069
:1054A00000202168086021684860216888602168C0
:1054B000C860216808612120216848612046FCF706
:1054C000FBFB054694F85C103F208840A860002054
:1054D000606584F8350000BF84F8340000BF00BF69
:1054E000D2E70000F8B50446002000908C48006820
:1054F0004FF41651B0FBF1F7A56D2E6894F85C10CF
:1055000008208840304098B12068006800F004000E
:1055100070B12068006820F004002168086094F8E9
:105520005C1008208840A860606D40F00100606554
:1055300094F85C1001208840304068B120684069D0
:1055400000F0800040B194F85C1001208840A86011
:10555000606D40F00200606594F85C1004208840A3
:10556000304068B12068006800F0020040B194F853
:105570005C1004208840A860606D40F00400606505
:1055800094F85C1010208840304078B320680068A0
:1055900000F0080050B394F85C1010208840A86018
:1055A0002068006800F4802080B12068006800F462
:1055B000002028B9206CC8B12046216C884715E02E
:1055C000A06C98B12046A16C88470FE02068006865
:1055D00000F4807028B92068006820F00800216875
:1055E0000860206C10B12046216C884794F85C104C
:1055F000202088403040002865D02068006800F0F6
:10560000100000285FD094F85C1020208840A8602B
:1056100094F83500052828D12068006820F016008D
:10562000216808602068406920F080002168486196
:10563000206C08B9A06C28B12068006820F0080030
:105640002168086094F85C103F208840A86000BF83
:10565000002084F8340000BF012084F83500206D5C
:1056600010B12046216D8847F8BD2068006800F41D
:10567000802080B12068006800F4002028B9606CA8
:1056800010B12046616C88471DE0E06BD8B1204620
:10569000E16B884717E02068006800F4807068B903
:1056A0002068006820F010002168086000BF00201A
:1056B00084F8340000BF012084F83500E06B10B19D
:1056C0002046E16B8847606D38B3606D00F00100E3
:1056D000F0B1052084F835002068006820F0010052
:1056E0002168086000BF0098401C0090B84200D9B3
:1056F00005E02068006800F001000028F3D100BF39
:1057000000BF002084F8340000BF012084F8350079
:10571000E06C10B12046E16C884700BFA4E70000B0
:10572000C40600202DE9F0410446002500F058FB96
:10573000074614B90120BDE8F081606A00B100BFDE
:1057400000BF002084F8340000BF022084F8350038
:105750002068006820F00100216808600AE000F07D
:105760003FFBC01B052805D920206065032084F875
:105770003500E0E72068006800F001000028EED165
:105780002068056821480540D4E901010843E16823
:1057900008432169084361690843A1690843E16935
:1057A0000843216A08430543606A042803D1D4E909
:1057B0000B0108430543206805602068456925F012
:1057C0000705606A0543606A04280DD1A06A054395
:1057D000E06A48B12046FCF789FA28B140206065AC
:1057E000012084F83500A6E7206845612046FCF7D3
:1057F00063FA064694F85C103F208840B0600020B1
:105800006065012084F83500002094E73F8010F0A7
:105810002DE9F04704460D4616461F464FF0000896
:10582000D4F8589000BF94F83400012802D1022027
:10583000BDE8F087012084F8340000BF94F83500FB
:1058400001282BD1022084F83500002060653B46FA
:10585000324629462046FCF79EFA94F85C103F2019
:105860008840C9F808002068006840F016002168E8
:1058700008602068406940F0800021684861206C21
:1058800028B12068006840F008002168086020689E
:10589000006840F001002168086006E000BF0020B9
:1058A00084F8340000BF4FF002084046C0E7000013
:1058B00070B5044600F094FA06462546681C10B1FF
:1058C00004480078054400BF00F08AFA801BA84213
:1058D000FAD370BDC00600202DE9F04104460E4603
:1058E0000127002500BF2548007E012802D10220A3
:1058F000BDE8F08101202149087600BF4CF250300C
:10590000FEF756FE0746002F31D1401E306020685A
:1059100001280FD1207C6168FEF788FD4CF25030E1
:10592000FEF746FE07461648006820F004001449BA
:1059300008601AE0A56812E0217C2846FEF70CFDFD
:105940004CF25030FEF734FE07460D48006820F058
:10595000FA000B4908600FB1356005E06D1CD4E911
:1059600002100844A842E7D800BFFEF723FD00BF9D
:1059700000200249087600BF3846B9E738E9002020
:10598000103C02402DE9F04106460F4614461D46E4
:105990004FF0010800BF1F48007E012802D10220FD
:1059A000BDE8F08101201B49087600BF4CF2503061
:1059B000FEF7FEFD8046B8F1000F23D126B9E1B213
:1059C0003846FEF74BFD12E0012E04D1A1B2384655
:1059D000FEF76CFD0BE0022E04D121463846FEF79F
:1059E00079FD04E022462B463846FEF749FD4CF28D
:1059F0005030FEF7DDFD80460748006820F00100CA
:105A00000549086000BF00200249087600BF4046F3
:105A1000C6E7000038E90020103C02400020094998
:105A2000096801F0004159B10749064A0C3A116072
:105A3000064911600349096801F0004101B10120E4
:105A400070470000103C024023016745AB89EFCD51
:105A5000F0B50C46002500220023002181E001263C
:105A600006FA01F504EA0502AA4279D106684FEA6E
:105A7000410C032707FA0CF7BE430660CF0800F17C
:105A8000200656F827604F074FEAD76C0F2707FA12
:105A90000CF7BE434FEAD10C00F1200747F82C6009
:105AA00086684FEA410C032707FA0CF7BE4386606D
:105AB000476801268E40B7434760C6684FEA410CED
:105AC000032707FA0CF7BE43C660284E8F0856F826
:105AD00027308E07370F0F26BE403340244EB0428A
:105AE00001D1002614E0234EB04201D101260FE07F
:105AF000214EB04201D102260AE0204EB04201D12F
:105B0000032605E01E4EB04201D1042600E0072620
:105B10008F073F0FBE409E4222D18E07370F0F26C0
:105B200006FA07F3114E8F0856F827609E430F4F71
:105B30004FEA910C47F82C60124E36689643114F8D
:105B40003E603E1D366896433F1D3E603E1D3668F2
:105B500096433F1D3E603E1D366896433F1D3E60A6
:105B6000491C1029FFF47BAFF0BD0000083801404C
:105B7000000002400004024000080240000C024005
:105B800000100240003C014010B50446B4F5805FAF
:105B900001D105F03FFB012C04D19FED0B0A0B480E
:105BA00080ED000AB4F5007F04D10948007808B9F7
:105BB000FBF7B4FBB4F5007F05D105480078012858
:105BC00001D109F0D7FE10BD000000001C06002026
:105BD0007701002010B5044604480068204020B139
:105BE000024804602046FFF7CFFF10BD143C01407F
:105BF000F8B503460A460025002400200021CDE028
:105C0000012606FA01F5166806EA0504AC4273D1CE
:105C10005668022E02D05668122E13D1CF0803F117
:105C2000200656F827004E07F70E0F26BE40B04359
:105C30004F07FF0E1669BE403043CF0803F1200620
:105C400046F8270018684F000326BE40B043167977
:105C500006F003064F00BE40304318605668012E20
:105C600008D05668022E05D05668112E02D056680C
:105C7000122E13D198684F000326BE40B0434F0048
:105C8000D668BE4030439860586801268E40B043C5
:105C90001679C6F300168E4030435860D8684F001E
:105CA0000326BE40B0434F009668BE403043D860E4
:105CB000566806F08056B6F1805F6ED100BF0026B0
:105CC0000096384E366846F48046364F3E603E4673
:105CD000366806F48046009600BF00BF324E8F083B
:105CE00056F827008E07370F0F26BE40B0432F4EC1
:105CF000B34202D1002615E04FE02D4EB34201D150
:105D000001260FE02B4EB34201D102260AE02A4EB3
:105D1000B34201D1032605E0284EB34201D1042647
:105D200000E007268F073F0FBE4030431E4E8F080E
:105D300046F82700224E3068A043566806F48036A5
:105D4000B6F5803F00D120431D4E3060361D3068CF
:105D5000A043566806F40036B6F5003F00D1204354
:105D6000174E361D3060361D3068A043566806F465
:105D70008016B6F5801F00D12043114E08363060E2
:105D8000361D3068A043566806F40016B6F5001FAD
:105D900000D120430A4E0C363060491C1029FFF414
:105DA0002FAFF8BD443802400838014000000240DF
:105DB0000004024000080240000C024000100240B3
:105DC000003C0140024613690B400BB1012000E08A
:105DD000002070470AB1816101E00B0483617047C4
:105DE0000148006870470000B806002003480068BA
:105DF000034909780844014908607047B806002043
:105E0000C006002010B50D48006840F400700B4932
:105E100008600846006840F4806008600846006832
:105E200040F480700860032000F0B6F8002000F015
:105E300007F800F02BF8002010BD0000003C0240E5
:105E400070B504460E4800784FF47A71B1FBF0F05B
:105E50000C490968B1FBF0F5284600F090FF08B145
:105E6000012070BD102C07D200222146501E00F0E8
:105E700054F80548046001E00120F2E70020F0E753
:105E8000C0060020C4060020BC06002010B5032078
:105E900000F082F8002211466FF00B0000F03DF890
:105EA000002211466FF00A0000F037F80022114678
:105EB0006FF0090000F031F800221146501F00F089
:105EC0002CF800221146101F00F027F8002211467E
:105ED000901E00F022F800221146501E00F01DF81E
:105EE00010BD000000BF00F01F0201219140034AD5
:105EF000430942F8231000BF7047000080E100E032
:105F000000BF00F01F02012191404209920002F1FE
:105F1000E022C2F8001100BF70472DE9F05F804613
:105F20000D461646002704F0DDFF074639462A468F
:105F3000334601F00700C0F1070ABAF1040F02D995
:105F40004FF0040A01E0C0F1070AD14600F1040A4B
:105F5000BAF1070F02D24FF0000A01E0A0F1030AE4
:105F6000D4464FF0010A0AFA09FAAAF1010A0AEA2C
:105F7000020A0AFA0CFA4FF0010B0BFA0CFBABF118
:105F8000010B0BEA030B4AEA0B042146404604F0DE
:105F9000B1FFBDE8F09F000000BF00F00702064B14
:105FA00019684FF6FF031940044B0B4343EA0221E3
:105FB000014B196000BF70470CED00E00000FA05CE
:105FC0000D4A126822F0030202430B4B1A600B4A7F
:105FD000126842F00402094B1A60012901D130BF56
:105FE00002E040BF20BF20BF044A126822F0040232
:105FF000024B1A60704700000070004010ED00E096
:1060000070B504460D460CB9012070BD58480068B3
:1060100000F00F00A84209D255490D7008460068EB
:1060200000F00F00A84201D00120EEE7207800F038
:10603000020002281DD1207800F00400042805D1B8
:106040004C48006840F4E0504A490860207800F06D
:106050000800082805D14748006840F460404549D9
:1060600008604448006820F0F000A16808434149F6
:106070000860207800F00100A8B36068012807D10B
:106080003C4808380068C0F34040B8B90120BCE77C
:106090006068022802D06068032807D135480838B4
:1060A0000068C0F3406048B90120AEE731480838C5
:1060B0000068C0F3400008B90120A6E72D48006839
:1060C00020F00300616808432A490860FFF788FE52
:1060D000064609E0FFF784FE801B41F288318842C2
:1060E00002D9032091E707E02248006800F00C0085
:1060F0006168B0EB810FEDD11D48006800F00F0022
:10610000A84209D91A490D700846006800F00F002E
:10611000A84201D0012078E7207800F0040004288C
:1061200007D11448006820F4E050E16808431149A1
:106130000860207800F00800082808D10D480068A1
:1061400020F46040216940EAC1000A49086000F07B
:106150003DF808490968C1F30311074A515CC8407A
:10616000064908600020FFF76BFE00204DE70000A5
:10617000003C024008380240E62A0308C40600201A
:106180000148006870470000C406002000B5FFF712
:10619000F7FF04490968C1F38221034A515CC840F2
:1061A00000BD000008380240F62A030800B5FFF7DA
:1061B000E7FF04490968C1F34231034A515CC84012
:1061C00000BD000008380240F62A03082DE9F04718
:1061D000002400250026A1462548006800F00C0098
:1061E00020B1042805D008283AD105E0DFF88490D2
:1061F00039E0DFF8849036E01D48001F006800F0A9
:106200003F041B48001F006800F4800078B11A4862
:106210001749091F0968C1F38811A0FB01700146E5
:10622000224600233846F9F7D1FF05460EE0114813
:106230000F49091F0968C1F38811A0FB01700146CD
:10624000224600233846F9F7C1FF05460848001FDB
:106250000068C0F30140401C4600B5FBF6F902E0BF
:10626000DFF8109000BF00BF4846BDE8F08700008F
:10627000083802400024F40000127A00F8B5044601
:106280000CB90120F8BD207800F00100002874D07E
:10629000F948006800F00C0004280DD0F6480068AA
:1062A00000F00C00082813D1F348001F006800F428
:1062B0008000B0F5800F0BD1EF4808380068C0F3BC
:1062C0004040002859D06068002856D10120D9E705
:1062D00000BF6068B0F5803F08D1E7480838006823
:1062E00040F48030E449083908601EE06068B0F589
:1062F000A02F0DD1E0480838006840F48020DE4926
:10630000083908600846006840F4803008600CE0F6
:10631000D9480838006820F48030D7490839086027
:106320000846006820F48020086000BF606890B1D3
:10633000FFF756FD054606E0FFF752FD401B6428B7
:1063400001D903209EE7CC4808380068C0F34040DC
:106350000028F1D011E0FFF743FD054606E0FFF706
:106360003FFD401B642801D903208BE7C248083851
:106370000068C0F340400028F1D1207800F002000E
:1063800002285FD1BC48006800F00C0058B1BA4840
:10639000006800F00C0008281CD1B748001F0068F6
:1063A00000F48000B0B9B44808380068C0F3400079
:1063B00020B1E068012801D0012063E7AE48083829
:1063C000006820F0F800216940EAC100AA490839B4
:1063D000086037E0E06800B30120A8490860FFF7D3
:1063E000FFFC054606E0FFF7FBFC401B022801D935
:1063F000032047E7A04808380068C0F340000028A1
:10640000F1D09D480838006820F0F800216940EA82
:10641000C10099490839086014E0002097490860D4
:10642000FFF7DEFC054606E0FFF7DAFC401B02281A
:1064300001D9032026E7904808380068C0F34000DF
:106440000028F1D1207800F0080008282CD16069DC
:10645000A8B101208A490860FFF7C2FC054606E0A2
:10646000FFF7BEFC401B022801D903200AE782483F
:106470006C300068C0F340000028F1D014E0002028
:106480007F490860FFF7ACFC054606E0FFF7A8FC73
:10649000401B022801D90320F4E677486C300068DD
:1064A000C0F340000028F1D1207800F00400042857
:1064B00070D1002670483830006800F0805090B9E4
:1064C00000BF002000906C483830006840F08050D9
:1064D0006949383108600846006800F08050009033
:1064E00000BF00BF01266748006800F48070B0B9A3
:1064F0006448006840F4807062490860FFF770FCEF
:10650000054606E0FFF76CFC401B022801D903207A
:10651000B8E65C48006800F480700028F2D000BF44
:10652000A068012808D154486830006840F0010094
:106530005149683108601DE0A06805280DD14E481A
:106540006830006840F004004B4968310860084634
:10655000006840F0010008600CE0474868300068BF
:1065600020F001004449683108600846006820F0C6
:106570000400086000BFA068A8B1FFF731FC054621
:1065800009E0FFF72DFC401B41F28831884202D917
:10659000032077E626E0384868300068C0F3400002
:1065A0000028EED013E0FFF71BFC054608E0FFF7DC
:1065B00017FC401B41F28831884201D9032061E673
:1065C0002D4868300068C0F340000028EFD1012E4C
:1065D00007D129483830006820F0805026493831EA
:1065E000086000BFA069B8B32348006800F00C0041
:1065F00008285ED0A069022846D100201F490866FD
:10660000FFF7EEFB054606E0FFF7EAFB401B02281A
:1066100001D9032036E6184808380068C0F3406006
:106620000028F1D1D4E907010843616A40EA8111E9
:106630000122A06AC2EB500041EA00412C20005D1B
:1066400041EA00600C49091F086001200B490866F7
:10665000FFF7C6FB054607E02DE0FFF7C1FB401B37
:10666000022801D903200DE6034808380068C0F36A
:1066700040600028F1D01EE0083802400000474288
:10668000800E47420070004000200C490866FFF76A
:10669000A7FB054606E0FFF7A3FB401B022801D934
:1066A0000320EFE506480068C0F340600028F2D1FF
:1066B00001E00120E6E50020E4E50000000047429B
:1066C000003802404FF0E020006940F002004FF037
:1066D000E0210861704710B504460CB9012010BDD7
:1066E000022084F851002068006820F040002168F2
:1066F0000860204600F050F80020606584F85100E2
:1067000000BF84F8500000BF00BFE8E710B50446A2
:106710000CB9012010BD606A00B900BF0021A16260
:1067200094F8510028B9002084F85000204600F069
:106730004BF8022084F851002068006820F04000E7
:1067400021680860D4E901010843E1680843216930
:10675000084361690843218B01F400710843E16932
:106760000843216A0843A16A08432168086004219C
:10677000A06901EA1040616A084321684860206806
:10678000C06920F400602168C861002060650120B4
:1067900084F851000020BDE710B504460749206881
:1067A000884209D10648006820F4805004490860F6
:1067B000E0210448FFF74CF910BD00000030014013
:1067C000443802400000024010B586B00446124929
:1067D000206888421DD100BF002000900F4800684B
:1067E00040F480500D4908600846006800F480506D
:1067F000009000BF00BFE020019002200290002026
:106800000390032004900520059001A90448FFF798
:10681000EFF906B010BD00000030014044380240DE
:10682000000002402DE9F84304460D4617461E4677
:106830004FF00008C1466068B0F5827F0DD1A068B6
:1068400058B9042084F851003B462A462946204680
:10685000009600F070F9BDE8F88300BF94F850008E
:10686000012801D10220F6E7012084F8500000BF82
:10687000FFF7B6FA804694F85100012802D04FF095
:1068800002097BE005B117B94FF0010976E0042059
:1068900084F8510000206065A563A787E78720631F
:1068A000A086E08620646064A068B0F5004F05D142
:1068B0002068006820F48040216808602068006833
:1068C00000F04000402805D02068006840F04000FB
:1068D00021680860E068E8B918E02068806800F086
:1068E000010038B12068007B28706D1CE08F401ECD
:1068F000E0870BE03EB1701C40B1FFF771FAA0EBEE
:106900000800B04202D34FF0030937E0E08F0028BF
:10691000E3D11CE018E02068806800F0010038B185
:106920002068C0682880AD1CE08F401EE0870BE027
:106930003EB1701C40B1FFF753FAA0EB0800B04223
:1069400002D34FF0030919E0E08F0028E3D160681B
:10695000B0F5827F0DD1A068B0F5004F03D0A068DC
:10696000B0F5806F05D12068006820F040002168F4
:106970000860606D08B14FF0010900BF012084F884
:10698000510000BF002084F8500000BF484662E775
:106990002DE9F84304460D4617461E464FF0000801
:1069A000C14600BF94F85000012802D10220BDE882
:1069B000F883012084F8500000BFFFF711FA8046E9
:1069C00094F85100012802D04FF00209A9E005B166
:1069D00017B94FF00109A4E0032084F8510000200A
:1069E00060652563A786E786A063A087E08760646B
:1069F0002064A068B0F5004F05D12068006840F41D
:106A00008040216808602068006800F0400040284D
:106A100005D02068006840F0400021680860E06808
:106A2000B0F5006F2AD1606810B1E08E012806D160
:106A300028882168C860AD1CE08E401EE08619E001
:106A40002068806800F00200022807D128882168A9
:106A5000C860AD1CE08E401EE0860BE03EB1701CAD
:106A600040B1FFF7BDF9A0EB0800B04202D34FF0F0
:106A7000030956E0E08E0028E2D129E0606810B1F9
:106A8000E08E012806D12878216808736D1CE08EFD
:106A9000401EE08619E02068806800F002000228AD
:106AA00007D12878216808736D1CE08E401EE086AF
:106AB0000BE03EB1701C40B1FFF792F9A0EB08006B
:106AC000B04202D34FF003092BE0E08E0028E2D160
:106AD0003346012202212046CDF8008005F09AFCC1
:106AE00010B14FF003091CE042463146204605F044
:106AF00059FC20B14FF001092020606511E0A06829
:106B000050B900BF002000902068C0680090206845
:106B10008068009000BF00BF606D08B14FF00109B0
:106B200000BF012084F8510000BF002084F850000D
:106B300000BF48463BE72DE9FE4F04460D4616468A
:106B40001F46DDF830804FF0000A00200290814699
:106B50004FF0010B019000BF94F85000012802D1C2
:106B60000220BDE8FE8F012084F8500000BFFFF72F
:106B700037F9814694F851A060680290BAF1010F8C
:106B80000BD00298B0F5827F04D1A06810B9BAF199
:106B9000040F02D002200190D2E00DB106B117B966
:106BA00001200190CCE094F85100012802D1052089
:106BB00084F8510000206065A663E787A7872563F6
:106BC000E786A786206460642068006800F04000C3
:106BD000402805D02068006840F040002168086027
:106BE000E068B0F5006F43D1606810B1E08E012815
:106BF00006D128882168C860AD1CE08E401EE08662
:106C00002FE0BBF1000F10D0E08E70B120688068DB
:106C100000F00200022808D128882168C860AD1C55
:106C2000E08E401EE0864FF0000BE08F68B12068D8
:106C3000806800F0010040B12068C0683080B61C58
:106C4000E08F401EE0874FF0010B08F1010040B1DA
:106C5000FFF7C6F8A0EB0900404502D303200190DE
:106C60006EE0E08E0028CCD1E08F0028C9D142E050
:106C7000606810B1E08E012806D128782168087379
:106C80006D1CE08E401EE0862FE0BBF1000F10D09F
:106C9000E08E70B12068806800F00200022808D100
:106CA00015F8010B21680873E08E401EE0864FF056
:106CB000000BE08F68B12068806800F0010040B1EF
:106CC0002068C06806F8010BE08F401EE0874FF097
:106CD000010B08F1010040B1FFF782F8A0EB0900B9
:106CE000404502D3032001902AE0E08E0028CCD159
:106CF000E08F0028C9D14346012202212046CDF869
:106D0000009005F087FB10B10320019018E04A467F
:106D10004146204605F046FB20B10120019020208D
:106D200060650DE0A06850B900BF002000902068A9
:106D3000C068009020688068009000BF00BF00BF5E
:106D4000012084F8510000BF002084F8500000BFEB
:106D5000019806E7042808D14FF0E021096941F0C5
:106D600004014FF0E022116107E04FF0E0210969D2
:106D700021F004014FF0E02211617047704770B5B7
:106D800004462546681EB0F1807F01D301200FE044
:106D9000681E4FF0E02148610F214FF0FF3004F0F2
:106DA000A9F800204FF0E021886107200861002049
:106DB00070BD10B5FFF7E2FF10BD4FF0E020006995
:106DC00020F002004FF0E0210861704770477047E3
:106DD00010B50346002200BF93F83800012801D106
:106DE000022010BD012083F8380000BF22F0FF0010
:106DF000CC6840EA040222F440708C6840EA040245
:106E000022F480604C6840EA040222F400600C68BE
:106E100040EA040222F480500C6940EA040222F4A1
:106E200000504C6940EA040222F480408C6940EA38
:106E3000040222F400408C6940EA040218684264AB
:106E400000BF002083F8380000BF00BFC9E702463A
:106E500000BF92F83800012801D1022070470120BC
:106E600082F8380000BF022082F8390010684068BC
:106E700020F0700013685860106840680B68184371
:106E8000136858601068806820F08000136898606C
:106E9000106880684B68184313689860012082F876
:106EA000390000BF002082F8380000BF00BFD5E7DE
:106EB00010B50446022084F8390000BF2068006A3B
:106EC00041F21111084050B92068006A8910084049
:106ED00028B92068006820F001002168086000BF20
:106EE000204600F023F8002084F8390000BF84F821
:106EF000380000BF10BD10B504460CB9012010BD0C
:106F000094F8390028B9002084F83800204600F0B1
:106F100021F8022084F83900211D206807F056F876
:106F2000012084F839000020E9E7000010B504468C
:106F300006492068884208D10548006820F0020010
:106F4000034908601D20FEF7CDFF10BD000400407E
:106F50004038024038B504460E492068884217D1AF
:106F600000BF002000900C48006840F002000A4971
:106F700008600846006800F00200009000BF00BFF3
:106F8000002211461D20FEF7C8FF1D20FEF7B8FFA6
:106F900038BD000000040040403802400146086847
:106FA000C06840F001000A68D0600868006840F0DE
:106FB00001000A6810600020704701460868C06838
:106FC00020F001000A68D06000BF0868006A41F242
:106FD0001112104050B90868006A9210104028B988
:106FE0000868006820F001000A68106000BF0020F7
:106FF00070472DE9F04104460D46002600BF94F885
:107000003800012802D10220BDE8F081012084F877
:10701000380000BF022084F839002068866826F016
:10702000770626F47F4620688660286850283BD083
:107030000CDC202860D004DC002853D0102865D157
:1070400055E030285DD0402860D141E0602835D03F
:1070500070280DD0B0F5805F03D0B0F5005F55D13A
:1070600015E02068806820F00700216888604EE005
:10707000D5E902136A68206807F00EF82068866870
:1070800026F0770646F07706206886603FE0D5E96F
:1070900002136A68206806F0FFFF2068806840F4E9
:1070A00080402168886032E0EA686968206807F0FB
:1070B000D5F85021206806F0FBFF28E0EA686968EF
:1070C000206807F0E0F86021206806F0F1FF1EE07C
:1070D000EA686968206807F0C1F84021206806F076
:1070E000E7FF14E00021206806F0E2FF0FE0102126
:1070F000206806F0DDFF0AE02021206806F0D8FFB6
:1071000005E03021206806F0D3FF00E000BF00BF9B
:10711000012084F8390000BF002084F8380000BF47
:1071200000BF71E7704710B5044620680069C0F3DE
:107130004000D8B12068C068C0F34000B0B16FF023
:10714000020021680861012020762068806900F033
:10715000030018B12046FFF7E5FF05E0204600F0E8
:10716000C7F8204600F07EF90020207620680069EC
:10717000C0F38000D8B12068C068C0F38000B0B10F
:107180006FF0040021680861022020762068806981
:1071900000F4407018B12046FFF7C4FF05E0204618
:1071A00000F0A6F8204600F05DF900202076206867
:1071B0000069C0F3C000D8B12068C068C0F3C00047
:1071C000B0B16FF0080021680861042020762068C3
:1071D000C06900F0030018B12046FFF7A3FF05E0E7
:1071E000204600F085F8204600F03CF9002020768B
:1071F00020680069C0F30010D8B12068C068C0F3EF
:107200000010B0B16FF010002168086108202076EE
:107210002068C06900F4407018B12046FFF782FF73
:1072200005E0204600F064F8204600F01BF900203D
:1072300020762068006900F0010058B12068C0681D
:1072400000F0010030B16FF00100216808612046B4
:1072500000F068F920680069C0F3C01058B12068D8
:10726000C068C0F3C01030B16FF0800021680861C1
:107270002046FFF7ABFD20680069C0F3801058B1CD
:107280002068C068C0F3801030B16FF04000216802
:107290000861204600F0D2F920680069C0F3401070
:1072A00058B12068C068C0F3401030B16FF02000C2
:1072B000216808612046FFF78AFD10BD10B586B031
:1072C00004460949206888420CD1C014019002206C
:1072D00002900020039004900120059001A903482A
:1072E000FEF786FC06B010BD000001400000024021
:1072F000704770B504460D46164600BF94F8380036
:10730000012801D1022070BD012084F8380000BF9F
:10731000022084F8390036B1042E1BD0082E31D05B
:107320000C2E5ED145E02946206806F0CBFE206891
:10733000806940F00800216888612068806920F039
:1073400004002168886120688069296908432168F0
:10735000886147E02946206806F0E6FE20688069DB
:1073600040F40060216888612068806920F48060B2
:107370002168886120688069296940EA01202168C4
:1073800088612FE02946206806F006FF2068C06962
:1073900040F008002168C8612068C06920F004003E
:1073A0002168C8612068C069296908432168C861EB
:1073B00018E02946206806F025FF2068C06940F4DF
:1073C00000602168C8612068C06920F4806021687D
:1073D000C8612068C069296940EA01202168C86144
:1073E00000E000BF00BF012084F8390000BF00208A
:1073F00084F8380000BF00BF85E710B504460CB91B
:10740000012010BD94F8390028B9002084F8380014
:10741000204600F00DF8022084F83900211D206874
:1074200006F0D4FD012084F839000020E9E70000CF
:1074300008B50A4A016891420FD100BF00210091AE
:107440000749096841F00101054A116011460968C0
:1074500001F00101009100BF00BF08BD0000014024
:10746000443802407047000030B504460D46012202
:107470002946206806F002FE0A492068884201D1A8
:10748000012000E0002028B12068406C40F400405A
:10749000216848642068006840F0010021680860A5
:1074A000002030BD0000014030B504460D460022EA
:1074B0002946206806F0E2FD19492068884201D17A
:1074C000012000E0002090B100BF2068006A41F276
:1074D0001111084050B92068006A8910084028B985
:1074E0002068406C20F400402168486400BF00BF61
:1074F0002068006A41F21111084050B92068006A02
:107500008910084028B92068006820F0010021682F
:10751000086000BF012084F83900002030BD000061
:107520000000014010B5044635480088401C34492D
:10753000088034480078401C324908703048008880
:10754000B0F57A7F51DB00202D4908802E48008855
:10755000401C2D4908802D4890ED000AF7EE000AE6
:1075600030EE200A80ED000A0120294908702648E3
:1075700000880A2821DDFAF73BFA03281DD000BF56
:1075800000BF00BF00BF00BFBFF34F8F00BF00BFF1
:1075900000BF2048006800F4E0601F490843001D58
:1075A0001C49086000BF00BF00BFBFF34F8F00BF82
:1075B00000BF00BF00BF00BFFDE71848B0F858008B
:1075C00098B94FF400711648FEF7FCFB68B1FAF762
:1075D0000FFA032809D013480368134802681348B8
:1075E00001681348006804F0FFFF0548008811494E
:1075F0000968884202D101200F49087010BD0000BF
:107600001C000020200600201E0000201C06002078
:10761000200000200CED00E00000FA059824002076
:1076200000040240700600206C060020680600205E
:10763000640600203C010020D9010020704710B5ED
:1076400004460CB9012010BD242084F839002046DE
:1076500000F0F2F80020E06384F8390084F83A0082
:1076600000BF84F8380000BF00BFECE710B5044647
:10767000204608F043FD10BD2DE9F0470446206880
:1076800005682068C668206847694FF00008C14651
:1076900005F00F08B8F1000F0AD105F0200038B14D
:1076A00006F0200020B1204606F0B4FFBDE8F087C8
:1076B000B8F1000F6DD007F0010018B906F4907012
:1076C000002866D005F0010030B106F4807018B1D2
:1076D000E06B40F00100E06305F0040030B107F01A
:1076E000010018B1E06B40F00200E06305F0020019
:1076F00030B107F0010018B1E06B40F00400E06326
:1077000005F0080030B107F0010018B1E06B40F05F
:107710000800E063E06B68B305F0200028B106F0D4
:10772000200010B1204606F075FF20684069C0F3C4
:107730008019E06B00F0080010B9B9F1000F22D0F9
:10774000204606F03DFF2068406900F04000B0B1DF
:107750002068406920F0400021684861606B50B1AA
:107760001748616B0865606BFDF776FE10B1606BC2
:10777000016D88470CE02046FFF778FF08E02046BF
:10778000FFF774FF04E02046FFF770FF0020E0637E
:107790008CE705F0800030B106F0800018B120467B
:1077A00007F03AF982E705F0400030B106F04000FA
:1077B00018B1204606F014FF78E700BF76E7000016
:1077C000C5E4020810B504460CB9012010BDA0693B
:1077D00000B100E000BF94F8390028B9002084F817
:1077E0003800204600F082F8242084F83900206810
:1077F000C06820F400502168C860204606F058FF99
:107800002068006920F49040216808612068406980
:1078100020F02A00216848612068C06840F40050C8
:107820002168C8600020E063202084F8390084F8D3
:107830003A000020CAE7000010B504462549206838
:10784000884214D12448006820F0100022490860C2
:107850004FF4C0612148FEF7FBF8606BFDF710FEA6
:10786000206BFDF70DFE2520FEF73CFB30E01C49A8
:107870002068884215D11848001F006820F40030A5
:107880001549091F08600C211448FEF7E1F8606BE8
:10789000FDF7F6FD206BFDF7F3FD2620FEF722FB3A
:1078A00016E010492068884212D10B48006820F089
:1078B000200009490860C0210B48FEF7C9F8606B39
:1078C000FDF7DEFD206BFDF7DBFD4720FEF70AFB31
:1078D00010BD00000010014044380240000002408A
:1078E00000440040001401400008024010B586B07A
:1078F0000446AA49206888426CD100BF002000904D
:10790000A748006840F01000A549086008460068D4
:1079100000F01000009000BF00BF4FF4C060019065
:10792000022002900120039003200490072005907C
:1079300001A99C48FEF75CF99B489C4908604FF000
:1079400000604860002199488160C1604FF4806107
:1079500001610021416181614FF48071C1610021A9
:1079600001624162FDF7DEFE20B140F2651190A098
:1079700008F03EFF00BF8D486063846300BF8A4803
:107980007830924908604FF00060486040218F488D
:1079900081600021C1604FF480610161002141617B
:1079A0008161C16101624162FDF7BCFE20B140F21C
:1079B00077117FA008F01CFF00BF84482063846318
:1079C00000BF002201212520FEF7A7FA2520FEF79F
:1079D00097FAE0E07E49206888426DD100BF002020
:1079E00000906F48001F006840F400306C49091F88
:1079F00008600846006800F40030009000BF00BF37
:107A00000C2001900220029001200390032004909A
:107A10000720059001A96348FEF7EAF86D486E4912
:107A200008604FF00060486000216B488160C160D1
:107A30004FF4806101610021416181614FF48071E7
:107A4000C161002101624162FDF76CFE20B14FF47B
:107A5000D27157A008F0CCFE00BF5F48606384631A
:107A600000BF5C4818305D4908604FF00060486016
:107A700040215A4881600021C1604FF4806101615A
:107A8000002141618161C16101624162FDF74AFEED
:107A900020B14FF4DB7146A008F0AAFE00BF4F48AA
:107AA0002063846300BF002201212620FEF735FAFF
:107AB0002620FEF725FA6EE04949206888426AD1FF
:107AC00000BF002000903648006840F02000344994
:107AD00008600846006800F02000009000BF00BF6A
:107AE000C020019002200290012003900320049006
:107AF0000820059001A93B48FEF77AF82A48183873
:107B00003949086080054860002137488160C160BC
:107B10004FF4806101610021416181614FF4807106
:107B2000C161002101624162FDF7FCFD20B140F21C
:107B3000E3111FA008F05CFE00BF2B486063846364
:107B400000BF19486030294908604FF02060486044
:107B50004021264881600021C1604FF480610161AD
:107B6000002141618161C16101624162FDF7DAFD7D
:107B700020B140F2F5110EA008F03AFE00BF1B48FC
:107B80002063846300BF002201214720FEF7C5F96E
:107B90004720FEF7B5F906B010BD00000010014007
:107BA000443802400000024040640240F8E60020F1
:107BB0002E2E2F5372632F73746D333266347878A0
:107BC0005F68616C5F6D73702E63000058E7002082
:107BD0000044004088600240B8E7002018E8002018
:107BE000001401400008024078E80020D8E8002096
:107BF00077B581B00446154694F83A00202850D154
:107C0000029800B115B9012004B070BD00BF94F80E
:107C10003800012801D10220F6E7012084F838005D
:107C200000BF0298A062A5850020E063222084F8AE
:107C30003A001D48616BC8631C48616B08641C48AE
:107C4000616BC8640020616B086502AE326823680E
:107C5000191D2B46606BFDF7DBFD00BF0020009077
:107C600020680068009020684068009000BF00BF56
:107C700000BF002084F8380000BF2068C06840F4CE
:107C800080702168C8602068406940F00100216868
:107C900048612068406940F0400021684861002048
:107CA000B2E70220B0E7000029E502086FE502080C
:107CB000D9E4020810B5034693F83A00202829D1E8
:107CC00001B10AB9012010BD00BF93F838000128A6
:107CD00001D10220F7E7012083F8380000BF996244
:107CE0009A85DA850020D863222083F83A0000BF05
:107CF000002083F8380000BF1868406940F0010098
:107D00001C6860611868C06840F490701C68E0608E
:107D10000020D8E70220D6E710B50446204608F038
:107D200027FA10BD70472DE9F84304460D46164664
:107D30001F464FF0000994F8390020285CD105B1A6
:107D400016B90120BDE8F88300BF94F83800012877
:107D500001D10220F6E7012084F8380000BF00209E
:107D6000E063212084F83900FEF73AF88146A684C2
:107D7000E6842BE0E08C401EE084A068B0F5805FD4
:107D800016D14B46002280212046009706F078FE4F
:107D900008B10320D6E7A846B8F80000C0F30800F1
:107DA00021684860206908B9AD1C0FE06D1C0DE02A
:107DB0004B46002280212046009706F061FE08B164
:107DC0000320BFE715F8010B21684860E08C00280C
:107DD000D0D14B46002240212046009706F050FEAD
:107DE00008B10320AEE7202084F8390000BF00204E
:107DF00084F8380000BFA5E70220A3E7F7B50446E2
:107E0000154694F8390020283DD1019800B10DB9EC
:107E10000120FEBD00BF94F83800012801D10220E6
:107E2000F7E7012084F8380000BF01982062A5849C
:107E3000E5840020E063212084F839001348216B99
:107E4000C8631348216B08641248216BC864002082
:107E5000216B086501AE23681A1D31682B46206B23
:107E6000FDF7D6FC6FF040002168086000BF0020DD
:107E700084F8380000BF2068406940F08000216825
:107E800048610020C5E70220C3E700007DE5020845
:107E9000B3E50208D9E4020810B5034693F83900A7
:107EA000202823D101B10AB9012010BD00BF93F8E9
:107EB0003800012801D10220F7E7012083F83800BB
:107EC00000BF19629A84DA840020D863212083F8E5
:107ED000390000BF002083F8380000BF1868C06870
:107EE00040F080001C68E0600020DEE70220DCE754
:107EF00010B50446204608F071FA10BD70472DE910
:107F0000FE4304460025A8460026002002900027D4
:107F10000CB1606808B9BDE8FE83A068402800D9AC
:107F2000F9E700252CE0204600F0DEF82E464FF061
:107F300000081DE0606A825D02AB4146204600F009
:107F40007CF90746022F0DD1606A0090E06A01902B
:107F50006068029A00EBC2006A464168204600F061
:107F6000A1F808E007B906E000BF761C08F1010897
:107F7000E06AB042DED800BF022F00D103E06D1CE2
:107F8000E06AA842CFD800BF00BFC4E70FB438B53D
:107F900004460D4607A80090D4E90601009B069A06
:107FA00008F064FC20620020009008480078012856
:107FB00003D1216AA06900F047FB29462046236AC5
:107FC000A26900F00DF838BC5DF814FBEC06002047
:107FD00010B50446A06B01F0A9FA002010BD000006
:107FE000F8B504460D4616461F463A463146204629
:107FF0006369984750B92046FFF7EAFF0094084BA1
:108000002A460021A06B01F033FB06E00094054BEB
:1080100001220021A06B01F02BFB0020F8BD000025
:10802000698102085981020870B504460D46802115
:10803000204601F0C9FB2868E06368686060A868B2
:10804000A060E868E0602869206168696061A869EB
:10805000A061E869E06100202062286A6062686AC5
:10806000A0620020E06284F83000A86A606304F136
:10807000380001F071FA10B14FF0FF3070BD2046AA
:1080800000F002F8FAE70000014611B94FF0FF30A6
:108090007047034800680860014801600020F7E766
:1080A000E806002070B504460D461646022D06D09F
:1080B000032D05D0042D04D0052D07D102E000BF0B
:1080C00000BF00BF2046FFF783FF00E000BF00BFF6
:1080D00032462946E06B00F0C5FA70BD01480078D1
:1080E00070470000EC06002010B504460122402134
:1080F00004F14000F8F7BDF810BD000010B50024F1
:10810000124804681EE0204621698847C8B9104813
:108110000078012810D1E16A606A01F0C5FB0128EE
:1081200003D1606A00F0B0F906E0E16A606A00F02D
:1081300051FA08A000F0A8F92046FFF7E0FE002061
:10814000E0622468002CDED110BD0000E8060020AB
:10815000EC0600200D0A000010B50446002205219F
:108160002046FFF79FFF10BD10B5044600220421F2
:108170002046FFF797FF10BD70B504460D46204618
:1081800000F02FF8012801D1801E70BD2068401C2E
:10819000E168B0FBF1F201FB120020602669236860
:1081A000A16803FB061032462946F8F750F8002074
:1081B000EBE710B58160C2600361012444600024D4
:1081C000046010BD01460868401CCA68B0FBF2F3A9
:1081D00002FB13004A68904201D101207047002041
:1081E000FCE701460868801CCA68B0FBF2F302FB9A
:1081F00013004A68904201D1012070470020FCE73B
:1082000070B504460D462046FFF7DCFF012801D17A
:10821000801E70BD2669D4E9013003FB0601324699
:108220002846F8F714F86068401CE168B0FBF1F2EA
:1082300001FB120060600020EBE7F0B504460D463C
:10824000002600211BE004F14000405C012815D10C
:10825000606850F83100405D904204D0002704F17E
:10826000400047540AE0761C606850F83170681C82
:10827000385C18B903B119600220F0BD491CA06830
:108280008842E0D80EB90020F7E70120F5E70000AA
:108290002DE9F04104460D469C46002700210023AD
:1082A000344E15B9481EBDE8F0810320B5FBF0F847
:1082B00000FB185020B90320B5FBF0F0870004E064
:1082C0000320B5FBF0F0401C8700781C844502D2E7
:1082D0004FF0FF30E7E70020D055002100232AE0CF
:1082E000E05C06EBA00000785054E05C80074FEAA9
:1082F0009068581C205C48EA201016F80080481C42
:1083000002F80080581C205C00074FEA9068981C17
:10831000205C48EAA01016F80080881C02F8008053
:10832000981C205C00F03F0016F80080C81C02F882
:108330000080DB1C091DB81E8842D1D80320B5FB84
:10834000F0F800FB1850012802D002280FD108E0F5
:108350004FF03D08881E02F80080481E02F8008099
:1083600005E04FF03D08481E02F8008000BF00BF46
:10837000002098E7DC38030810B5024612B94FF028
:10838000FF3010BD00BF10688842FCD31068401A4F
:10839000106050680844D368B0FBF3F403FB14008A
:1083A00050600020EDE710B5024612B94FF0FF30E3
:1083B00010BD10680844106000BFD3681068984270
:1083C000FBD890680844D368B0FBF3F403FB1400B7
:1083D00090600020ECE7F0B50446002522B11BB107
:1083E000E6682068B04202D34FF0FF30F0BD266847
:1083F000E068801B884202D24FF0FF30F6E7A068A9
:108400000844E668B0420BD9D4E90260851B2668AF
:10841000E068801B4E19B04202D24FF0FF30E5E712
:10842000A0682844E668B0FBF6F706FB170010606A
:10843000681818600020D9E701464868704701466F
:1084400088687047024612B94FF0FF30704700202D
:10845000506090601060D16000BFF7E7014609B935
:1084600001207047086808B90120FAE70020F8E702
:10847000014609B9012070470A68C868904201D1D5
:108480000120F8E70020F6E70FB410B5ADF5027D46
:10849000F9F7AEFA28B100200DF5027D10BC5DF8A9
:1084A00014FB002485A881904FF4007101A8819BE2
:1084B000849A08F0DBF9044600208190B4F5007F2F
:1084C00001D340F2FF14224601A9002007F0B0FEBC
:1084D0000020E1E70FB410B5ADF5027D002485A8BA
:1084E00081904FF4007101A8819B849A08F0BEF935
:1084F000044600208190B4F5007F01D340F2FF14C0
:10850000224601A9002007F093FE00200DF5027D10
:1085100010BC5DF814FB00000FB430B5ADF5097D5B
:10852000F9F766FA28B100200DF5097D30BC5DF839
:1085300014FB0024FDF754FC4FF47A71B0FBF1F208
:1085400001FB12059DF81E009DF81D109DF81C20D2
:10855000CDE90405CDE902219DF81B009DF81A1014
:10856000CDE90010BDF8183011A24FF4007108A831
:1085700001F0A7FA0446224608A9002007F058FE99
:108580008DA888904FF4007108A8889B8C9A08F0F9
:108590006DF9044600208890B4F5007F01D340F2C5
:1085A000FF14224608A9002007F042FE0020BBE786
:1085B000253034752D253032752D25303275202526
:1085C0003032753A253032753A253032752E2530E5
:1085D00033752000F0B591B006460C46F9F708FA5D
:1085E00010B1002011B0F0BD002515480078012819
:1085F00001D00020F6E700BF102C01D9102500E0C3
:108600002546402101A8F7F73BFE0120402301AA9F
:1086100029460090304601F08BF80AA101A8F7F72F
:108620003AFE01A8F7F75FFE07463A4601A9002087
:1086300007F0FEFD641B2E44002CDDD10020D1E7A5
:108640007C0300200D0A000070B504460D46F9F7C2
:10865000CFF908B1002070BD2A462146002007F05E
:10866000E7FDF8E72DE9FC4104460D4617464FF0BB
:1086700000080026608801281FD1206950B9606871
:108680000068CDE900051AA200212046E368FBF747
:10869000F7FF12E0206950F8250000782D280CD053
:1086A000206950F8250061680968CDE9001018A21A
:1086B00000212046E368FBF7E3FF66683A46294657
:1086C0002046F368984780460BE0706840B17068B8
:1086D0003A462946C368204698478046766800E0B7
:1086E00002E0B8F1010FF0D000BFBDE8FC8100004E
:1086F00046534D3A252D38732053544154453A255D
:108700002D323873204556454E543A25750D0A00D2
:1087100046534D3A252D38732053544154453A253C
:108720002D323873204556454E543A25730D0A00B4
:108730002DE9F04704460E4617469846DDE9089AAB
:1087400000250CB9BDE8F08730212046F7F798FDE9
:10875000C4F80890C4F810806660E7600021A16248
:1087600061620E4800882080A4F802A00C480068CE
:1087700060610B48046009480088401C0749088074
:10878000656806E06560002211462046FFF76AFF33
:10879000AD68002DF6D100BFD4E70000CC06002064
:1087A000C8060020024612B94FF0FF307047D16270
:1087B0000020FBE72DE9F84305460E4617461C4608
:1087C000DDF820904FF000082188484661F31F40F3
:1087D0008046054B3A4631462846CDF8008000F0E9
:1087E00047FFBDE8F8830000F54602082DE9F04197
:1087F00096B005460E461746D5F8048000240020A2
:108800001590444629E06C60002201212846FFF7BC
:1088100029FFA64205D13A4600212846FFF722FF4C
:108820001DE0502101A8F7F72BFD15AB01AA214649
:108830003046FBF740FF78B90AE015980068686099
:108840003A4600212846FFF70DFF1598406815901D
:1088500015980028F1D102E06468002CD3D100BF44
:10886000B46806E06C603A4600212846FFF7FAFE3D
:10887000A468002CF6D116B0BDE8F081016E05E0C9
:1088800000F17C024B1CD35C5354491CC26D8A42DC
:10889000F6D8704710B5C26D511E05E000F17C029C
:1088A000545C4B1CD454491E026E8A42F6DD10BD46
:1088B00070B505460C46A87910B101282ED100E00C
:1088C00000BF432C1BD004DC412C0CD0422C22D105
:1088D0000FE0442C19D07E2C1DD1002208212846FF
:1088E00000F028FB18E000220321284600F022FBBC
:1088F00012E000220421284600F01CFB0CE00022BC
:108900000621284600F016FB06E000220521284635
:1089100000F010FB00E000BF00BF2CE0432C1BD098
:1089200004DC412C0CD0422C22D10FE0442C19D075
:108930007E2C1DD100220821284600F07FF818E087
:1089400000220321284600F079F812E000220421D9
:10895000284600F073F80CE000220621284600F0BB
:108960006DF806E000220521284600F067F800E0D7
:1089700000BF00BF00BF00BF70BD70B504460D460C
:10898000432D45D008DC1B2D0DD0332D24D0412D97
:108990003CD0422D4CD13AE0442D3AD05B2D10D042
:1089A0007E2D45D123E0207910B1042804D100E0C8
:1089B00000BF0120207102E00020207100BF00BF35
:1089C00039E02079012802D10220207102E0002044
:1089D000207100BF00BF2EE02079022802D10320C1
:1089E000207102E00020207100BF00BF23E0207949
:1089F000032806D129462046FFF75AFF042020719C
:108A000002E00020207100BF00BF14E000BF00BFE3
:108A100000BF2079022806D129462046FFF748FFEB
:108A20000420207102E00020207100BF00BF02E09E
:108A30000020207100BF00BF207970BD2DE9F041FA
:108A400004460D461746092D02D00020A066E066B8
:108A50000A2D6FD2DFE805F06E0540CDFDFCFBFA74
:108A6000F9F8607910B1012833D100E000BFE06D62
:108A700063282BD23846D4F8981588472046FFF74C
:108A800009FF04F17C00216E4754206E401C2066D3
:108A9000E06D401CE065266E4FF0000808E004F130
:108AA0007C02905DD4F898158847761C08F101087F
:108AB000E06DB042F3D803E00820D4F89815884759
:108AC000B8F10000A8F10108F6D100BF00206071E4
:108AD00000E000BF00BF28E2E06D20B9FEA0D4F89E
:108AE0009415884721E2607910B1012866D122E00F
:108AF000002104F17C00E26D8154616F01EBC10241
:108B000002EB011204F5A27101EB8200C839F7F7FC
:108B10000CFC606F401C6067606F0A2801DB00205E
:108B20006067A06F401CA067A06F0A2801D30A20CD
:108B3000A06744E0F8E100BF00BF206F00EBC00277
:108B400002EB001204F5A27000EB8201642204F231
:108B50002C50F7F77CFB266F19E0701C0A21B0FB44
:108B6000F1F201FB120808EBC80202EB081304F54E
:108B7000A27202EB830106EBC60202EB061304F5B8
:108B8000A27202EB83006422F7F761FB4646606F36
:108B900009300A2190FBF1F201FB1200B042DCD156
:108BA00006EBC60101EB061204F5A27101EB82008F
:108BB000642204F22C51F7F74AFB00E000BF00BF2B
:108BC000C6A0D4F894158847204600F0A9FC04F10B
:108BD0007C0000F007FC002000F0A2FC00202066D2
:108BE000E065606F0A302067BDA0D4F8941588470F
:108BF0009BE1607910B1012853D100E000BFA06F64
:108C000000B94FE0A06F0A2803D1D4E91C018842C3
:108C10000ED1A06F0A2841D0606F0A30A16F401AB0
:108C20000A21B0FBF1F201FB1200216F884235D01E
:108C3000206F09300A21B0FBF1F201FB120020671E
:108C4000206F00EBC00205E008E1CCE08EE07EE0A2
:108C500072E029E002EB001204F5A27000EB820141
:108C6000C838F7F762FB04F17C00F7F73CFBE065DE
:108C7000E06D20669BA0D4F894158847226F02EB24
:108C8000C20303EB021304F5A27202EB8300D4F8D3
:108C90009415884794A0D4F89415884701206071F2
:108CA00000E000BF00BF40E1607910B1012840D171
:108CB00000E000BFA06F00B93CE0606F09300A21FE
:108CC00090FBF1F201FB1200216F88422ED0206F41
:108CD000401C0A21B0FBF1F201FB12002067206F5B
:108CE00000EBC00202EB001204F5A27000EB82015F
:108CF000C838F7F71AFB04F17C00F7F7F4FAE065DF
:108D0000E06D206677A0D4F894158847226F02EBB7
:108D1000C20303EB021304F5A27202EB8300D4F842
:108D20009415884770A0D4F8941588470120607185
:108D300000E000BF00BFF8E0206E002806DD206ED6
:108D4000401E20660820D4F898158847EDE0D4E945
:108D50001710884209D204F17C02236ED05CD4F84B
:108D600098158847206E401C2066DEE0607910B1BF
:108D7000012835D100E000BFE06D70B3206E0028FF
:108D80002BDD0820D4F898158847266E4FF001088F
:108D900008E004F17C02905DD4F898158847761CB1
:108DA00008F10108E06DB042F3D82020D4F89815FE
:108DB000884703E00820D4F898158847B8F10000E8
:108DC000A8F10108F6D1206E401E20662046FFF76C
:108DD00055FDE06D401EE06500BF0020607100E0C1
:108DE00000BF00BFA1E0607910B1012833D100E0DD
:108DF00000BFE06D60B3206E002829DDD4E91701C3
:108E0000884225D0206E461C4FF0010808E004F18E
:108E10007C02905DD4F898158847761C08F101080B
:108E2000E06DB042F3D82020D4F89815884703E0CD
:108E30000820D4F898158847B8F10000A8F1010877
:108E4000F6D12046FFF71AFDE06D401EE06500BF39
:108E50000020607100E000BF00BF66E0607910B1E3
:108E600001285ED100E000BFE06D98B3E06E50B91C
:108E70000120E06604F17C0104F1E000E26DF7F707
:108E8000E6F9E06D60663CE0A06E00F0F1FA06469F
:108E900004F1E001626EF7F751FAE0B913A0D4F8DB
:108EA00094158847A06E00F0E3FA0646D4F89415AE
:108EB0008847A06E00F0DCFA0646314604F17C00DB
:108EC000F7F733FA04F17C00F7F70DFAE065E06D8F
:108ED00020660FE022E011E00D0A3E000D0A0000BE
:108EE0003E0000000D3E00001B5B4A000D1B5B4A6C
:108EF0003E000000A06E401CA06607E0A06E401C73
:108F0000A06600F0AFFAA16E8842BDD800BF00F0A5
:108F1000A9FAA16E884201D80020A06600206071E5
:108F200000E000BF00BF00E000BF00BFBDE8F0816F
:108F3000002070472DE9F04104460E461746092EE1
:108F40007DD2DFE806F07C05457C7C9BA6BDF80061
:108F5000E06D63283BD2A079012804D12A20D4F8FF
:108F60009815884703E03846D4F898158847204676
:108F7000FFF790FC04F17C00216E4754206E401CEA
:108F80002066E06D401CE065256E4FF0000810E0A3
:108F9000A079012804D12A20D4F89815884705E043
:108FA00004F17C02505DD4F8981588476D1C08F1D7
:108FB0000108E06DA842EBD803E00820D4F898152A
:108FC0008847B8F10000A8F10108F6D1ECE0EBE029
:108FD000E06D30B9A07920B975A0D4F89415884710
:108FE000E2E0A07910B1012845D115E0002104F19B
:108FF0007C00E26D815472A0D4F89415884701205A
:10900000A07100202066E06504F17C02102104F1CB
:109010000C0000F056FD2FE0002104F17C00E26D11
:1090200081540020E06504F17C02402104F11C0021
:1090300000F047FD04F11C0104F10C0000E0B2E077
:1090400000F070F950B962A0D4F894158847022056
:10905000A07100202066E06560710BE060A0D4F88C
:109060009415884752A0D4F8941588470020A07121
:109070002066E06500E000BF00BF95E0206E00289C
:1090800006DD206E401E20660820D4F8981588471B
:109090008AE0D4E91710884211D2A079012804D1BE
:1090A0002A20D4F89815884706E004F17C02236E44
:1090B000D05CD4F898158847206E401C206673E079
:1090C000E06DB0B3206E002833DD0820D4F8981589
:1090D0008847256E4FF0010810E0A079012804D1DF
:1090E0002A20D4F89815884705E004F17C02505DE9
:1090F000D4F8981588476D1C08F10108E06DA84266
:10910000EBD82020D4F89815884703E00820D4F83D
:1091100098158847B8F10000A8F10108F6D1206E33
:10912000401E20662046FFF7A9FBE06D401EE0656B
:1091300000BF39E0FFE7E06DA0B3206E002831DD0D
:10914000D4E9170188422DD0206E451C4FF001084C
:1091500010E0A079012804D12A20D4F89815884776
:1091600005E004F17C02505DD4F8981588476D1C29
:1091700008F10108E06DA842EBD82020D4F898153A
:10918000884703E00820D4F898158847B8F1000014
:10919000A8F10108F6D12046FFF770FBE06D401EF4
:1091A000E06500BF00E000BF00BFBDE8F081000047
:1091B0000D0A757365726E616D653A2000000000DE
:1091C0000D0A70617373776F72643A2000000000BB
:1091D0000D0A57656C636F6D65210D0A3E00000036
:1091E0000D0A55736572207665726966792066612D
:1091F000696C65642E00000038B5002000900024E2
:10920000424804687EE076E000F0D6F905469DF815
:1092100000102046FFF7B1FB00B16CE0FFF788FEBD
:1092200001280AD1A068281A3949884207D9A560BF
:109230000020A071E065206601E00220A071A07905
:1092400010B101282BD100E000BF9DF800000D28CF
:1092500006D19DF8002002212046FFF76BFE1DE09D
:109260009DF800000A2819D09DF80000082805D1B3
:10927000002207212046FFF75DFE0FE09DF8000069
:10928000092805D1002209212046FFF753FE05E0F9
:109290009DF8002001212046FFF74CFE29E09DF8B3
:1092A00000000D2806D19DF8002002212046FFF77E
:1092B000C5FB1DE09DF800000A2819D09DF80000AC
:1092C000082805D1002207212046FFF7B7FB0FE051
:1092D0009DF80000092805D1002209212046FFF74A
:1092E000ADFB05E09DF8002001212046FFF7A6FB1D
:1092F00000BF00BF00BF6846D4F89C15884700280F
:1093000082D02468002C7FF47EAF38BDF0060020A8
:1093100040771B00024909680160014908607047F5
:10932000F0060020024600207047000000BFEFF367
:10933000058000B170470748006820B9012080F31C
:10934000108800BF00BF03480068401C0149086046
:1093500000BFEFE7D006002070B504460D4600F0D0
:1093600099F850B100F096F8D0F8900528B100F0C7
:1093700091F8D0F8901502A08847002070BD000039
:109380001B5B481B5B4A000030B502460C460021BF
:10939000002302B114B94FF0FF3030BD002100238B
:1093A00015E00E4850F8310080B952F833000B4DEB
:1093B00045F8310002EBC300406805EBC105686069
:1093C00007480068401C064D28605B1C491C50295A
:1093D00001D2A342E5D30020DFE70000FC06002015
:1093E000F8060020F0B595B00446002600E0641CA5
:1093F00020782028FBD02046F6F775FF10B9002012
:1094000015B0F0BD2046F6F76EFF2044461E02E080
:1094100000203070761E30782028F9D0142301AA5D
:109420002021204600F064FB0746002511E00C498E
:1094300051F835002146F6F75DFF48B9084800EBC2
:10944000C50001A942683846904700B905E004E02C
:109450006D1C00F007F8A842E9D800BF0020CFE754
:10946000FC0600200148006870470000F806002054
:10947000014605480068814201D304A070470448B2
:1094800050F83100FAE70000F80600200000000064
:10949000FC0600200148006870470000F406002028
:1094A0002DE9F04106460F4600252AE0002412E08F
:1094B000FFF7F0FF70B1FFF7EDFFD0F8900548B16E
:1094C000FFF7E8FFD0F890252819114B53F830101A
:1094D00010A09047641C052C04DAFFF7C3FF29197C
:1094E0008842E5D8FFF7D6FF50B1FFF7D3FFD0F899
:1094F000900528B1FFF7CEFFD0F8901507A0884758
:109500006D1DFFF7AFFFA842D0D80020BDE8F08165
:10951000FC060020252D3136730000000D0A0000E6
:109520000149086070470000F40600200146202928
:1095300002D34FF0FF3070470120C1EBC102054B51
:1095400043F822000020C1EBC10203EB8202D0608D
:1095500000BFF0E758E9002070B5054600240DB9BA
:10956000601E70BD00240DE0C4EBC4000C4951F82E
:10957000200030B90120C4EBC401094A42F821009F
:1095800002E0641C202CEFD300BF202C05D105A0E5
:10959000FEF77AFF4FF0FF30E3E72C600020E0E7B2
:1095A00058E9002074696D65722049442069732070
:1095B00066756C6C0D0A0000014800687047000079
:1095C000D806002010B5002400BF4AE0C4EBC40058
:1095D000254951F82000022842D1C4EBC40001EB18
:1095E0008000C06821490968081AC4EBC4011E4AFA
:1095F00002EB81010969884232D9C4EBC4001146EB
:1096000001EB8000806928B3C4EBC40001EB80004B
:10961000007928B90120C4EBC40142F821000CE014
:109620000220C4EBC401104A42F821000F48006830
:10963000C4EBC40102EB8101C860C4EBC4020A4B55
:1096400003EB82025069C4EBC40203EB820291690E
:10965000884705E00120C4EBC401034A42F8210019
:10966000641C202CB2D310BD58E90020D80600207D
:10967000F0B50446059D202C02D34FF0FF30F0BD1D
:109680000220C4EBC406114F47F82600C4EBC40007
:109690003E4606EB800001710D480068C4EBC4062D
:1096A00007EB8606F060C4EBC4003E4606EB800084
:1096B0000261C4EBC40006EB80008361C4EBC4000C
:1096C00006EB800045610020D9E7000058E9002042
:1096D000D806002007480068401C06490860064874
:1096E00002684068521C40F1000003490A6048606B
:1096F00070470000D8060020E006002000BFEFF30E
:10970000058000B170470948006820B1074800682B
:10971000401E064908600548006820B9002080F313
:10972000108800BF00BF00BFECE70000D00600209B
:109730002DE9F04305460C469846079F0026002376
:1097400099460DB102B114B90020BDE8F083012F94
:1097500001D1032000E002206043401C404501D9B4
:109760000020F2E7002618E015F806904FEA1910DD
:1097700000F019F819465B1C505409F00F0000F076
:1097800012F819465B1C5054012F05D14FF0200CE4
:1097900018465B1C02F800C0761CA642E4D30020E9
:1097A000D0541846D1E70146092903DC01F1300005
:1097B000C0B270470A2905DB0F2903DC01F137002D
:1097C000C0B2F6E73020F4E770B504460D462946EE
:1097D0002046F6F755FD70BD0146302904DB3929D6
:1097E00002DCA1F130000EE0412904DB462902DC55
:1097F000A1F1370007E0612904DB662902DCA1F151
:10980000570000E00020C0B2704710B502460B467A
:10981000002406E01078FFF7DFFF00EB0414521C71
:109820005B1E002BF6D1204610BD00B5024600237A
:1098300005E01078FFF7D0FF00EB0313521C1078FF
:109840000028F6D1184600BD70B588B005460C4614
:10985000002007900690059004902846F6F743FDF7
:10986000064604A805A906AA07ABCDE90021029087
:109870000AA23146284600F031F8042803D04FF000
:10988000FF3008B070BD079820700698607005988A
:10989000A0700498E0700020F3E7000025642E25F6
:1098A000642E25642E25640002460B46002100BF6D
:1098B00010E0505C202803DB505C7E2800DC08E0D0
:1098C000505C0D2802D0505C0A2800D101E0002035
:1098D0007047491C9942ECD30120F9E70FB42DE9F8
:1098E000F8470446002000900022202600270CB1F3
:1098F0000B9820B90020BDE8F8075DF814FB0CA810
:109900000090D4E041B90B980078252803D10B983A
:109910004078652800D0CFE00B980078252874D1D6
:109920000B98401C0B900B9810F8016B0B90652E58
:109930006CD004DC2A2E07D0642E68D113E0702E80
:109940007AD0782EF9D144E008E020780B9B1B7880
:10995000984202D0641C491E00E001E00029F4D1C5
:1099600000BF521C92E04FF0000CE046002300259F
:109970002020DDF8009059F8045BCDF800901AE043
:109980002078B8F1000F06D12D2804D14FF0010C3A
:109990004FF001080DE030280ADB392808DC4FF0D1
:1099A0000108A0F1300903EB830A09EB4A0300E048
:1099B00003E0641C491E0029E2D100BFBCF1010F85
:1099C00003D16FEA030909F1010305B12B60521CB1
:1099D0005CE000230025DDF800C05CF8045BCDF8F6
:1099E00000C022E02078302806DB392804DCA0F112
:1099F000300C0CEB031316E0612809DB662807DC4A
:109A0000A0F1570C0CEB03130DE043E033E03AE018
:109A1000412807DB462805DCA0F1370C0CEB0313CB
:109A200001E009E003E0641C491E0029DAD100BF0F
:109A300005B12B60521C29E0DDF800C05CF8040B76
:109A4000CDF800C00025002325460CE094F800C0A6
:109A5000DDF82C8098F80080C44501D05B1C00E044
:109A600003E0641C491E0029F0D100BF08B1056065
:109A70004360521C0AE0009B01CB009300B10460DC
:109A8000521C012702E00127002200BF00BF012F66
:109A90000DD111E020780B9B1B78984205D1641CF6
:109AA0000B98401C0B90491E01E0002204E00B982B
:109AB000007800287FF426AF00BF002000901046F9
:109AC00019E70FB4F8B506460C46002509A8009022
:109AD00021463046009B089A06F0C8FE0546002045
:109AE0000090A54200D3651E2846F8BC5DF814FB23
:109AF000F0B504460E461D46214600230DB104B1C3
:109B00000AB90020F0BD18465B1C42F820100AE09C
:109B10000878B04206D100200870481C1F465B1C24
:109B200042F82700491C087808B1AB42F0D3184628
:109B3000E8E770B506460025002478213046F6F7A0
:109B4000C8FB044624B958213046F6F7C2FB044648
:109B50005CB1641C05E02078FFF73EFE00EB0515C4
:109B6000641C20780028F6D103E03046F6F7F5FBB8
:109B70000546284670BD2DE9F04106460F461446BD
:109B80003846F6F7B0FB054615B93046BDE8F0811A
:109B9000A54201D90020F9E709E0641E2A463946AA
:109BA0003046F6F7B5FB08B93046EFE7761CAC4215
:109BB000F3D20020EAE770B504460D4604B115B9AA
:109BC0004FF0FF3070BD012104F11000FEF7D4FB0F
:109BD00004F12000A968FEF7CFFB0020F2E770B582
:109BE00004460D4604B115B94FF0FF3070BD012198
:109BF00004F11000FEF7D7FB04F12000A968FEF77E
:109C0000D2FB0020F2E710B504460CB9002010BDCD
:109C100004F11000FEF722FC012801D10020F6E734
:109C200004F12000FEF71AFC012801D10020EEE724
:109C300004F11000FEF700FC00EB4000216801EB8E
:109C40008000E4E77CB504460E4600250020019024
:109C5000009004B97CBD04F11000FEF709FC08B1C6
:109C60000020F7E76B4601AA314604F12000FEF719
:109C7000B2FB08B10020EDE704F11000FEF7DFFBB6
:109C800000EB4000216801EB8005A06801990844C1
:109C900028606E600098A8602846DBE72DE9F04157
:109CA00004460E4617461D464FF0000805EB4500DA
:109CB000B7EB800F03D84FF0FF30BDE8F08105EB24
:109CC00045004FEA80082660C4F80480606830448C
:109CD000A060A7EB0801E160294604F11000FEF73F
:109CE000B1FB04F12000E168FEF7ACFB0020E4E7E3
:109CF00010B5044621460CA0FEF7C6FB10480078BC
:109D000068B11048006803F0C5FD012804D00D4873
:109D1000006803F0D5FC02E00020094908700A48F9
:109D20000068FFF703FC10BD4572726F72206F630D
:109D3000637572726564204025730D0A000000008F
:109D40005C050020600500206405002038B504464D
:109D50000D463548007802282BD134480068C828C1
:109D600021D12CB932A0FFF7C3FF4FF0FF3038BD2F
:109D7000002060552B46224636493748FBF7F6F857
:109D800028B136A0FFF7B4FF4FF0FF30EFE7042013
:109D900002F040FC3A48008882B23A493A480068EA
:109DA00003F0D6FC3DE039A0FFF7A2FF4FF0FF30F3
:109DB000DDE71D480078032819D11C480068C82831
:109DC0000FD1052002F026FC002039490860394BEC
:109DD0004EF660220146009037480068FFF748FCC5
:109DE0001FE036A0FFF784FF4FF0FF30BFE70E48BB
:109DF0000078052815D12CB939A0FFF779FF4FF06D
:109E0000FF30B4E700202B4B4EF660220146009055
:109E100029480068FFF72CFC2A462146C820F7F79E
:109E200075FD0020A3E700005C05002080050020F0
:109E30002E2E5C464D4C5C496E7465726E65745C8A
:109E40004E54524950436C69656E742E633A3332F6
:109E50003000000054C4002074C400202E2E5C4644
:109E60004D4C5C496E7465726E65745C4E5452491B
:109E700050436C69656E742E633A333237000000CC
:109E800070050020D4C30020600500202E2E5C4603
:109E90004D4C5C496E7465726E65745C4E545249EB
:109EA00050436C69656E742E633A3333360000009C
:109EB0007805002075E40208640500202E2E5C461B
:109EC0004D4C5C496E7465726E65745C4E545249BB
:109ED00050436C69656E742E633A33353000000070
:109EE0002E2E5C464D4C5C496E7465726E65745CDA
:109EF0004E54524950436C69656E742E633A333543
:109F00003800000005E003A109A006F073FC05F08D
:109F1000A9FBF8E72E2E2F5372632F73746D333223
:109F2000663478785F69742E633A38350000000033
:109F30002573205552545265737461727400000089
:109F40002DE9F04106460C46002514E016F8017B89
:109F50003A111449022303FB051013A106F072FC09
:109F600007F00F026900491C0E4BC8180EA106F03D
:109F700069FC681CC5B2A542E8DB0D20094A02F85D
:109F800014000A216000401C1154F7F731FD02282B
:109F900005D16000821C0349002006F049F9BDE8A4
:109FA000F08100005E1C00202578000010B5002222
:109FB0004FF400510D48FBF70DFF00224FF4804194
:109FC0000A48FBF707FF0A2007F0F5F901225103C1
:109FD0000648FBF7FFFE0A2007F0EDF900224FF4D8
:109FE00000510248FBF7F6FE10BD000000040240DD
:109FF00010B500224FF400510C48FBF7EBFE012294
:10A0000091030A48FBF7E6FE0A2007F0D4F9012283
:10A0100051030648FBF7DEFE0A2007F0CCF90022C8
:10A020004FF400510148FBF7D5FE10BD000402407B
:10A0300070B50546002400261CE000224FF40051B4
:10A040001148FBF7C7FE0A2007F0B5F901225103BA
:10A050000D48FBF7BFFE6006040E4FF480410A482E
:10A06000FBF7B0FE08B1601CC4B2052007F0A3F9ED
:10A07000701CC6B2082EE0DB15B9FFF7B9FF01E08E
:10A08000FFF794FF204670BD0004024070B50446FF
:10A0900000224FF400511748FBF79CFE002525E0F5
:10A0A000E00928B1012291031248FBF793FE05E075
:10A0B00000224FF480410F48FBF78CFE6006040E2F
:10A0C0000A2007F078F9012251030A48FBF782FEC3
:10A0D0000A2007F070F900224FF400510548FBF701
:10A0E00079FE0A2007F067F9681CC5B2082DD7DB96
:10A0F00070BD00000004024010B5012291030C481D
:10A10000FBF768FE012251030948FBF763FE0022BA
:10A110004FF480410648FBF75DFE0A2007F04BF93B
:10A1200000224FF400510248FBF754FE10BD00001E
:10A130000004024010B500224FF400510C48FBF718
:10A1400049FE00224FF480410948FBF743FE0A20F4
:10A1500007F031F9012251030548FBF73BFE0122CC
:10A1600091030348FBF736FE0A2007F024F910BDDF
:10A170000004024010B50024012291031248FBF7AD
:10A1800029FE062007F017F9012251030E48FBF7BC
:10A1900021FE062007F00FF907E0601CC4B2FA2C7C
:10A1A00003DDFFF7C7FF012010BD4FF480410648D3
:10A1B000FBF708FE0028F0D100224FF400510248BE
:10A1C000FBF708FE0020EFE70004024010B5154839
:10A1D000808A00EE100AB8EE400A1348D0ED000A5B
:10A1E000B4EEE00AF1EE10FA03D201200F49087034
:10A1F00002E000200D4908700A48408F00EE100A66
:10A20000B8EE400A0848D0ED000AB4EEE00AF1EEDC
:10A2100010FA05D20348C08F012801D107F022FEB1
:10A2200010BD0000982400201C060020080000201B
:10A2300010B50F48B0F86000012809D100200C4982
:10A24000A1F860000BA110A006F0D4FA05F00AFAFC
:10A250000748008845F2AA51884202D10448C088C4
:10A2600028B90DA108A006F0C5FA05F0FBF910BD4C
:10A27000982400202E2E5C41504C5C7577625F6103
:10A2800070702E633A39340025732055525452654C
:10A2900073746172740000002E2E5C41504C5C752A
:10A2A00077625F6170702E633A39390010B5F8F744
:10A2B00021FB10B14FF0FF3010BD04F04DF810B18C
:10A2C0004FF0FF30F8E703F0FDFF10B14FF0FF3023
:10A2D000F2E70020F0E710B5F9F770FD10BD0000BF
:10A2E00010B500220F210248FEF7BCF9002010BD76
:10A2F0008CC3002010B5FFF7EEFF012804D14FF406
:10A300000800074908600AE00648007820B14FF4C9
:10A3100008400349086002E000200149086010BDC0
:10A320006C0600201602002010B53721202000F016
:10A3300079F80321212000F075F84021222000F057
:10A3400071F80821232000F06DF8AA21302000F0D8
:10A3500069F801200B490887084690F83810322028
:10A3600000F060F80221332000F05CF85F2120202B
:10A3700000F058F8044800F009F80A2007F01BF82C
:10A3800010BD0000982400205506002010B504469A
:10A3900021460F2000F023F808B9002010BD01204D
:10A3A000FCE770B504460025FFF7A6FE3220FFF754
:10A3B0006DFEFFF7DFFEE0B2FFF768FEFFF7DAFEA3
:10A3C000FFF79AFE3320FFF761FEFFF7D3FE002070
:10A3D000FFF72EFE0546FFF7ADFE284670BD70B5AF
:10A3E00005460C462846FFF7DCFF2070012070BDB3
:10A3F00070B504460D46FFF77FFE3220FFF746FE9C
:10A40000FFF7B8FEE0B2FFF741FEFFF7B3FE2846C4
:10A41000FFF73CFEFFF7AEFEFFF78CFE0A2006F0CA
:10A42000CAFF70BD70B504460D4629462046FFF7A9
:10A43000DFFF012070BD000001460020174A914255
:10A4400003D2B1F1006F00D326E0154A914204D245
:10A45000124A914201D301201EE0124A914204D2D5
:10A460000F4A914201D3022016E00F4A914204D2D2
:10A470000C4A914201D303200EE00C4A914204D2CF
:10A48000094A914201D3042006E0094A914203D2CD
:10A49000064A914200D305207047000000400008A2
:10A4A0000080000800C00008000001080000020849
:10A4B000000004081FB51F481F4908604FF4803092
:10A4C000486000211C4881600121016181610021F7
:10A4D0000162C162194981620021C1600221C1612A
:10A4E000012101634161FAF781FE20B140F20511BB
:10A4F00013A006F07DF90120009001900720029042
:10A5000069460D48FAF7A8FD20B140F20F110CA0E2
:10A5100006F06EF91120009002200190694606486D
:10A52000FAF79AFD20B14FF48C7105A006F060F99E
:10A530001FBD000000200140C0E400200100000F0A
:10A540002E2E2F5372632F6D61696E2E63000000F3
:10A5500008B500BF002000902A48006840F4800041
:10A56000284908600846006800F48000009000BF99
:10A5700000BF00BF002000900846006840F40010B3
:10A5800008600846006800F40010009000BF00BF9B
:10A59000002211461020FBF7C0FC1020FBF7B0FC96
:10A5A000002211461120FBF7B8FC1120FBF7A8FC94
:10A5B000002211463820FBF7B0FC3820FBF7A0FC46
:10A5C000002211463920FBF7A8FC3920FBF798FC44
:10A5D000002211463A20FBF7A0FC3A20FBF790FC42
:10A5E000002211464520FBF798FC4520FBF788FC2C
:10A5F000002211464620FBF790FC4620FBF780FC2A
:10A6000008BD00003038024000B587B000BF002010
:10A6100001908748006840F00400854908600846BA
:10A62000006800F00400019000BF00BF00BF0020E0
:10A6300001900846006840F0800008600846006805
:10A6400000F08000019000BF00BF00BF002001901B
:10A650000846006840F0010008600846006800F005
:10A660000100019000BF00BF00BF0020019008461C
:10A67000006840F0020008600846006800F0020030
:10A68000019000BF00BF00BF002001900846006895
:10A6900040F0080008600846006800F008000190DB
:10A6A00000BF00BF012248F210116248FBF792FB85
:10A6B000012241F210016048FBF78CFB0022A5212A
:10A6C0005E48FBF787FB012246F248415B48FBF7F7
:10A6D00081FB00224FF480715748FBF77BFB00227F
:10A6E0004FF480515348FBF775FB00220421544876
:10A6F000FBF770FB4FF40050029000200390049091
:10A7000002A94D48FBF774FA012002904D480390CE
:10A710000020049002A94748FBF76AFA49F210109A
:10A7200002900120039000200490059002A9414866
:10A73000FBF75EFA41F21010029001200390002016
:10A740000490059002A93C48FBF752FA40F2ED4014
:10A7500002900120039000200490059002A9374840
:10A76000FBF746FA0220029036480390012004903D
:10A7700002A93248FBF73CFA4FF48050029031486E
:10A7800003900020049002A92C48FBF731FA4FF403
:10A79000C0400290112003900020049003200590F7
:10A7A00002A92648FBF724FA4FF4007002902548CE
:10A7B00003900020049002A91F48FBF719FA042017
:10A7C000029001200390002004900220059002A92D
:10A7D0001B48FBF70DFA4FF4047002900020039021
:10A7E000049002A91548FBF703FA00220121062074
:10A7F000FBF793FB0620FBF783FB002201210720D8
:10A80000FBF78BFB0720FBF77BFB002201211720C6
:10A81000FBF783FB1720FBF773FB00221146282070
:10A82000FBF77BFB2820FBF76BFB07B000BD0000AC
:10A83000303802400000024000080240000402409C
:10A84000000C02400000111010B5104810490860BB
:10A850004FF48270486000210D488160C160016141
:10A8600041614FF4007181610821C16100210162E1
:10A87000416281620A21C162FBF748FF20B14FF4B7
:10A88000987104A005F0B4FF10BD00000030014035
:10A8900068E500202E2E2F5372632F6D61696E2E96
:10A8A0006300000000B591B02848294908600920DC
:10A8B00048600021264881604FF43761C160002163
:10A8C00001614161FCF799FD20B140F2451121A0E1
:10A8D00005F08EFF00200F9010900FA91C48FCF788
:10A8E000B6FA20B14FF4A6711AA005F081FF6020DE
:10A8F00008904FF4B760099000200A900C900D90DA
:10A900000E900C2208A91248FCF7F3FC20B140F28B
:10A91000571110A005F06CFF0020019002900390E9
:10A92000049005904FF4005006900020079001A974
:10A930000748FCF74DFA20B140F2631105A005F07D
:10A9400057FF0348FCF7BAFC11B000BD00000140FE
:10A95000C0E500202E2E2F5372632F6D61696E2E7D
:10A960006300000000B587B01848194908604F20FF
:10A9700048600021164881604FF47A71C16000215F
:10A980000161FCF7B8FA20B14FF4BC7111A005F0D9
:10A990002FFF4FF48050039003A90D48FCF729FBCB
:10A9A00020B14FF4BF710BA005F022FF00200190F1
:10A9B000029001A90648FCF74AFA20B140F285113D
:10A9C00004A005F015FF07B000BD00000004004022
:10A9D000FCE500202E2E2F5372632F6D61696E2EC1
:10A9E0006300000010B50C480C4908604FF4E130DA
:10A9F0004860002109488160C16001610C2141610A
:10AA000000218161C161FCF7DDFE20B14FF4CC7102
:10AA100003A005F0EDFE10BD0010014038E6002057
:10AA20002E2E2F5372632F6D61696E2E630000000E
:10AA300010B50C480C4908604FF4164048600021DE
:10AA400009488160C16001610C214161002181617F
:10AA5000C161FCF7B7FE20B140F2AB1103A005F0D5
:10AA6000C7FE10BD0044004078E600202E2E2F5374
:10AA700072632F6D61696E2E6300000010B50C4883
:10AA80000C4908604FF4E1304860002109488160BA
:10AA9000C16001610C21416100218161C161FCF74C
:10AAA00091FE20B14FF4DF7103A005F0A1FE10BDAF
:10AAB00000140140B8E600202E2E2F5372632F6D34
:10AAC00061696E2E6300000000BFFEE7004870471A
:10AAD0001080002000487047F07F00200048704739
:10AAE000008000200048704725800020024604486E
:10AAF0000260044801600120034B18700020704779
:10AB000048040020440400204C0400200146034A6D
:10AB1000505C0022014B5A54704700005E04002034
:10AB20000146034A505C0022014B5A547047000012
:10AB30006104002070B504460D460648006830B137
:10AB40000548294602682046024B1B6898470020AA
:10AB500070BD000050040020540400200146012074
:10AB6000024A50540020024A505470475E040020AC
:10AB70006104002001460120024A50540020024A8C
:10AB800050547047610400205E04002010B5044654
:10AB900014B94FF0FF3010BD01200449087022465F
:10ABA00080210348FEF78DFF0020F4E764040020B5
:10ABB00025800020024908780021014A1170704761
:10ABC00064040020014600207047000070B505466F
:10ABD0000C46152C07D2224629460448F5F737FBC8
:10ABE000002002490855002070BD000010800020A0
:10ABF00070B505460C46022C02D24FF0FF3070BDF6
:10AC0000A41E102C07D2224629460448F5F71FFB44
:10AC10000020024908550020F1E70000F07F0020E5
:10AC200070B505460C46022C02D24FF0FF3070BDC5
:10AC3000A41E102C07D2224629460448F5F707FB2C
:10AC40000020024908550020F1E7000000800020A4
:10AC5000024603480260034801600020704700007C
:10AC60005004002054040020024908780021014AC1
:10AC7000117070474C04002010B504460648006867
:10AC800028B1064801682046034A126890470448E4
:10AC90000460002010BD000048040020440400208F
:10ACA000400400207047000008B50F48FEF754FC30
:10ACB00010B14FF0FF3008BD0C48FEF74DFC10B14D
:10ACC0004FF0FF30F7E70020094B42F210720121EC
:10ACD000009006480068FEF7CBFC0020054908609C
:10ACE000F6F76EFE0020E6E7340200203C0200206A
:10ACF000D91802083802002070B504460E462046D6
:10AD0000F5F7F1FA05462946204600F0D7F870BD60
:10AD1000F8B504460E4615461F46642C04D0652C33
:10AD200003D0C82C29D117E000BF16480068401C8A
:10AD3000144908600846006803280AD90020124B0D
:10AD400047F230520146009010480068FEF790FC30
:10AD500001E0F6F735FE11E000200A4908602A46B6
:10AD60003146022005F064FA10B109A0FDF78CFB12
:10AD700029460DA0FDF788FB00E000BF00BF0020C2
:10AD8000F8BD00003802002041E40208340200202F
:10AD900052544B20446174612053656E64204572A7
:10ADA000726F720D0A0000002575422052544B202C
:10ADB000446174612053656E740D0A002DE9F84FEB
:10ADC00004460F4615461E46DDE90B8ADDF828903D
:10ADD0004FF0000B1E48007818B14FF0FF30BDE86F
:10ADE000F88F24B1B8F1000F01D005B116B94FF0BA
:10ADF000FF30F4E7224640211648FEF762FE4A463D
:10AE000020211548FEF75DFE2B4614A2402115486F
:10AE10000096FEF756FE83468023134A5946114892
:10AE2000FDF736FA114807601148C0F80080114854
:10AE3000C0F800A0012001F0EDFB0C48008882B2B0
:10AE400004490D48006802F083FC0020C7E70000B9
:10AE50005C050020D4C3002054C4002025733A258B
:10AE60007300000014C40020B5C400207005002049
:10AE7000680500206C0500206005002010B500204A
:10AE80000A49087000230A4A01210A4802F086FC98
:10AE900010B14FF0FF3010BD0748FEF75DFB10B159
:10AEA0004FF0FF30F7E70020F5E700005C050020D9
:10AEB000D9D50208600500206405002070B504465D
:10AEC0000D4606480078052805D12A462146044843
:10AED000006802F089FE002070BD00005C050020C3
:10AEE0006005002002480068C0F30220704700009F
:10AEF0000CED00E010B5002807DA0A07140E054A29
:10AF000000F00F031B1FD45403E00A07130E024A7C
:10AF1000135410BD18ED00E000E400E038B5002542
:10AF20000020009000BF5E480068C0F580525D4878
:10AF30005B4B1B68C1186B465B48006802F098FDCC
:10AF400005460DB9009800B9A7E05548006800997A
:10AF500008445349086008460068B0F5805F03D391
:10AF600052A0FEF7C5FE98E059480078052808D1A0
:10AF70004B4801684B48FEF7E9FE0020484908604D
:10AF80008AE05348007803281BD152A14548009A13
:10AF9000FEF7F1FD504908600846006800287AD0A5
:10AFA0004E4B4FA23F480099FEF798FC032803D070
:10AFB0004EA0FEF79DFE70E000210846FEF7C6FE9B
:10AFC00069E043480078022865D15148007800289C
:10AFD00055D150A13348009AFEF7CDFD3E49086097
:10AFE00008460068002856D0002408460068001D66
:10AFF00008603A4B3AA22B480099FEF76FFC0328F1
:10B0000003D046A0FEF774FE47E04DA12548009A04
:10B01000FEF7B1FD04466CB3103400E0641C2078E8
:10B020002028FBD01F48201A009A111A494B4AA227
:10B030002046FEF753FC012803D049A0FEF758FE36
:10B040002BE0254800681749401A4249096808441E
:10B050004C49086001202E49087011480068494990
:10B06000096888420AD33B4801681B480068FEF71C
:10B070006DFE12E044A0FEF73BFE0EE00BE0084838
:10B08000006840490968884205D33248016812487F
:10B090000068FEF75BFE00BF45E700BF002038BD3B
:10B0A0007805002035C90020600500202E2E5C4662
:10B0B0004D4C5C496E7465726E65745C4E545249B9
:10B0C00050436C69656E742E633A33393500000065
:10B0D0005C0500200D0A0000880500208005002086
:10B0E000252A20256420252A0D0A00002E2E5C46E4
:10B0F0004D4C5C496E7465726E65745C4E54524979
:10B1000050436C69656E742E633A3431330000002D
:10B110005D0500200D0A0D0A000000002E2E5C4681
:10B120004D4C5C496E7465726E65745C4E54524948
:10B1300050436C69656E742E633A343334000000FA
:10B14000436F6E74656E742D4C656E6774683A203B
:10B15000000000008405002025640D0A00000000A6
:10B160002E2E5C464D4C5C496E7465726E65745C47
:10B170004E54524950436C69656E742E633A3435AF
:10B18000300000007C0500202E2E5C464D4C5C49B2
:10B190006E7465726E65745C4E54524950436C69AE
:10B1A000656E742E633A34363500000010B50446DF
:10B1B000F6F764FBFFF70AF803480088401C0249D1
:10B1C000088006F0EBFE10BD0A00002010B501203B
:10B1D0000549087000F09EF9012211030348FAF7AF
:10B1E000F9FD00F005F810BD160200200000024035
:10B1F00010B504F093FA0121044806F055FC002034
:10B2000006F098FC002006F01DFC10BD00D02324A1
:10B210007047000010B54FF480511048FAF7D2FD86
:10B22000D0B14FF47A7006F0BCF84FF480510B485F
:10B23000FAF7C8FD80B10EE04FF480510748FAF7E5
:10B24000C1FD40B9642006F0ACF800224FF48071D3
:10B250000348FAF7BFFDEFE710BD0000000402400D
:10B260000000024010B52DED028B4FF4007195489F
:10B27000FAF7A8FD002874D000209349088093496C
:10B2800008709348007850B99248007838B9F6F7BA
:10B2900055FB0320F6F7D0FC01208D49087073E0C0
:10B2A000FEF78AF98C490968401A41F270718842A8
:10B2B0002AD9FEF781F98849086083480088801DF3
:10B2C000814908804FF480617E48FAF77BFD40B1E8
:10B2D00000F026F9BCEEC00A10EE100A7F49087093
:10B2E00012E0012291027748FAF774FD00F018F994
:10B2F000BCEEC00A10EE100A7849087000224FF424
:10B3000080617048FAF766FD75480068F5F7E6F960
:10B3100041EC180B9FED730B53EC102BF5F70AFA69
:10B3200008D86A48007828B90120684908700020C8
:10B33000654908806A480068F5F7D0F941EC180BB8
:10B340009FED680B53EC102BF5F7F4F90AD85E4823
:10B350000088B0F5E16F05DB4FF408006349086031
:10B3600004E01BE04FF4084060490860642006F0E8
:10B3700018F8F6F77BFBFEF7B3FF5C480022114696
:10B380000368104601F030F94FF400714D48FAF7A8
:10B3900019FD18B1F6F72CFB032881D00020544981
:10B3A00008704B480078C8B10020F6F745FC002033
:10B3B00047490870FFF70AFF4FF400714148FAF758
:10B3C00001FD58B9642005F0ECFF00224FF48071B4
:10B3D0004848FAF7FFFC642005F0E3FF4FF40071E2
:10B3E0003848FAF7EFFC10B900203A490870FEF728
:10B3F000E3F84FF47A71B0FBF1F201FB12000A2876
:10B400001CD23D48007858BB344800780F2803DD33
:10B4100088203649086003E04FF40840334908604B
:10B4200001203549087031480368344802683448BF
:10B4300001683448006801F0D7F811E02E48007820
:10B4400070B100202C49087028490860084603683C
:10B450002A4802682A4801682A48006801F0C4F8AE
:10B46000FEF7AAF81C490968401A41F2883188425F
:10B4700025D9FEF7A1F8184908604FF480611148FA
:10B48000FAF7A0FC40B100F04BF8BCEEC00A10EE99
:10B49000100A1249087012E0012291020948FAF7D5
:10B4A00099FC00F03DF8BCEEC00A10EE100A0B4902
:10B4B000087000224FF480610248FAF78BFCBDEC63
:10B4C000028B10BD000402400C0000200E00002082
:10B4D0000F0000207E030020140000201E02002028
:10B4E000340600209A999999999910407006002085
:10B4F00010000020000002402F0000206C060020F9
:10B50000680600206406002010B50020FFF726FB27
:10B51000002010BD10B50020FFF72CFB002010BD4F
:10B5200010B52DED068B9FED3D0AB0EE408A9FEDE4
:10B530003B0AF0EE408A00F081F8B0EE408A9FEDC1
:10B54000380AB4EEC08AF1EE10FA04D29FED330A45
:10B55000F0EE408A19E0B1EE000AB4EEC08AF1EED6
:10B5600010FA04DD9FED2F0AF0EE408A0DE09FED0A
:10B570002C0A38EE400A9FED2C1AC0EE010A9FED0E
:10B58000290A20EE800AF0EE408A284890ED000A51
:10B59000B5EEC00AF1EE10FA06D2C0ED008AFEF751
:10B5A0000BF82349086033E0204890ED000A30EEA4
:10B5B000680A10EE101A0846F5F790F841EC1A0BDD
:10B5C000B0EE4A0AF0EE6A0A05F06AF9B0EE409A67
:10B5D000F0EE609A9FED170B53EC102B51EC190B0A
:10B5E000F5F790F804D2FDF7E7FF114908600FE086
:10B5F000FDF7E2FF0E490968401A4EF660218842C5
:10B6000006D90A48C0ED008AFDF7D6FF0849086050
:10B61000064890ED000ABDEC068B10BD000000004E
:10B62000333353400000C8423333333F38060020E1
:10B630003C060020000000000000E03F2DE9F04142
:10B640002DED0C8B0020F5F7E3FC85B20024284695
:10B65000F5F718F841EC1B0B9FED500B53EC102B3A
:10B66000F4F7A1FF41EC1A0B9FED4E0B53EC102B9E
:10B67000F4F727FF41EC190BF5F774F808EE100A00
:10B68000B0EE000A28EE000AB0EE408A2846F4F731
:10B69000F9FF41EC1B0B9FED410B53EC102BF4F722
:10B6A00082FF41EC1A0B9FED3F0B53EC102BF4F78C
:10B6B00008FF41EC190BF5F755F83C4908600846BE
:10B6C00090ED000AF0EE000A20EE200A80ED000A5C
:10B6D0000020F5F79DFC87B20120F5F799FC1FFAD1
:10B6E00080F8334806883846F4F7CCFF41EC1B0B52
:10B6F0003046F4F7C7FF41EC1D0B9FED2A0B53ECCE
:10B70000102BF4F7DEFE41EC1C0B53EC1B2BF4F773
:10B71000D8FE41EC1A0B9FED270B53EC102BF4F7DE
:10B72000D0FE41EC190BF5F71DF800EE100AC8EB3E
:10B73000083000EE900AF8EEE00A80EE201AF0EEF3
:10B74000418A18EE900AF4F7C9FF41EC190B9FEDFE
:10B75000150B53EC102BF4F7D5FF02D2012017493B
:10B7600008609FED170A38EEC00A9FED161AC0EE6A
:10B77000010A9FED150A20EE800ABDEEC00A10EE08
:10B78000104A642C00DD6424002C00DA0024B0EEA2
:10B79000480ABDEC0C8BBDE8F08100000000000001
:10B7A00000FEAF406666666666660A4034060020A4
:10B7B0002A7AFF1F00000000000000403006002031
:10B7C00033335340CDCC4C3F0000C84210B500216C
:10B7D0000248FFF73DFA002010BD0000E1B7020863
:10B7E000014B1A60704700007C0100201CB506F078
:10B7F000CFFC4FF48070BC4948800120BB490870E1
:10B80000B94890F84400BA49087001200870084609
:10B81000007848B94FF47A70B349C8800120C887CE
:10B820000A20488700208887AF48C088322802DA7B
:10B830006420AD49C880AC48C088B0F57A7F03DD8C
:10B840004FF47A70A849C880A748008F0A2802DD03
:10B850000220A5490887A448C08E432802DD432062
:10B86000A149C886A048C08E002802DA00209E495F
:10B87000C8869D48808A4FF6FF71884202D10A200F
:10B88000994988829848808C42F21071884202DD82
:10B89000002095498884944890F8360095490870AE
:10B8A000914890F83E00944908708F4890F83C0009
:10B8B000924908708C48807A914908708A4880883B
:10B8C000904908600520904908808748C088098809
:10B8D00090FBF1F08D49088083488088098890FBAF
:10B8E000F1F201FB12008849098848438849088021
:10B8F00008460088874908807B48C0884FF47A71E1
:10B9000091FBF0F08449088008460088C82191FB2B
:10B91000F0F0824908800020814908805520814943
:10B920000870AA2048707048408C000B4FF47A7160
:10B9300010FB01F16C48408CC0F3032000EBC00207
:10B9400002EB001001EB8000674991F82210C1F36F
:10B95000031101EB810100EB4100634991F82210D2
:10B9600001F00F010844704908805F48808C000B8B
:10B970004FF47A7110FB01F05B49898CC1F303210C
:10B9800001EBC10202EB011100EB8100564991F875
:10B990002410C1F3031101EB810100EB4100524976
:10B9A00091F8241001F00F010844604908804E48C6
:10B9B000C08C000B4FF47A7110FB01F14A48C08C27
:10B9C000C0F3032000EBC00202EB001001EB80008B
:10B9D000454991F82610C1F3031101EB810100EBF9
:10B9E0004100414991F8261001F00F0108445049E7
:10B9F00008803D48008D000B4FF47A7110FB01F078
:10BA00003949098DC1F3032101EBC10202EB011198
:10BA100000EB8100344991F82810C1F3031101EBC8
:10BA2000810100EB4100304991F8281001F00F012D
:10BA30000844404908802C48008B3F490880314821
:10BA400001683EA004F0D6FE2748827840880112A3
:10BA50003EA004F0CFFE3848008836490988CDE979
:10BA6000001033480388314802882F48018840A0DD
:10BA700004F0C0FE1C48B0F8560001280DD11A4849
:10BA8000008B1949098DCDE900101748C38C828CB1
:10BA9000418C3FA004F0AEFE25E01348B0F85600FC
:10BAA000022819D1454946A004F0A4FE0E48B0F87A
:10BAB000A01247A004F09EFE4049223148A004F0A5
:10BAC00099FE3E4942314BA004F094FE3B4962315D
:10BAD0004DA004F08FFE06E00348B0F8560010B900
:10BAE0004FA004F087FE1CBD982400202D000020EC
:10BAF0000C02002075060020F4010020F501002052
:10BB0000D7010020CC010020E0010020E20100204C
:10BB1000DC010020EC010020EA01002000020020EE
:10BB20000E02002064160020AC010020AE010020AF
:10BB3000B0010020B2010020B4010020C9E8B1B872
:10BB400049443A202578202E0D0A0000B9CCBCFECD
:10BB5000B0E6B1BE3A205552542D4D4BB0B2B0EEC6
:10BB6000B3B5D4D8205625642E25642E200D0A00A6
:10BB7000B7FECEF1C6F7B5D8D6B73A2025642E2544
:10BB8000642E25642E25643A25642E0D0A000000DB
:10BB90005443505F5254434DC4A3CABD2CB7FECE8C
:10BBA000F1C6F7B5D8D6B73A2025642E25642E25E0
:10BBB000642E25643A25642E0D0A00001827002003
:10BBC0004E74726970486F73743A25732E0D0A00B3
:10BBD0004E74726970506F72743A25642E0D0A00AB
:10BBE0004E74726970557365726E616D653A257336
:10BBF0002E0D0A004E7472697050617373776F7204
:10BC0000643A25732E0D0A004E74726970536F7575
:10BC10007263656E616D653A25732E0D0A00000032
:10BC2000B5A5B5E3B6A8CEBBC4A3CABDC4A3CABD5F
:10BC30002E200D0A0000000030B503460224144DEA
:10BC40002C70002007E0134C34F810409C4200D1C7
:10BC500005E0441CE0B2104C2478A042F3DB00BFA6
:10BC60000D4C2478A04209D10B4C2478B4F5957F73
:10BC700004DC094C2478641C074D2C70054C24F816
:10BC80001030064C24F81010054C225430BD000032
:10BC90001A020020343E00201B0200208C400020AD
:10BCA000E442002000B54FF40000034908604FF45F
:10BCB000FA7006F0CBFB00BD1804024030B5044614
:10BCC000002517230AE024FA03F000F0010515B15E
:10BCD00000F01AF801E000F005F85B1E002BF2DA24
:10BCE00030BD000000B5802006490860022006F043
:10BCF000ADFB4FF40000034908600A2006F0A6FBE4
:10BD000000BD00001804024000B58020064908600C
:10BD10000B2006F09BFB4FF4000003490860022053
:10BD200006F094FB00BD00001804024038B504463C
:10BD30001CB9002000F010F808E00020044B224657
:10BD40000146009003480068FDF792FC38BD0000F2
:10BD500059BD02082C06002072B60649064A116039
:10BD600000BF00BF00BFBFF34F8F00BF00BF00BFC9
:10BD7000704700000400FA050CED00E000B585B046
:10BD800014216846F4F77CFA642005F00AFB0022CF
:10BD90004FF400411148FAF71DF84FF400400090AD
:10BDA0000120019000200290039069460B48F9F7AA
:10BDB0001FFF642005F0F5FA4FF4004000900320C7
:10BDC000019000200290039069460448F9F710FFA3
:10BDD000022005F0E6FA05B000BD000000040240B4
:10BDE00010B50446204600F0CCFA00B118E0204619
:10BDF00000F034F80022C721204600F039FA00B1E3
:10BE000011E0204600F016F8204600F0A9FA00B133
:10BE100006E0204600F03CFA00B101E0002010BD31
:10BE20004FF0FF30FBE7204600F004F84FF0FF3002
:10BE3000F5E7000010B5044604EB8402064B03EB63
:10BE4000C202118904EB840203EBC2025068012292
:10BE5000F9F7C0FF10BD0000C87F002010B50446F0
:10BE600004EB8402064B03EBC202118904EB84024B
:10BE700003EBC20250680022F9F7ACFF10BD0000CE
:10BE8000C87F00202DE9F04107460C4615461E46A6
:10BE90004FF0000807EB87001C4901EBC000406A27
:10BEA000A04211D985B1601907EB8701174A02EB4F
:10BEB000C101496A884207D8154850F82600401E3B
:10BEC000204008B9032E03DB4FF0FF30BDE8F081BE
:10BED00064B907EB87000D4901EBC000406AA84236
:10BEE00004D83846FFF77CFF0020EFE709E004EBB9
:10BEF00008013246384600F06FF9054850F8260030
:10BF00008044A845F3D30020E0E70000C87F00206C
:10BF1000E825030838B5044603226946204600F0A8
:10BF200011F910B14FF0FF3038BD9DF80000FF2827
:10BF300010D19DF80100FF280CD19DF80200FF28C8
:10BF400008D103226946204600F0FCF810B14FF0FA
:10BF5000FF30E9E79DF80200152806D016280DD01D
:10BF6000172814D0182824D11AE04FF4800004EBCD
:10BF70008401164A02EBC101486223E04FF48000BD
:10BF800004EB8401114A02EBC10148621AE04FF44C
:10BF9000000004EB84010D4A02EBC101486211E08C
:10BFA0004FF0807004EB8401084A02EBC101486243
:10BFB00008E04FF4800004EB8401044A02EBC10165
:10BFC000486200BF00BF0020AEE70000C87F00202D
:10BFD0002DE9F04782460C4690461D46DDF820903C
:10BFE00000260027E0B2C0F58077AF4200D92F4687
:10BFF000504600F04DF900B147E0504600F0C1F95D
:10C0000000B142E05046FFF729FF002202215046CE
:10C0100000F02EF900B13BE00022C4F30741504686
:10C0200000F026F900B133E00022C4F307215046A6
:10C0300000F01EF900B12BE0E1B20022504600F002
:10C0400017F900B124E0002608E018F806100022D5
:10C05000504600F00DF900B11AE0761CBE42F4D350
:10C060005046FFF7E7FE504600F07AF900B10CE0C9
:10C07000504600F00DF900B107E0B9F1000F01D012
:10C08000C9F800700020BDE8F0874FF0FF30FAE7F4
:10C090005046FFF7CFFE4FF0FF30F4E730B500EB2E
:10C0A0008004074D05EBC404241D44F8312000EB47
:10C0B000800405EBC404241D04EBC104A38030BD3F
:10C0C000C87F00202DE9F04180460E4614461F46E9
:10C0D00000254046FFF7C2FE00220321404600F043
:10C0E000C7F800B128E00022C4F30741404600F041
:10C0F000BFF800B120E00022C4F30721404600F061
:10C10000B7F800B118E0E1B20022404600F0B0F804
:10C1100000B111E0002507E07219FF21404600F050
:10C12000A7F800B108E06D1CBD42F5D34046FFF70B
:10C1300081FE0020BDE8F0814046FFF77BFE4FF016
:10C14000FF30F7E72DE9F04107460D46164600247B
:10C150003846FFF783FE00229F21384600F088F81A
:10C1600000B111E0002407E02A19FF21384600F051
:10C170007FF800B108E0641CB442F5D33846FFF7FD
:10C1800059FE0020BDE8F0813846FFF753FE4FF01E
:10C19000FF30F7E770B506460C4600253046FFF73E
:10C1A0005DFE00220521304600F062F805462DB9FB
:10C1B0002246FF21304600F05BF805463046FFF787
:10C1C00039FE284670BD000000EB8002014B03F8E9
:10C1D00032107047C87F002070B506460C461546E1
:10C1E000214850F82500401E8443304600F0C9F82D
:10C1F00000B130E03046FFF731FE1C48415D0022BF
:10C20000304600F035F800B128E00022C4F30741C1
:10C21000304600F02DF800B120E00022C4F30721E1
:10C22000304600F025F800B118E0E1B200223046B7
:10C2300000F01EF800B111E03046FFF7FBFD30467C
:10C2400000F08EF800B106E0304600F021F800B1B1
:10C2500001E0002070BD4FF0FF30FBE73046FFF7F4
:10C26000E9FD4FF0FF30F5E7E8250308F425030862
:10C2700037B50446154604EB8401044A12F8310030
:10C28000012301AA294600F0A1F83EBDC87F002085
:10C2900038B5054600240020009000BF69462846B6
:10C2A000FFF778FF044604B105E09DF8000000F0B8
:10C2B00001000028F2D100BF204638BD2DE9FC4125
:10C2C00004460D4617461E464FF000080020019018
:10C2D00004EB8400214901EBC000406AA84201D967
:10C2E00007B11EB94FF0FF30BDE8FC8104EB8400BC
:10C2F0001A4901EBC000416A04EB8400174A02EBC3
:10C30000C000406A401E2840081AB0420DD204EB1B
:10C310008400114601EBC000416A04EB840002EB8B
:10C32000C000406A401E28400E1A13E001A83346A0
:10C330003A46294600902046FFF74AFE10B14FF0DA
:10C34000FF30D1E701980544019807440198361A57
:10C3500001988044002EE9D10020C5E7C87F002065
:10C3600070B5044600252046FFF778FD0022042121
:10C370002046FFF77DFF05462046FFF75BFD284678
:10C3800070BD70B5044600252046FFF767FD00220A
:10C3900006212046FFF76CFF05462046FFF74AFDC1
:10C3A000284670BDF8B504460D4616462B460022B9
:10C3B00080212046009600F02DF828B1606D40F0F5
:10C3C000200060650320F8BD0020FCE7F8B50646B4
:10C3D0000D4617461C462DB922463946304600F018
:10C3E0006FF8F8BD642104FB01F0A3B2044900908A
:10C3F00051F826002A463946FAF79DFB0020F0E75F
:10C40000240600200246024840F82210002070470F
:10C41000240600202DE9F04104460E4617461D462D
:10C42000DDF818803FE0681CE0B32DB1F9F7D8FCC7
:10C43000A0EB0800A84236D32068406820F0E00056
:10C44000216848606068B0F5827F0DD1A068B0F5C2
:10C45000004F03D0A068B0F5806F05D12068006858
:10C4600020F0400021680860A06AB0F5005F0ED19E
:10C4700000BF206800684DF6FF7108402168086021
:10C480002068006840F400502168086000BF012067
:10C4900084F8510000BF002084F8500000BF032042
:10C4A000BDE8F081FFE7206880683040B04201D1EC
:10C4B000012000E00020B842B5D10020F0E70000E4
:10C4C00070B505460E461446642104FB01F3A2B282
:10C4D000034951F825003146FAF75AFA002070BD99
:10C4E000240600207047000038B504460D460020A1
:10C4F000009055201B490870AA20487003208870BE
:10C50000601DC87003200871084645718471164883
:10C5100000EB450122461348C01DF3F798FE0020AA
:10C5200008E0811C0F4A515CBDF80020114489B21B
:10C530000091401C611D8842F3DB0A48801CF5F71E
:10C54000D5F90090E01D07490844BDF800100180AE
:10C550004FF47A7304F1090202490448FBF7E3FB44
:10C5600038BD00001C2900209824002038E6002057
:10C5700008B50948094B0A4A4FF480610090094800
:10C58000FDF79FFA0849086008460649026807480F
:10C59000006801F029FB08BDB5C4002074C4002068
:10C5A0007037030835C500207405002060050020A1
:10C5B00010B5084B084A4FF480610848FDF781FA2E
:10C5C000074908600846054902680648006801F006
:10C5D0000BFB10BDB5C40020F436030835C50020A0
:10C5E0007405002060050020F0B507460C4615468E
:10C5F0001E4672B6FFF756FB3846FFF75FFB204634
:10C60000FFF75CFB2846FFF759FB3046FFF756FB68
:10C6100062B6F0BD10B50446062C0BDA064850F899
:10C620002420064B1B7850F8231005A0FBF72CFFA5
:10C6300002480470002010BD8C0500205C0500201D
:10C64000436C69656E7453746174652066726F6DB6
:10C65000205B25735D206368616E676520746F20C1
:10C660005B25735D0D0A000070B504460D46022C73
:10C670000FD0FCF70FFF50B1FCF70CFFD0F890057E
:10C6800028B1FCF707FFD0F8906504A0B047002060
:10C6900070BD6868FEF77AFA0020F9E74552524FFC
:10C6A000520D0A0070B505460E460220FEF756FAF6
:10C6B000FCF7F0FE50B1FCF7EDFED0F8900528B184
:10C6C000FCF7E8FED0F8904501A0A047002070BD1F
:10C6D0004F4B0D0A000000002DE9F04105460E46C3
:10C6E000022D0DD0FCF7D6FE50B1FCF7D3FED0F8EA
:10C6F000900528B1FCF7CEFED0F8907529A0B84778
:10C700007068F3F72AFE04469CB90020F5F794FA06
:10C71000FCF7C0FE002842D0FCF7BCFED0F8900524
:10C7200000283CD0FCF7B6FED0F8907520A0B847A2
:10C7300035E0012C11D1FCF7ADFE50B1FCF7AAFE9B
:10C74000D0F8900528B1FCF7A5FED0F8907518A098
:10C75000B8470120F5F770FA21E0022C11D1FCF75F
:10C7600099FE50B1FCF796FED0F8900528B1FCF781
:10C7700091FED0F890750EA0B8470220F5F75CFA4C
:10C780000DE0FCF787FE50B1FCF784FED0F8900571
:10C7900028B1FCF77FFED0F8907503A0B8470020C1
:10C7A000BDE8F081417267204552524F520D0A0098
:10C7B0004F4B0D0A000000002DE9F04180460D4668
:10C7C0006868F3F7CAFD04464FF47A70B4FBF0F0E2
:10C7D00001036420B4FBF0F00A22B0FBF2F302FB89
:10C7E000130001EB0021B4FBF2F0B0FBF2F302FB0B
:10C7F000130001EB00101146B4FBF1F201FB1241F2
:10C8000046180C498E80084680880B49086005F060
:10C810007DFDFCF73FFE50B1FCF73CFED0F89005E3
:10C8200028B1FCF737FED0F8907504A0B847002077
:10C83000BDE8F08198240020CC0100204F4B0D0A68
:10C840000000000070B504460E46022C10DAFCF71A
:10C8500021FE50B1FCF71EFED0F8900528B1FCF780
:10C8600019FED0F8905503A0A8474FF0FF3070BDD7
:10C870000020FCE764656275675F6F666620666C22
:10C8800061670D0A0000000070B504460E46022CD8
:10C8900010DAFCF7FFFD50B1FCF7FCFDD0F8900575
:10C8A00028B1FCF7F7FDD0F8905503A0A8474FF04A
:10C8B000FF3070BD0020FCE764656275675F6F6ED6
:10C8C00020666C61670D0A002DE9F04105460E46B1
:10C8D000022D0DD0FCF7DEFD50B1FCF7DBFDD0F8EA
:10C8E000900528B1FCF7D6FDD0F8907511A0B84797
:10C8F0007068F3F732FD0446C4F30F201049A1F825
:10C900005200A1F8544005F001FD2146022003F039
:10C91000F9FAFCF7BFFD50B1FCF7BCFDD0F890056B
:10C9200028B1FCF7B7FDD0F8907506A0B8470020F5
:10C93000BDE8F081417267204552524F520D0A0006
:10C94000982400204F4B0D0A000000002DE9F04113
:10C9500006460F46FCF79EFD58B1FCF79BFDD0F84C
:10C96000900530B1FCF796FD1EA1D0F8904520A0AF
:10C97000A047FCF78FFD70B1FCF78CFDD0F8900557
:10C9800048B1FEF7A7F80546FCF784FD2946D0F824
:10C9900090451DA0A047FCF77DFD70B1FCF77AFD26
:10C9A000D0F8900548B1FEF791F80546FCF772FD06
:10C9B0002946D0F890451AA0A047FCF76BFD70B14E
:10C9C000FCF768FDD0F8900548B1FEF787F80546FA
:10C9D000FCF760FD2946D0F8904517A0A04700203D
:10C9E000BDE8F081563230323130353130303000F0
:10C9F00056657273696F6E3A202020202020202017
:10CA00002025730D0A000000494D45493A20202099
:10CA100020202020202020202025730D0A00000047
:10CA2000434349443A202020202020202020202059
:10CA30002025730D0A000000494D53493A2020205B
:10CA400020202020202020202025730D0A00000017
:10CA500010B522210248FCF797FC002010BD000011
:10CA6000B424030870B504460E46022C10D0FCF71F
:10CA700011FD50B1FCF70EFDD0F8900528B1FCF780
:10CA800009FDD0F890550AA0A8474FF0FF3070BDBF
:10CA9000FCF700FD50B1FCF7FDFCD0F8900528B183
:10CAA000FCF7F8FCD0F8905506A0A8470020EEE768
:10CAB00075736167653A206C6F6720737472696E75
:10CAC000670D0A004F4B0D0A0000000070B50546C7
:10CAD0000E46FCF7DFFC50B1FCF7DCFCD0F890050B
:10CAE00028B1FCF7D7FCD0F8904502A0A047002061
:10CAF00070BD00004F4B0D0A000000002DE9F04111
:10CB000004460F460026032C11D0FCF7C3FC50B19D
:10CB1000FCF7C0FCD0F8900528B1FCF7BBFCD0F8BE
:10CB2000905504A0A8474FF0FF30BDE8F0810020E9
:10CB3000FBE7000075736167653A206C6F675F7093
:10CB400072696E74206173635B302D315D20636E9A
:10CB5000740D0A000246002070470000F8B5054633
:10CB60000C46022D10D0FCF795FC50B1FCF792FC5E
:10CB7000D0F8900528B1FCF78DFCD0F890651AA08C
:10CB8000B0474FF0FF30F8BD4CF6CC4000901BA0F2
:10CB9000FBF77AFC002302224FF488311846FFF796
:10CBA00071F902236A464FF488310020FFF786FBB3
:10CBB00000234FF480724FF490311846FFF762F96A
:10CBC0006068F3F790FB461C33464FF49031002029
:10CBD0006268FFF773FB0A2004F0E3FB0020FFF715
:10CBE000A5F80020CFE7000075736167653A206FF4
:10CBF00074612075726C0D0A00000000676F746F1D
:10CC0000206F7461206170706C69636174696F6E0C
:10CC10000D0A000070B505460E460220FDF7AAFF7A
:10CC2000FCF738FC50B1FCF735FCD0F8900528B182
:10CC3000FCF730FCD0F8904501A0A047002070BD63
:10CC40004F4B0D0A0000000070B505460E4600204F
:10CC5000FDF784FFFCF71EFC50B1FCF71BFCD0F87D
:10CC6000900528B1FCF716FCD0F8904501A0A0472C
:10CC7000002070BD4F4B0D0A0000000070B5054646
:10CC80000E460020FDF776FFFCF704FC50B1FCF7E0
:10CC900001FCD0F8900528B1FCF7FCFBD0F89045DA
:10CCA00001A0A047002070BD4F4B0D0A00000000FE
:10CCB00070B504460E46022C10D0FCF7EBFB50B1C9
:10CCC000FCF7E8FBD0F8900528B1FCF7E3FBD0F8BF
:10CCD00090550AA0A8474FF0FF3070BDFCF7DAFB73
:10CCE00050B1FCF7D7FBD0F8900528B1FCF7D2FB88
:10CCF000D0F8905508A0A8470020EEE7757361674B
:10CD0000653A207274635F7365745F616C61726D04
:10CD1000207365630D0A00004F4B0D0A00000000F0
:10CD2000024600207047000070B504460E46072CEE
:10CD300010D0FCF7AFFB50B1FCF7ACFBD0F890057E
:10CD400028B1FCF7A7FBD0F8905503A0A8474FF0F7
:10CD5000FF3070BD0020FCE775736167653A207293
:10CD600074635F7365742079797979206D6D2064BF
:10CD700064206868206D6D2073730D0A0000000048
:10CD800070B504460D460020FEF7D0FF002070BDB0
:10CD90002DE9F04107460E46032F0DD0FCF77AFB34
:10CDA00050B1FCF777FBD0F8900528B1FCF772FB87
:10CDB000D0F890851FA0C0477068F3F7CEFA0446FC
:10CDC000B068F3F7CAFA0546142C22DC002C20DDEB
:10CDD000322D1EDC002C1CDD1949A1F870404FF4E7
:10CDE0007A7090FBF5F0C88005F090FAFCF752FBE2
:10CDF00050B1FCF74FFBD0F8900528B1FCF74AFB87
:10CE0000D0F890850FA0C04701200D49A1F860001F
:10CE10000DE0FCF73FFB50B1FCF73CFBD0F8900570
:10CE200028B1FCF737FBD0F8908502A0C04700205E
:10CE3000BDE8F081417267204552524F520D0A0001
:10CE4000982400204F4B0D0A0000000070B50546E5
:10CE50000C46062D10DAFCF71DFB50B1FCF71AFB4F
:10CE6000D0F8900528B1FCF715FBD0F890651EA00E
:10CE7000B0474FF0FF3070BD1DA220211D486368F0
:10CE800003F0C8FCA068FCF754FE1B49A1F8A002FF
:10CE900017A2202117482230E36803F0BBFC14A23C
:10CEA000202114484230236903F0B4FC10A2202151
:10CEB00010486230636903F0ADFC05F027FAFCF717
:10CEC000E9FA50B1FCF7E6FAD0F8900528B1FCF782
:10CED000E1FAD0F8906509A0B04701200649A1F811
:10CEE00060000020C7E700004552524F520D0A0073
:10CEF0002573000018270020982400204F4B0D0AAE
:10CF00000000000070B505460C46052D10DAFCF750
:10CF1000C1FA50B1FCF7BEFAD0F8900528B1FCF781
:10CF2000B9FAD0F890651BA0B0474FF0FF3070BD44
:10CF30001AA220211A48636803F06CFC17A2202172
:10CF400017482030A36803F065FC14A22021144880
:10CF50004030E36803F05EFC10A2202110486030EE
:10CF6000236903F057FC05F0D1F9FCF793FA50B1AF
:10CF7000FCF790FAD0F8900528B1FCF78BFAD0F8BE
:10CF8000906508A0B04701200849A1F86000002082
:10CF9000CDE700004552524F520D0A0025730000A4
:10CFA000982600204F4B0D0A000000009824002016
:10CFB000F8B505460C46022D10DAFCF76BFA50B1B5
:10CFC000FCF768FAD0F8900528B1FCF763FAD0F8BE
:10CFD000906516A0B0474FF0FF30F8BD6946606815
:10CFE000FCF732FC6068FCF7A4FD1249B1F856105A
:10CFF000884205D06068FCF79CFD0E49A1F85600F8
:10D0000005F084F9FCF746FA50B1FCF743FAD0F882
:10D01000900528B1FCF73EFAD0F8906506A0B0471D
:10D0200001200449A1F860000020D6E74552524F84
:10D03000520D0A00982400204F4B0D0A00000000FA
:10D04000F8B505460C46032D10DAFCF723FA50B16B
:10D05000FCF720FAD0F8900528B1FCF71BFAD0F8BD
:10D06000906528A0B0474FF0FF30F8BD6946606872
:10D07000FCF7EAFB9DF800002449498C884211D155
:10D080009DF801002149898C88420BD19DF802004E
:10D090001E49C98C884205D19DF803001B49098DA2
:10D0A00088420CD09DF80000184948849DF8010082
:10D0B00088849DF80200C8849DF803000885A06854
:10D0C000FCF737FD1149098B884204D0A068FCF7B2
:10D0D00030FD0E49088305F019F9FCF7DBF950B172
:10D0E000FCF7D8F9D0F8900528B1FCF7D3F9D0F8BF
:10D0F000906507A0B04701200449A1F86000002016
:10D10000B3E700004552524F520D0A009824002008
:10D110004F4B0D0A00000000F8B505460C46032DE4
:10D1200010DAFCF7B7F950B1FCF7B4F9D0F8900574
:10D1300028B1FCF7AFF9D0F890652DA0B0474FF0BB
:10D14000FF30F8BD69466068FCF77EFB9DF8000083
:10D150002949B1F86610884214D19DF8010026498A
:10D16000B1F8681088420DD19DF802002249B1F84B
:10D170006A10884206D19DF803001F49B1F86C106F
:10D18000884210D09DF800001B49A1F866009DF868
:10D190000100A1F868009DF80200A1F86A009DF85E
:10D1A0000300A1F86C00A068FCF7C3FC1249B1F8B9
:10D1B0006E10884205D0A068FCF7BBFC0E49A1F8B0
:10D1C0006E0005F0A3F801200B49A1F86000FCF700
:10D1D00061F950B1FCF75EF9D0F8900528B1FCF781
:10D1E00059F9D0F8906505A0B0470020A9E70000E4
:10D1F0004552524F520D0A00982400204F4B0D0A01
:10D2000000000000F8B505460C46022D10DAFCF7C8
:10D2100041F950B1FCF73EF9D0F8900528B1FCF780
:10D2200039F9D0F8906516A0B0474FF0FF30F8BD3F
:10D2300069466068FCF708FB6068FCF77AFC1249F5
:10D24000B1F85810884205D06068FCF772FC0E49AE
:10D25000A1F8580005F05AF8FCF71CF950B1FCF79A
:10D2600019F9D0F8900528B1FCF714F9D0F89065B9
:10D2700006A0B04701200449A1F860000020D6E7CD
:10D280004552524F520D0A00982400204F4B0D0A70
:10D2900000000000024600207047000070B50546FF
:10D2A0000C461646214602A0FBF7EEF870BD0000C2
:10D2B0004576656E743A25750D0A00002DE9F0413A
:10D2C00004460D46022C0DD0FCF7E4F850B1FCF7F3
:10D2D000E1F8D0F8900528B1FCF7DCF8D0F89065BB
:10D2E00014A0B0476868F3F738F80746384600F0EE
:10D2F000E7F970B9FCF7CEF8C8B1FCF7CBF8D0F875
:10D300009005A0B1FCF7C6F8D0F890650CA0B04726
:10D310000DE0FCF7BFF850B1FCF7BCF8D0F8900571
:10D3200028B1FCF7B7F8D0F8906503A0B04700200B
:10D33000BDE8F081417267204552524F520D0A00FC
:10D340004F4B0D0A000000002DE9F04705460C4642
:10D35000042D0DD0FCF79EF850B1FCF79BF8D0F8E7
:10D36000900528B1FCF796F8D0F8908518A0C04732
:10D370006068F2F7F2FF8146A668E068F2F7EDFF19
:10D3800087B23A463146484600F0E2F970B9FCF7F8
:10D3900081F8C8B1FCF77EF8D0F89005A0B1FCF791
:10D3A00079F8D0F890850DA0C0470DE0FCF772F831
:10D3B00050B1FCF76FF8D0F8900528B1FCF76AF887
:10D3C000D0F8908503A0C0470020BDE8F08700009A
:10D3D000417267204552524F520D0A004F4B0D0AC1
:10D3E00000000000F8B505460E460020009000231E
:10D3F000194A0121684600F0D1F9E8B9FCF74AF86A
:10D4000058B1FCF747F8D0F8900530B1FCF742F876
:10D41000D0F8904511A00099A047FCF73BF8C8B19F
:10D42000FCF738F8D0F89005A0B1FCF733F8D0F845
:10D4300090450DA0A0470DE0FCF72CF850B1FCF78B
:10D4400029F8D0F8900528B1FCF724F8D0F89045D9
:10D4500007A0A0470020F8BD9DD20208536F636B60
:10D4600049443A25750D0A004F4B0D0A0000000093
:10D470004552524F520D0A002DE9F04106460C4626
:10D48000032E0DD0FCF706F850B1FCF703F8D0F8E6
:10D49000900528B1FBF7FEFFD0F8907518A0B847AB
:10D4A0006068F2F75AFF8046A5682846F2F71BFF2E
:10D4B00007463A462946404600F096FB70B9FBF70E
:10D4C000E9FFC8B1FBF7E6FFD0F89005A0B1FBF784
:10D4D000E1FFD0F890750DA0B8470DE0FBF7DAFF3B
:10D4E00050B1FBF7D7FFD0F8900528B1FBF7D2FF7A
:10D4F000D0F8907503A0B8470020BDE8F081000087
:10D50000417267204552524F520D0A004F4B0D0A8F
:10D510000000000070B504460D46042102A000F092
:10D5200029FF002070BD0000B2E2CAD40000000054
:10D53000F8B505460E464AF6AA200090FBF7AAFF6A
:10D5400050B1FBF7A7FFD0F8900528B1FBF7A2FF79
:10D55000D0F890450AA0A047002302224FF488315A
:10D560001846FEF78FFC02236A464FF488310020EC
:10D57000FEF7A4FE01200549A1F860000020F8BDD7
:10D58000757064617465204F4B0D0A00982400206B
:10D5900070B5B2B004460E46214608A0FAF774FFF3
:10D5A000234606A2C8216846FCF78BFAC5B2294675
:10D5B000684602F021F832B070BD00003447207395
:10D5C00069676E616C20696E74656E736974792029
:10D5D00069732025750D0A00F8B505460C461646F8
:10D5E00034B1012C15D0022C44D0032C5AD156E072
:10D5F0002E480078012803D02C480078042807D151
:10D600000020FFF707F8002211466420F4F77EF9A6
:10D6100049E000202649086024480078012812D1FA
:10D62000FEF7C6FF0020234908700220FEF7F2FF34
:10D630000020214B47F23052014600901F480068FD
:10D64000FCF716F815E019480078042811D1FEF708
:10D650008FFF0020174908700320FEF7DBFF002032
:10D66000154B47F230520146009014480068FBF712
:10D67000FFFF18E00D480078042800D113E00F48A0
:10D680000068FBF753FF0948007838B10020FEF727
:10D69000C1FF002211466520F4F738F903E0FDF7D9
:10D6A0003DFC00E000BF00BFF8BD00005C050020AD
:10D6B000780500205D05002075E40208640500205F
:10D6C0000246C2EB8210C0EB00100A4B03EB800154
:10D6D000002A02DB032A00DA11B94FF0FF3070474D
:10D6E000087820B10878012801D0052008700020B2
:10D6F000F5E70000A880002070B50025002400BFD9
:10D700001FE0C5EB8510C0EB0010104901EB800451
:10D710002078032804D0042803D006280ED101E085
:10D7200000BF00BF0020A07001202070A06820B1C1
:10D7300002212846D4E90232984700E000BF00BF2A
:10D740006D1C032DDDDB002070BD0000A8800020D3
:10D750002DE9F04104460E461746C4EB8410C0EB99
:10D7600000100C4901EB8005002C02DB032C00DAD1
:10D770001DB94FF0FF30BDE8F081334606A22A21E3
:10D7800005F11000FCF79DF96F8703202870002039
:10D79000F1E70000A8800020257300002DE9F04784
:10D7A00007460E46904699460025002400BF38E003
:10D7B000C5EB8510C0EB00101C4901EB800474B36D
:10D7C000207860BB40F6C4612046FBF7FDFF656032
:10D7D000667002202070C4F80880C4F80C901023F2
:10D7E0004FF4C06204F1C40104F13C00FCF756FAA6
:10D7F000012E08D10123DA0204F2C46104F1B00061
:10D80000FAF7D7FC07E01023DA0104F2C46104F14F
:10D810006C00FCF743FA3D600020BDE8F087FFE7AD
:10D820006D1C032DC4DB4FF0FF30F6E7A88000200D
:10D830000146032908DAC1EB8110C0EB0010034A4E
:10D8400002EB80001030704701A0FCE7A8800020A8
:10D85000000000000146032908DAC1EB8110C0EB8B
:10D860000010034A02EB8000408F70470020FCE765
:10D87000A88000200146032908DAC1EB8110C0EB23
:10D880000010034A02EB80003C3070470020FCE7A8
:10D89000A88000200146032907DAC1EB8110C0EB04
:10D8A0000010034A12F8200070470020FCE7000037
:10D8B000A88000200146032908DAC1EB8110C0EBE3
:10D8C0000010034A02EB8000407870470020FCE71C
:10D8D000A88000200146032908DAC1EB8110C0EBC3
:10D8E0000010034A02EB8000807870470020FCE7BC
:10D8F000A8800020014603290ADA0120C1EB811229
:10D90000C2EB0212044B03EB8202907000207047BE
:10D910004FF0FF30FBE70000A880002001460329FC
:10D9200009DA0020C1EB8112C2EB0212034B03EBB8
:10D930008202907070474FF0FF30FBE7A880002014
:10D9400070B50546C5EB8510C0EB00100D4901EB25
:10D950008004002D02DB032D00DA14B94FF0FF30F4
:10D9600070BD2078042801D1401FF9E70120207004
:10D97000A06820B102212846D4E90232984700204D
:10D98000EEE70000A880002070B50546C5EB8510C5
:10D99000C0EB00100A4901EB8004002D02DB032DCF
:10D9A00000DA14B94FF0FF3070BD07202070A06876
:10D9B00020B100212846D4E9023298470020F3E73D
:10D9C000A880002070B50546C5EB8510C0EB00109F
:10D9D000184901EB8004002D02DB032D00DA14B995
:10D9E0004FF0FF3070BD062020701023020204F1BA
:10D9F000C40104F13C00FCF751F96078012808D11A
:10DA00000123C20204F2C46104F1B000FAF7D1FBB1
:10DA100007E01023DA0104F2C46104F16C00FCF7A2
:10DA20003DF9A06820B101212846D4E90232984787
:10DA30000020D7E7A880002070B50446C4EB84100E
:10DA4000C0EB0010094901EB8005002C02DB032C20
:10DA500000DA15B94FF0FF3070BDA86820B103217E
:10DA60002046D5E9023298470020F5E7A88000203B
:10DA70002DE9F84F0746884691461D464FF0FF3086
:10DA800000900024C7EB8710C0EB0010224901EB87
:10DA90008006002F03DB032F01DA06B11DB94FF01A
:10DAA000FF30BDE8F88F707801281BD14FF0000AD5
:10DAB0004FF0000B00BF0EE008EB0A0106F1B000CA
:10DAC000FAF79EFB18B1C5F800B00020E9E70BF1AA
:10DAD000010B0AF1010ACA45EED3C5F800B00020D7
:10DAE000009016E006F16C00FCF78DF8044684B156
:10DAF0006068484508D24046D4E90012F2F7A7FB17
:10DB00006068286000200090214606F16C00FCF758
:10DB100052F80098C5E70000A88000202DE9F047E2
:10DB2000044689461546C4EB8410C0EB0010254915
:10DB300001EB80060027002C02DB032C00DA1EB963
:10DB40004FF0FF30BDE8F087707801280FD1002733
:10DB50000AE009EB070106F1B000FAF70DFB10B17E
:10DB60004FF0FF30EEE77F1CAF42F2D328E000BF5A
:10DB7000C4EB8411C1EB0111124A02EB810101F1E6
:10DB80006C002946FCF75EF88046B8F1000F12D011
:10DB90002A464946D8F80000F2F759FBC4EB841135
:10DBA000C1EB0111074A02EB810101F16C00414612
:10DBB000FCF715F803E0214603A0FAF765FC00BF67
:10DBC0000020BFE7A8800020536F636B65745B255E
:10DBD000755D2052656376204275666665722046E3
:10DBE000756C6C0D0A0000002DE9F0410446884672
:10DBF00015460026C4EB8410C0EB0010134901EB5E
:10DC00008007002C03DB032C01DA07B11DB94FF0AC
:10DC1000FF30BDE8F081294607F13C00FCF712F81F
:10DC2000064636B921460AA0FAF72EFC4FF0FF301F
:10DC3000EFE72A4641463068F2F709FB314607F123
:10DC40003C00FBF7CCFF0020E3E70000A8800020A9
:10DC5000736F636B65745B25645D2073656E642010
:10DC60006275662066756C6C0D0A00000246032A18
:10DC700008DAC2EB8210C0EB0010044B03F820104E
:10DC8000002070474FF0FF30FBE70000A880002025
:10DC900001460020044A126890B24FF6C772104045
:10DCA0000843014A106070470030014010B5FBF78F
:10DCB00011FDF8F79BF8F9F77CF810BD10B592B09C
:10DCC00000BF002000902F48006840F080502D4990
:10DCD00008600846006800F08050009000BF00BF58
:10DCE00000BF002000902848006820F4404040F425
:10DCF0000040254908600846006800F44040009054
:10DD000000BF00BF012006900004079002200C9085
:10DD100041050D9108210E91A0210F910221109132
:10DD20000421119106A8F8F7A9FA18B1D22117A079
:10DD300002F05EFD0F20019002200290002003906F
:10DD40004FF48050049000200590022101A8F8F7BC
:10DD500057F918B1E0210DA002F04AFDF8F710FACA
:10DD60004FF47A71B0FBF1F42046F9F708F804207B
:10DD7000F8F7F0FF00221146501EF8F7CEF812B067
:10DD800010BD000040380240007000402E2E2F537E
:10DD900072632F6D61696E2E630000001348006886
:10DDA00040F47000114908601148006840F001001B
:10DDB0000F49086000200E49083108600C480068CF
:10DDC0000C4908400A4908600B48091D0860081FF3
:10DDD000006820F48020091F0860002004490C31ED
:10DDE00008600648014980390860704788ED00E006
:10DDF00000380240FFFFF6FE103000240000020849
:10DE000070B505460C46FBF7D7FB0949086044B1DD
:10DE100022462946022002F00BFA10B105A0FAF7BB
:10DE200033FB214609A0FAF72FFB002070BD00004C
:10DE30009001002052544B20446174612053656E60
:10DE400064204572726F720D0A0000002575422031
:10DE500052544B20446174612053656E740D0A0066
:10DE600010B50020044908700023044A0121044829
:10DE7000FFF794FC002010BD8C01002045DF020854
:10DE8000880100203EB5FCF726FA01283FD1FBF7B8
:10DE900093FB04462048007840BB20480078D8B95E
:10DEA00001201D4908701E48008D1D49C98C1C4A5F
:10DEB000928CCDE9002102901948438C19A24FF4AD
:10DEC00080611B48FBF7FDFD1548028B1849194876
:10DED0000068FFF73DFC19E017480068201A174951
:10DEE000884213D900200D4908700FE00A480078D5
:10DEF00002280BD112480068201A42F210718842A1
:10DF000004D30F48046000200349087002E0002099
:10DF10000149087000203EBD8C01002094010020C2
:10DF20009824002025752E25752E25752E25750023
:10DF300080290020880100209801002080EE360012
:10DF400090010020F8B506460C46174634B1012C66
:10DF50000CD0022C12D0032C26D113E014480078E8
:10DF6000012802D10020124908701EE010480078F4
:10DF7000012802D102200E49087016E000200C4949
:10DF8000087012E00025002000906B4640F2FF323E
:10DF9000084909480068FFF76BFD05461DB90548AB
:10DFA0000099FFF72DFF00E000BF00BFF8BD0000A3
:10DFB0008C010020802900208801002010B5024833
:10DFC000F9F7B1F810BD0000FCE50020002202685E
:10DFD000234B98420BD0B0F1804F08D0214B984290
:10DFE00005D0214B984202D0204B984201D1012309
:10DFF00000E000231BB122F070024B681A43184B5B
:10E00000984214D0B0F1804F11D0164B98420ED0E8
:10E01000154B98420BD0154B984208D0144B9842A0
:10E0200005D0144B984202D0134B984201D10123E2
:10E0300000E000231BB122F44072CB681A43026057
:10E040008B68C3620B688362054B984201D1012340
:10E0500000E000230BB10B690363012343617047A8
:10E06000000001400004004000080040000C004097
:10E0700000400140004401400048014030B5002309
:10E08000012404FA01F3046A9C430462046A02FA5C
:10E0900001F52C43046230BD30B50C460021816887
:10E0A00021F47F4142EA032525432943816030BDA5
:10E0B0000A460021816821F0700142F007031943EC
:10E0C0008160704730B5002400220023056A25F0E6
:10E0D00001050562026A4368846924F0700424F033
:10E0E00003040D682C4322F002028D682A430D4D73
:10E0F000A84201D1012500E000256DB122F00802FF
:10E10000CD682A4322F0040223F4807323F40073C1
:10E110004D692B438D692B43436084614D68456392
:10E12000026230BD0000014030B50024002200230F
:10E13000056A25F010050562026A4368846924F4C3
:10E14000E04424F440740D6844EA052422F02002DF
:10E150008D6842EA05120F4DA84201D1012500E069
:10E16000002585B122F08002CD6842EA051222F036
:10E17000400223F4806323F400634D6943EA85037E
:10E180008D6943EA8503436084614D68856302625B
:10E1900030BD00000000014030B500240022002303
:10E1A000056A25F480750562026A4368C46924F033
:10E1B000700424F003040D682C4322F400728D686F
:10E1C00042EA05220E4DA84201D1012500E00025BA
:10E1D00085B122F40062CD6842EA052222F4806211
:10E1E00023F4805323F400534D6943EA05138D69EA
:10E1F00043EA05134360C4614D68C563026230BDE4
:10E200000000014030B5002200230024056A25F4F7
:10E2100080550562036A4468C26922F4E04222F430
:10E2200040720D6842EA052223F400538D6843EAE8
:10E230000533094DA84201D1012500E0002525B193
:10E2400024F480444D6944EA85144460C2614D68F9
:10E250000564036230BD00000000014030B50B468C
:10E26000144600210022026A056A25F001050562B4
:10E27000816921F0F00141EA041122F00A021A43F7
:10E280008161026230BD30B50B4614460021002288
:10E29000056A25F0100505628169026A21F4704162
:10E2A00041EA043122F0A00242EA031281610262D3
:10E2B00030BD000010B50248FBF7A5FC10BD000002
:10E2C00038DD002010B504231A0203490348FBF788
:10E2D000E5FC002010BD000038D9002038DD00200A
:10E2E00070B505460E4604200D49086006B115B903
:10E2F0004FF0FF3070BD31460A48FBF7A3FC0446DF
:10E3000014B94FF0FF30F5E7324629462068F1F79F
:10E310009EFF21460348FBF762FC0020EAE700006D
:10E32000180C024038DD002010B50446FFF7C2FF8C
:10E33000A04204D121460348FBF73DFC10BD00205C
:10E34000FCE7000038DD002010B50248FBF75BFC5D
:10E3500010BD000068E1002010B504231A02034933
:10E360000348FBF79BFC002010BD000068DD002087
:10E3700068E1002070B505460E4604211248F7F703
:10E3800021FD38B904201049183108604FF4487055
:10E3900003F007F806B115B94FF0FF3070BD3146F4
:10E3A0000A48FBF74FFC044614B94FF0FF30F5E77D
:10E3B000324629462068F1F74AFF21460348FBF719
:10E3C0000EFC0020EAE70000000C024068E100209B
:10E3D00010B50446FFF7B8FFA04204D12146034818
:10E3E000FBF7E9FB10BD0020FCE7000068E100201E
:10E3F00010B50021002016E00E4A135C125C521C7E
:10E400000C4C2254052B0CDA0B4A32F810200A4B24
:10E4100023F811202246145C0A464B1C99B2054B86
:10E420009C54421C90B2054A12889042E4DB034A95
:10E43000118010BD205200209C4E0020760200204A
:10E4400010B5044604A0FAF71FF800200849086038
:10E45000F3F7B6FA10BD00004E54524950204170F7
:10E4600070205265636F6E6E6563740D0A00000064
:10E470003802002010B5044603A0FAF705F808A0FA
:10E48000FBF736FC10BD00004E5452495020436C3F
:10E4900069656E742074696D65206F75740D0A006E
:10E4A0002E2E5C464D4C5C496E7465726E65745CD4
:10E4B0004E54524950436C69656E742E633A31383C
:10E4C0003800000070B50546AC6B0020E085E084A4
:10E4D0002046F9F7CBF870BD70B506460025B46B41
:10E4E00020684069C0F3C01594F83900212805D18F
:10E4F00025B10020E084204600F082F820684069C1
:10E50000C0F3801594F83A00222805D125B10020E7
:10E51000E085204600F054F8E06B40F01000E06326
:10E520002046F9F7A3F870BD70B50546AC6B2868B6
:10E53000006800F48070B0B90020E0852068C068F1
:10E5400020F480702168C8602068406920F00100D4
:10E55000216848612068406920F0400021684861D6
:10E56000202084F83A002046F9F7D6FB70BD70B53C
:10E570000446A56B2846F9F7D5FB70BD70B5054676
:10E58000AC6B2868006800F4807070B90020E084EB
:10E590002068406920F08000216848612068C068D8
:10E5A00040F040002168C86002E02046F9F7A0FC76
:10E5B00070BD70B50446A56B2846F9F79FFC70BD89
:10E5C0000168C96821F490710268D16001684969E5
:10E5D00021F0010102685161202180F83A10704752
:10E5E00010B504462068C06820F040002168C8606B
:10E5F000202084F839002046F9F77AFC002010BD6D
:10E600000168C96821F0C0010268D160202180F84A
:10E610003910704770B5044694F83A00222844D166
:10E62000A068B0F5805F13D1A56A206940B9206861
:10E630004068C0F308002880A06A801CA06219E02E
:10E6400020684068C0B22880A06A401CA06211E027
:10E65000206938B920684068C1B2A26A501CA06223
:10E66000117007E02068406800F07F01A26A501C2A
:10E67000A0621170E08D401E80B2E08598B92068DC
:10E68000C06820F490702168C8602068406920F05C
:10E69000010021684861202084F83A002046F9F7FB
:10E6A0003BFB002070BD0020FCE70220FAE70000E1
:10E6B0002DE9F041044600252068056925F4405500
:10E6C000E0680543206805612068C56849F20C6070
:10E6D00085432169A068084361690843E1690843EB
:10E6E00005432068C5602068456925F44075A06928
:10E6F000054320684561E069B0F5004F7ED1C4490B
:10E700002068884203D0C349206888425DD1F7F76A
:10E710004DFD00EBC00101EB001061684900B0FB4A
:10E72000F1F06421B0FBF1F00601F7F73FFD00EBDB
:10E73000C00101EB001061684900B0FBF1F7F7F789
:10E7400035FD00EBC00101EB001061684900B0FB32
:10E75000F1F06421B0FBF1F000EBC00101EB00101F
:10E76000A7EB8000322101EBC0006421B0FBF1F087
:10E7700000F0F80006EB4006F7F718FD00EBC001CB
:10E7800001EB001061684900B0FBF1F7F7F70EFDEF
:10E7900000EBC00101EB001061684900B0FBF1F033
:10E7A0006421B0FBF1F000EBC00101EB0010A7EB1E
:10E7B0008000322101EBC0006421B0FBF1F000F0D9
:10E7C000070030442168886020E1F7F7DFFC00EBA8
:10E7D000C00101EB001061684900B0FBF1F0642159
:10E7E000B0FBF1F00601F7F7D1FC00EBC00101EB43
:10E7F000001061684900B0FBF1F700E045E0F7F771
:10E80000C5FC00EBC00101EB001061684900B0FBE2
:10E81000F1F06421B0FBF1F000EBC00101EB00105E
:10E82000A7EB8000322101EBC0006421B0FBF1F0C6
:10E8300000F0F80006EB4006F7F7A8FC00EBC0017B
:10E8400001EB001061684900B0FBF1F7F7F79EFC9F
:10E8500000EBC00101EB001061684900B0FBF1F072
:10E860006421B0FBF1F000EBC00101EB0010A7EB5D
:10E870008000322101EBC0006421B0FBF1F000F018
:10E880000700304421688860C0E061492068884200
:10E8900003D06049206888425CD1F7F787FC00EB21
:10E8A000C00101EB001061688900B0FBF1F6F7F7D9
:10E8B0007DFC00EBC00101EB001061688900B0FB3A
:10E8C000F1F06421B0FBF1F000EBC00101EB0010AE
:10E8D000A6EB8000322101EB00106421B0FBF1F0C7
:10E8E00000F0F006F7F762FC00EBC00101EB00104E
:10E8F00061688900B0FBF1F06421B0FBF1F006EB38
:10E900000016F7F753FC00EBC00101EB0010616843
:10E910008900B0FBF1F7F7F749FC00EBC00101EB10
:10E92000001061688900B0FBF1F06421B0FBF1F0E8
:10E9300000EBC00101EB0010A7EB8000322101EBDE
:10E9400000106421B0FBF1F000F00F0030442168AA
:10E9500088605BE0F7F71AFC00EBC00101EB0010E8
:10E9600061688900B0FBF1F6F7F710FC00EBC0011D
:10E9700001EB001061688900B0FBF1F06421B0FB8D
:10E98000F1F000EBC00101EB0010A6EB800032219A
:10E9900001EB00106421B0FBF1F000F0F006F7F796
:10E9A000F5FB00EBC00101EB001061688900B0FBD2
:10E9B000F1F06421B0FBF1F006EB0016F7F7E6FB8F
:10E9C00000EBC00101EB001061688900B0FBF1F7BA
:10E9D000F7F7DCFB00EBC00101EB00106168890078
:10E9E000B0FBF1F06421B0FBF1F000EBC00101EBF2
:10E9F0000010A7EB8000322101EB00106421B0FB76
:10EA0000F1F000F00F00304421688860BDE8F0812B
:10EA10000010014000140140014691F839002128FE
:10EA20002CD18868B0F5805F0FD10A6A1088C0F3D6
:10EA300008000B685860086918B9086A801C0862E9
:10EA400009E0086A401C086205E00B6A581C08626D
:10EA500018780B685860C88C401E80B2C88458B9BA
:10EA60000868C06820F080000B68D8600868C0683B
:10EA700040F040000B68D860002070470220FCE79F
:10EA80002DE9F04104460D4617469846069E21E0C2
:10EA9000701CF8B12EB1F7F7A3F9A0EB0800B04253
:10EAA00018D92068C06820F4D0702168C860206838
:10EAB000406920F0010021684861202084F8390075
:10EAC00084F83A0000BF002084F8380000BF03201B
:10EAD000BDE8F081206800682840A84201D10120EB
:10EAE00000E00020B842D3D00020F1E72DE9F04F3C
:10EAF000BFB007468846002400203290FD49FEA0A2
:10EB0000F9F7C2FC0822FEA13846F1F717FC0028ED
:10EB100070D10C2333AA2C213846FAF7E9FF0446BA
:10EB2000052C04D24FF0FF303FB0BDE8F08F349891
:10EB3000FAF77BFEF5498988884259D100250026DD
:10EB40003598FAF7F6FF0546F048B0F87000A8428D
:10EB500003D0EE49A1F87050012631A93698FAF792
:10EB600073FE9DF8C400E949B1F86610884214D1DB
:10EB70009DF8C500E549B1F8681088420DD19DF8AF
:10EB8000C600E249B1F86A10884206D19DF8C70074
:10EB9000DE49B1F86C10884214D001269DF8C400FB
:10EBA000DA49A1F866009DF8C500A1F868009DF853
:10EBB000C600A1F86A009DF8C700A1F86C0000200B
:10EBC000D34908703798FAF7B4FFD049B1F86E10FE
:10EBD000884206D03798FAF7ACFFCC49A1F86E000E
:10EBE00001262EB103F092FB0120C849A1F8600074
:10EBF00089E3FFE70822C7A13846F1F79FFB002809
:10EC000046D10C2333AA2C213846FAF771FF04466B
:10EC1000042C02D24FF0FF3086E73498FAF705FE55
:10EC2000BA4989888842E3D1BDA13698F1F762FBE1
:10EC30000028DDDD4CF6CC403190BCA0F9F724FC77
:10EC4000002302224FF488311846FDF71BF90223F6
:10EC500031AA4FF488310020FDF730FB00234FF438
:10EC600080724FF490311846FDF70CF93598F1F7A2
:10EC70003AFB451C2B464FF490310020359AFDF7A6
:10EC80001DFB0A2002F08DFB0020FDF74FF83AE350
:10EC90000822ACA13846F1F751FB78B90C2333AA0E
:10ECA0002C213846FAF724FF0446032C02D24FF0F9
:10ECB000FF3039E73498FAF7B8FD24E30922A4A11C
:10ECC0003846F1F73BFB002853D10C2333AA2C2103
:10ECD0003846FAF70DFF0446032C02D24FF0FF30FE
:10ECE00022E73498FAF7A1FD884989888842CED175
:10ECF0009AA13598F1F7FEFA20B93698FAF719FF7C
:10ED00009849088098A13598F1F7F4FA20B9369817
:10ED1000FAF70FFF9749087097A13598F1F7EAFACB
:10ED20000028B4D13698F1F7DEFA05462946369820
:10ED3000FFF720FB7548838890A24FF480616D48EF
:10ED4000FAF7BFFE32906B499148329A0068FEF79D
:10ED50004BFF6E48838889A24FF480616548FAF7BB
:10ED6000B0FE329063498A48329A0068FEF73CFF51
:10ED7000C9E20A2287A13846F1F7E0FA40B9F2F772
:10ED800037FE022899D15B495BA0F9F7A3FBBAE2F1
:10ED9000092283A13846F1F7D1FA40BB30A82EAB47
:10EDA00082A2414600903846FAF798FD02281DD10C
:10EDB0000020DDE92E1288542E98FAF736FD5349CB
:10EDC0008988884212D1DDE93001FFF789FA4F487E
:10EDD00083886AA24FF480614648FAF772FE329047
:10EDE00044496B48329A0068FEF7FEFE8BE2092226
:10EDF00073A13846F1F7A2FA60BB0C2333AA2C2189
:10EE00003846FAF775FE04463498FAF70EFD3F4986
:10EE1000898888421DD1022C02D24FF0FF3083E650
:10EE20003598FAF786FE85B23698FAF782FE86B2F2
:10EE3000102D02D14B4806800BE0B5F5007F02DAB9
:10EE4000324820F8156003F061FA01202F49A1F83B
:10EE5000600058E20A225DA13846F1F76FFA0028F7
:10EE600046D10C2333AA2C213846FAF741FE04463A
:10EE70003498FAF7DAFC25498988884239D1022C7E
:10EE800002D24FF0FF304FE63598FAF752FE86B2C5
:10EE90003698FAF74EFE1FFA80FB4FA1684601F044
:10EEA000D1FC85B219498A880DEB05004DA101F00E
:10EEB000C9FC1FFA80F905EB090085B2B24610E0E3
:10EEC000124931F81A200DEB050047A101F0BAFCF8
:10EED0001FFA80F905EB090085B20AF101001FFA5B
:10EEE00080FA0BEB06005045EADC652228467DE0FF
:10EEF0009DE09BE0802D002025730D0A000000009E
:10EF000024636F6E6669672C00000000982400205F
:10EF1000A0010020247570646174652C000000005D
:10EF2000563230323130353130303000676F746FE7
:10EF3000204F5441204170706C69636174696F6E39
:10EF40000D0A0000246765746C6F672C00000000D8
:10EF500024636F6E74726F6C2C00000062656570C4
:10EF600065720000040000207577625F656E616263
:10EF70006C6500002D00002054545300245265633A
:10EF800065697665766F6963652C25580D0A000002
:10EF90009C0100202475736572646174612C00000B
:10EFA00024736574746F6E652C000000247365749F
:10EFB000746F6E652C25702C25700D0A0000000002
:10EFC00024736574706172612C00000024726561A5
:10EFD00064706172612C0000247265706C797061DC
:10EFE00072612C0025782C0025642C00691C8DB2E0
:10EFF0000DF800206E222846691C8DB20DF8002005
:10F0000064222846691C8DB20DF800200D22284686
:10F01000691C8DB20DF800200A222846691C8DB2A9
:10F020000DF800202946684600F0E6FA6BE112224E
:10F03000B6A13846F1F782F900287BD10C2333AA18
:10F040002C213846FAF754FD0446062C02D24FF024
:10F05000FF3069E53498FAF7E8FB1FFA80FA359833
:10F06000FAF7E3FB80B231903698FAF762FD85B289
:10F070003798FAF75EFD86B23898FAF75AFD1FFA0C
:10F0800080F9A748BDF8C4100180A6488088504583
:10F0900002D04FF0FF3047E500204EE000EB40018A
:10F0A000A14A02EB410149889D4A1288914205D04C
:10F0B00000EB40019C4A12F81110C1B99849098827
:10F0C00000EB4002984B03EB4202518000EB400200
:10F0D00003EB4202567000EB400203F8125000EBC3
:10F0E00040011A4602EB4101A1F8049027E01D28D7
:10F0F00021D18E490A780978491C8C4B19701E2A37
:10F1000002DB00211A461170884A127802EB420293
:10F11000854B03EB42025670844A127802EB42029E
:10F1200003F8125000EB40011A4602EB4101A1F82E
:10F13000049004E005E0411CC8B21E28AEDB00BF0D
:10F14000E1E011227AA13846F1F7F8F8E8BB0C2388
:10F1500033AA2C213846FAF7CBFC0446032C02D202
:10F160004FF0FF30E0E43498FAF75FFB80B2319063
:10F170003598FAF7DEFC85B2C8264FF06409684876
:10F18000BDF8C410018000204FE000EB4001664A4A
:10F1900002EB41014988624A1288914205D000EB96
:10F1A0004001614A12F81110D1B95D49098800EB9C
:10F1B00040025D4B03EB4202518000EB400203EB47
:10F1C0004202567000EB400200E032E003F81250B9
:10F1D00000EB40011A4602EB4101A1F8049026E041
:10F1E0001D2820D151490A780978491C4F4B1970C4
:10F1F0001E2A02DB00211A4611704C4A127802EBDB
:10F200004202494B03EB42025670484A127802EB25
:10F21000420203F8125000EB40011A4602EB410192
:10F22000A1F8049003E0411CC8B21E28ADDB00BF6A
:10F2300069E0142243A13846F1F780F8E8BB0C23BB
:10F2400033AA2C213846FAF753FC0446042C02D288
:10F250004FF0FF3068E4F6F7E1FB4FF400413F4820
:10F26000F5F754F83598F1F73EF83190042231A9BA
:10F270003A48F5F7CFF9319A521C39483599F5F7E4
:10F28000C9F94CF6CC403090AFF26030F9F7FCF899
:10F29000002302224FF488311846FCF7F3FD0223C5
:10F2A00030AA4FF488310020FDF708F800234FF40E
:10F2B00080724FF49031184600E008E0FCF7E2FD60
:10F2C0000A2002F06EF80020FCF730FD1BE0172248
:10F2D00024A13846F1F732F8A8B90C2333AA2C211F
:10F2E0003846FAF705FC0446022C02D24FF0FF30F4
:10F2F0001AE43498FAF799FA204908703498FAF722
:10F3000094FA1F49087000200EE400002477726907
:10F310007465706172615F616E63686F722C00006A
:10F32000A80100209824002080310020AA0100209C
:10F330002472656164706172615F616E63686F728F
:10F340002C00000024646F776E6C6F61645F616EE7
:10F3500063686F7262696E2C000000000080000814
:10F3600000810008247365745F7570646174656161
:10F370006E63686F725F6D6F64652C00AB01002077
:10F380007701002070B58AB000242B48007802284D
:10F390004FD12A4800780890294890ED000B8DED58
:10F3A000060B284890ED000B8DED040B26482749ED
:10F3B0000968274A1278CDE9002102902548838800
:10F3C00025A24FF480613048FAF77BFB0446002603
:10F3D0000BE02E4931F816202B4908192CA101F019
:10F3E00031FA05462C44701C86B2144800788642D7
:10F3F000EFDB00260BE0274931F9162022490819D6
:10F4000025A101F01FFA05462C44701C86B20B485A
:10F4100000788642EFDB1C49081900221EA101F08A
:10F4200011FA05462C44224617491C480068FEF78D
:10F43000DBFB00200AB070BDA00100201B020020F1
:10F44000F8030020F0030020B47D00200004002019
:10F450001E02002098240020246D65737361676587
:10F46000322C68656172742C253034782C2530324A
:10F470007525252C25642C25732C256C662C256C74
:10F48000662C256400000000802D0020343E002002
:10F490002C2578008C4000202C2564009C01002045
:10F4A00010B50023034A02210348FEF777F9002034
:10F4B00010BD000079F502089C0100203EB5FAF766
:10F4C0000AFF012836D11E480078D8B901201C490E
:10F4D00008701C4800881C4909881C4A1288CDE91C
:10F4E000002102901A4803881AA24FF480611C4838
:10F4F000FAF7E7FA1B48028819491B480068FEF72B
:10F5000027F91AE00E480078022816D1FAF754F8C5
:10F51000044616480068201AB0F57A7F09D3002007
:10F520001349087011480460FFF72CFF00201149AF
:10F53000087002E000200249087000203EBD000073
:10F54000A0010020B2010020B0010020AE01002087
:10F55000AC01002025752E25752E25752E257500EC
:10F56000802D0020B40100209C010020A401002077
:10F57000B6010020B7010020F8B506460C46174634
:10F5800034B1012C0CD0022C12D0032C2AD113E060
:10F5900016480078012802D100201449087022E0A2
:10F5A00012480078012802D10220104908701AE0A0
:10F5B00000200E49087016E00025002000906B46E0
:10F5C00040F2FF320A490B480068FEF751FA05463F
:10F5D0003DB900200649009A885405480099FFF774
:10F5E00085FA00E000BF00BFF8BD0000A0010020C8
:10F5F000802D00209C01002070B505460C46144863
:10F600000078022821D11349134A1268881822462B
:10F610002946F0F71CFE1048006820440E49086097
:10F62000F9F7CAFF0D490968401AC8280DD3F9F740
:10F63000C3FF0A490860084806490268084800688C
:10F64000FEF7D2FA002004490860002070BD0000D7
:10F65000A001002034360020C4010020C801002091
:10F660009C01002010B5F6F7D9F900224FF41041A3
:10F670000748F6F7AFFB002204210648F6F7AAFB7D
:10F68000642001F08EFE0020FCF750FB10BD00004E
:10F69000000002400004024010B50248F7F7ECFFFA
:10F6A00010BD000038E6002010B50248F7F7E4FF6F
:10F6B00010BD000078E6002010B50248F7F7DCFF27
:10F6C00010BD0000B8E6002010B5F9F775FF0E492F
:10F6D0000968401AB0F57A7F05D3F9F76DFF0A493A
:10F6E000086000F017F8F9F767FF08490968401A41
:10F6F0000749C988884205D3F9F75EFF03490860C6
:10F7000000F03AF810BD000024020020280200207A
:10F710009824002010B5FEF76BFE10BD70B54FF4B5
:10F7200080100F49886140F68C2001F044FE1020C3
:10F730000B49886102F03AF904460CE002F036F910
:10F740000446FAF775FD2846691CCDB2142802DD7F
:10F7500004A001F04FF807488442EFD170BD0000CB
:10F76000000002404457204944204552524F522E37
:10F770000D0A00003001CADEF8B5002138E0002093
:10F780002EE06B4A32F910301446421C34F9122034
:10F79000934223DD674D35F81020254635F810508B
:10F7A000ABB2654D2C5C634E451C36F8155026F8FF
:10F7B00010505F4E451C36F8155026F810505E4E1E
:10F7C000451C755D35545B4E451C26F815201EB250
:10F7D000574F27F81560584E745500BF421C90B221
:10F7E000564A1278521E521A8242CADC481C81B212
:10F7F00052480078401E8842C1DC504800780028FA
:10F8000009DD4F48006818B988204D49086002E0BA
:10F8100000204B4908604B4803684B4802684B483E
:10F82000016847480068FCF7DFFE44480078142868
:10F8300002DD1420414908701220454988703F4874
:10F84000007800EB80000F30C870084641490988F5
:10F850008180414800783E4988713F48018800888E
:10F86000401C3D4A108008123949C8713B48007855
:10F8700008723B4800783B49097840EA41003A4920
:10F88000097840EA81003949097840EA411038494D
:10F89000097840EA81102E494872002008734873A5
:10F8A0008873C8732548007808742448007842009B
:10F8B000204927481130F0F7CAFC204909784A004E
:10F8C0001E490978112303EB4101214BC81818493F
:10F8D000F0F7BDFC19490978112202EB81011C4A9D
:10F8E000881816490A781449F0F7B1FC13480078D3
:10F8F00000EB800000F10F011548801CF1F7F6FFC6
:10F9000000900E48007800EB800011301049084448
:10F91000BDF8001001800948007800EB800000F17C
:10F9200013010B48FAF70CFB002004490870F8BDDE
:10F930008C400020343E0020E44200201B020020C6
:10F9400064060020700600206C0600206806002077
:10F9500064160020CC010020180200201E020020A6
:10F960002C000020080000201A01002009000020BF
:10F970002E00002038B50020009000212D4802F014
:10F9800093F800210F2001F0F5FF2B49086008468D
:10F99000008800F4804000283AD04FF480420021D3
:10F9A0000F2002F082F90021102001F0E3FFC4B221
:10F9B00000222146214802F031F82048B0F8010029
:10F9C00000901F48007850B11C48407A302806D17A
:10F9D00000201B490870BDF800001A490880BDF8D6
:10F9E000000018490988884219D102221649134893
:10F9F000401DF0F78DFC90B91048407A30280ED1A8
:10FA00000120124908600D48807A1149087006E00B
:10FA100001F06AFE0F4A00210F2002F046F9012191
:10FA2000044802F041F8002002F084F8002002F0BF
:10FA300009F838BD00D023246C0300202465002081
:10FA4000AB0100207801002070030020600300203B
:10FA50006B030020009027242DE9F04104460D4659
:10FA60004FF0FF360DB1032C03DB4FF0FF30BDE844
:10FA7000F08104EB4400C0EB4410554901EB8000D9
:10FA80008078002874D100BF00BF04EB4402C2EBB1
:10FA900044120B4603EB8202926804EB4403C3EB6F
:10FAA00044130F4607EB8303DB681A4404EB44035B
:10FAB000C3EB441307EB83035B685B6B1B685B68FA
:10FAC000D11A04EB4402C2EB44123B4603EB820220
:10FAD000D2680A4404EB4403C3EB441307EB8303EB
:10FAE0001B69D21A04EB4403C3EB441307EB8303F3
:10FAF000DB68B2FBF3F703FB172001280DD84BD1CD
:10FB000004EB4402C2EB4412314B03EB8202526815
:10FB10001268126802F020025ABB04EB4402C2EBE6
:10FB200044122B4B03EB8202126912782A7004EB09
:10FB30004402C2EB441203EB8202126904EB440359
:10FB4000C3EB4413224F07EB83035B699A4211D145
:10FB500004EB4402C2EB44123B4603EB8202926880
:10FB600004EB4403C3EB441307EB83031A6112E075
:10FB700013E011E004EB4402C2EB4412144B03EB1C
:10FB800082021269521C04EB4403C3EB4413104F6E
:10FB900007EB83031A61002617E004EB4400C0EB77
:10FBA00044100B4901EB8000807801280DD104EB53
:10FBB0004401C1EB4411064A02EB810101F1180036
:10FBC0002946F8F71DFB00B9002630464FE7000034
:10FBD00098E10020024609B1032A02DB4FF0FF3012
:10FBE000704702EB4200C0EB4210034B03EB800076
:10FBF000406808600020F3E798E100202DE9F0411B
:10FC000005460C460CB1032D03DB4FF0FF30BDE879
:10FC1000F08105EB4500C0EB4510524901F820503A
:10FC2000207805EB4501C1EB45114E4A02EB8101FD
:10FC30004870607805EB4501C1EB451102EB81018D
:10FC4000887005EB4501C1EB451102EB810160684D
:10FC5000886005EB4501C1EB451102EB8101A0680D
:10FC6000C860607838BB05EB4500C0EB4510114615
:10FC700001EB8000806805EB4501C1EB451102EB0B
:10FC80008101086105EB4500C0EB4510114601EB11
:10FC90008000806805EB4501C1EB451102EB810155
:10FCA000C9680844401E05EB4501C1EB451102EB54
:10FCB0008101486110E0607801280DD105EB450312
:10FCC000C3EB4513274E06EB830303F11800012312
:10FCD000D4E90112F8F76DFA05EB4501C1EB4511C6
:10FCE000204A02EB8101E068C86205EB4501C1EBE7
:10FCF000451102EB81012069086305EB4501C1EB69
:10FD0000451102EB8101A069086705EB4501C1EBD4
:10FD1000451102EB810160694863207810B12078B9
:10FD200001280DD105EB4506C6EB45160D4F07EB37
:10FD3000860606F13800D4E90423E168F9F7AEFF3E
:10FD4000607818B9284600F00FF808E060780128BC
:10FD500002D06078022802D1284600F083F8002003
:10FD600055E7000098E100207CB5044628E004EB4C
:10FD70004400C0EB44103A4901EB80004068006841
:10FD8000406880B20190BDF80400019000BF0020DF
:10FD9000009004EB4400C0EB441001EB800040688D
:10FDA00000680068009004EB4400C0EB441001EBD5
:10FDB0008000406800684068009000BF00BF00BF3E
:10FDC00004EB4400C0EB4410254901EB800040687F
:10FDD0000068006800F008000028C8D104EB440067
:10FDE000C0EB441001EB8000806804EB4401C1EBE0
:10FDF00044111B4A02EB8101086104EB4400C0EB93
:10FE00004410114601EB8000806804EB4401C1EB13
:10FE1000441102EB8101C9680844401E04EB44010F
:10FE2000C1EB441102EB8101486104EB4403C3EBD5
:10FE30004413154605EB83039B899AB204EB4403F4
:10FE4000C3EB441305EB8303996804EB4403C3EB52
:10FE5000441305EB83035868F7F7CAFE7CBD000026
:10FE600098E100201CB5044628E004EB4400C0EBF8
:10FE70004410234901EB800040680068406880B26C
:10FE80000190BDF80400019000BF0020009004EB39
:10FE90004400C0EB441001EB80004068006800683B
:10FEA000009004EB4400C0EB441001EB800040687C
:10FEB00000684068009000BF00BF00BF04EB440032
:10FEC000C0EB44100E4901EB8000406800680068F8
:10FED00000F008000028C8D104EB4402C2EB441231
:10FEE0000B4603EB820202F1680104EB4402C2EB11
:10FEF000441203EB820250680122F7F7DBFE1CBDBF
:10FF000098E1002070B504460D4604EB4401C1EBB6
:10FF10004411114A02EB81014868F7F790FB04EBAA
:10FF20004400C0EB44100C4901EB80004068456080
:10FF300004EB4401C1EB4411074A02EB810148681C
:10FF4000F7F740FC10B14FF0FF3070BD204600F0D5
:10FF500005F80020F9E7000098E1002070B504469C
:10FF600004EB4400C0EB4410534901EB800080785F
:10FF700038BB04EB4400C0EB441001EB8000806808
:10FF800004EB4401C1EB44114B4A02EB81010861CF
:10FF900004EB4400C0EB4410114601EB8000806884
:10FFA00004EB4401C1EB441102EB8101C968084430
:10FFB000401E04EB4401C1EB441102EB8101486196
:10FFC00023E004EB4400C0EB44103B4901EB80000C
:10FFD0008078012819D104EB4403C3EB44130D4688
:10FFE00005EB8303DA6804EB4403C3EB441305EB2E
:10FFF0008303996804EB4403C3EB441305EB8303C9
:020000040803EF
:1000000003F118000123F8F7D4F804EB4400C0EB27
:100010004410294901EB8000407840B104EB4400D2
:10002000C0EB441001EB8000407801281FD104EBA5
:100030004405C5EB4415204E06EB85056B6B04EBC0
:100040004405C5EB441506EB85052A6B04EB440516
:10005000C5EB441506EB8505E96A04EB4405C5EBE1
:10006000441506EB850505F13800F9F717FE04EB9A
:100070004400C0EB4410104901EB8000807818B9AF
:100080002046FFF771FE15E004EB4400C0EB44107E
:10009000094901EB80008078012808D004EB440076
:1000A000C0EB441001EB80008078022802D120468A
:1000B000FFF7D8FE002070BD98E1002070B504461F
:1000C0000D460DB1032C02DB4FF0FF3070BD04EB89
:1000D0004401C1EB4411084A02EB81007421F9F795
:1000E00073FB04EB4400C0EB4410034901EB8000B8
:1000F00045600020EAE7000098E1002070B5054661
:10010000002400BF2EE004EB4400C0EB441017496C
:1001100001EB80004068A84222D104EB4400C0EB10
:10012000441001EB8000807818B92046FFF71CFED0
:1001300015E004EB4400C0EB44100C4901EB8000D7
:100140008078012808D004EB4400C0EB441001EB98
:1001500080008078022802D12046FFF783FE03E06A
:10016000601CC4B2032CCEDB00BF70BD98E1002040
:1001700038B50546002400BF54E004EB4400C0EB52
:1001800044102A4901EB80004068A84248D104EBA2
:100190004400C0EB441001EB80008078012818D1A6
:1001A00004EB4400C0EB441001EB800090F86800C1
:1001B000009004EB4401C1EB44111C4A02EB8101A5
:1001C00001F118006946F7F7D7FF2046FFF74AFE0E
:1001D00025E004EB4400C0EB4410144901EB80001F
:1001E000807802281BD104EB4400C0EB441001EBE3
:1001F0008000006F80B104EB4402C2EB44120B4656
:1002000003EB820292F8680004EB4402C2EB441252
:1002100003EB8202116F88472046FFF723FE03E0BD
:10022000601CC4B2032CA8DB00BF38BD98E10020DD
:100230002DE9F04104460F4615464FF0000817B16E
:100240000DB1032C03DB4FF0FF30BDE8F08104EB70
:100250004400C0EB4410604901EB8000406810B9D5
:100260004FF0FF30F1E704EB4400C0EB44105A4973
:1002700001EB80004078E8BB00BFF9F757F804EBCA
:100280004401C1EB4411544A02EB810101F13800F1
:100290002946F9F7D7FC064626B9F9F72FFA4FF0A9
:1002A000FF382EE004EB4401C1EB44114A4A02EB53
:1002B000810101F138003146F9F791FC2A463946AF
:1002C0003068EFF7C4FF04EB4401C1EB4411424A2C
:1002D00002EB810101F13800F9F795FC0646F9F7C8
:1002E0000DFAB3889AB204EB4403C3EB4413DFF86E
:1002F000E8C000E006E00CEB830331685868F7F7CC
:100300007DFD66E004EB4400C0EB4410324901EB94
:1003100080004078012843D100BFF9F707F804EBCB
:100320004401C1EB44112C4A02EB810101F1380078
:100330002946F9F787FC064626B9F9F7DFF94FF0A9
:10034000FF382CE004EB4401C1EB4411224A02EBDC
:10035000810101F138003146F9F741FC2A4639465E
:100360003068EFF774FF04EB4401C1EB44111A4A03
:1003700002EB810101F13800F9F745FC0646F9F777
:10038000BDF9B3889AB204EB4403C3EB4413DFF81E
:1003900048C00CEB830331685868F7F77DFD18E01F
:1003A00004EB4400C0EB44100B4901EB80004078A3
:1003B00002280ED1642105FB01F3AAB204EB44012B
:1003C000C1EB4411044E06EB810148683946F7F74A
:1003D000AAFC404639E7000098E100202DE9F041F1
:1003E0000646002400BF88E004EB4400C0EB441044
:1003F000454901EB80004068B0427CD104EB4400E9
:10040000C0EB441001EB8000407898BB00BF04EBC8
:100410004401C1EB44113C4A02EB810101F1380077
:10042000F9F7F1FB054604EB4401C1EB4411364AF0
:1004300002EB810101F138002946F9F7BCFB04EB1E
:100440004401C1EB4411304A02EB810101F1380053
:10045000F9F7D9FB054665B1AB889AB204EB4403C2
:10046000C3EB4413284F07EB830329685868F7F759
:10047000C5FC3EE0FFE704EB4400C0EB441022491A
:1004800001EB80004078012833D100BF04EB440128
:10049000C1EB44111C4A02EB810101F13800F9F76C
:1004A000B2FB054604EB4401C1EB4411164A02EBD2
:1004B000810101F138002946F9F77DFB04EB440185
:1004C000C1EB4411104A02EB810101F13800F9F748
:1004D0009AFB054665B1AB889AB204EB4403C3EBC3
:1004E0004413094F07EB830329685868F7F7D4FCD6
:1004F00000BF05E0FFE7601CC4B2032CFFF674AF39
:1005000000BFBDE8F081000098E1002038B5044646
:10051000622C0CD100201549A1F86200088001F07E
:10052000F5FE13A11AA000F065F9FFF79BF8642C03
:100530001BD14AF6AA200090002302224FF48831F2
:100540001846FBF79FFC02236A464FF488310020CF
:10055000FBF7B4FE0A20F5F7ABF911A10CA000F0EF
:1005600049F90020FBF7E2FB00BF38BD98240020CA
:100570002E2E5C41504C5C73657269616C5F6174D6
:100580005F636D645F6170702E633A353500000003
:1005900025732055525452657374617274000000C3
:1005A0002E2E5C41504C5C73657269616C5F6174A6
:1005B0005F636D645F6170702E633A3637000000D0
:1005C00000BFFEE770B5044600256448007808289F
:1005D0005AD100BF002004E06149095C29448DB272
:1005E000401C60490978491F8142F5DC5E4800786B
:1005F000284485B25B480078284485B25B4800787F
:10060000284485B25A480078284485B25948007871
:10061000284485B26019C0B2FF282BD15248007817
:1006200001281DD0022823D150480078FFF76EFF23
:1006300051494E4A127888184D490A784849EFF7CF
:1006400006FE4A480078602803DB484800786428A2
:1006500005DD01F05BFE01204749A1F8600008E0DC
:1006600042480078411042480078FBF73DFF00E027
:1006700000BF00BF0020394908703C490870394963
:1006800008703E49087067E034480078072812D1A6
:1006900033483A490978445438480078401C37496F
:1006A000087030480078401F0978884254D10820EB
:1006B0002A49087050E029480078062805D12C48BE
:1006C000047007202549087046E024480078052872
:1006D00005D1264804700620204908703CE01F48D8
:1006E0000078042805D12048047005201B490870B3
:1006F00032E01A480078032808D11A480470002014
:100700001A49087004201549087025E0134800783C
:1007100028B9552C03D10120104908701CE00F485E
:100720000078012805D1AA2C03D102200B490870BA
:1007300012E00A480078022807D1032C05D10320D3
:10074000064908700B48047006E000200349087051
:10075000064908700349087070BD00008001002040
:10076000B82800208201002085010020830100209C
:1007700081010020840100209824002086010020AF
:1007800010B502211348F5F71DFBC8B9F8F714FF9F
:1007900011490968401A40F6B83188420DD9022043
:1007A0000E49088001200E4908700E4908700E4954
:1007B0000870F8F701FF08490860F8F7FDFE07E048
:1007C000F8F7FAFE04490860F8F7F6FE07490860F2
:1007D00010BD00000004024024000020040000209E
:1007E000B70100202C000020B601002028000020C6
:1007F00000BFFEE70FB4054B10B503A9044A0298E9
:1008000000F028FA10BC5DF814FB0000C11D0308BD
:100810007C0900200FB41CB50246002007AC00295B
:100820000BD0491ECDE90021054B6A4621460698AA
:1008300000F010FA009A002111701CBC5DF814FB46
:10084000831303080FB4084B10B504A902AA039838
:1008500000F000FA044602A9002000F09DFD2046A9
:1008600010BC5DF814FB0000991303087CB5044626
:1008700000201D46164600290BD0491ECDE9004137
:10088000044B6A462946304600F0E4F9009A0021FC
:1008900011707CBD83130308004870478009002055
:1008A0002DED020B019820F0004001909DED000B12
:1008B00002B070470000000000B583B09FED060B4A
:1008C0000A4601468DED000B6846EFF7BAFF9DED35
:1008D000000B03B000BD000000000000000000009D
:1008E00002E008C8121F08C1002AFAD170477047F9
:1008F000002001E001C1121F002AFBD1704708B59A
:10090000002000906B46012202212C2001F0E5F925
:10091000022000906B46012202212C2001F0DDF91B
:1009200008BD38B504466D2000906B46012240F6A4
:1009300006012E2001F0D1F93CB140F2076241F6E8
:1009400006012E2001F09EF906E041F2076241F611
:1009500006012E2001F096F938BD38B504466B46E5
:1009600002220021362001F027F80E2C57D2DFE8B2
:1009700004F011071A56565656233256563F464D26
:1009800000208DF800009DF8010000F0FE008DF8B9
:10099000010045E09DF8000000F0FC0040F001007F
:1009A0008DF800003CE09DF8000000F0FC0040F0F5
:1009B00002008DF8000033E09DF8000000F0B30065
:1009C00040F048008DF800009DF8010040F08000E4
:1009D0008DF8010024E09DF8000000F0B3008DF8D0
:1009E00000009DF8010000F07F008DF8010017E085
:1009F0009DF8010040F002008DF8010010E09DF824
:100A0000010000F0FD008DF8010009E09DF80000F4
:100A100000F0CF0040F020008DF8000000E000BFA3
:100A200000BF6B4601220021362001F056F90DF17E
:100A3000010301221146362001F04FF938BD08B5F7
:100A400003208DF8010001208DF800006B46022282
:100A50000021362001F041F94FF4004206212D20FB
:100A600001F010F9012000F09CFC0120FFF775FF58
:100A700008BD38B50446200A8DF80100E0B28DF8B3
:100A800000006B46022204212D2001F026F90320EC
:100A90008DF800006B46012206212D2001F01DF982
:100AA00000208DF800006B46012206212D2001F068
:100AB00014F90A212D2000F05DFF0546284638BDB7
:100AC0002DE9FF5F82B00021DDE90430020DDDF881
:100AD00040B0034318D044F61050A2F2FF32424314
:100AE0001514119801281FD0A5EB0B00401C5FEADC
:100AF000000A4FF000064E4FDFF83891B0465046DE
:100B000015D5CAF1000413E0119801244AA3012865
:100B100001D16FEA0B010298119AC0E90031C0E9D6
:100B2000024206B0BDE8F09FCBF10000DFE70446CB
:100B30000021404A491842EB0450CDE9001012E070
:100B4000E00707D032463B4640464946EFF7B9FC3E
:100B50008046894632463B4610461946EFF7B1FCBF
:100B600006460F466410002CEAD1DDE90401DDE9F8
:100B70000023BAF1000F06DAEFF7A3FC42464B461A
:100B8000EFF79FFC05E0EFF70EFD42464B46EFF70F
:100B90000AFD04460E460022284BEFF7CBFD03D892
:100BA0004FF0FF30014607E00022254B204631463A
:100BB000EFF7E0FBEFF744FF102409E0002C0ADB1D
:100BC0000A220023EFF702FB039B30321A55641E02
:100BD00050EA0102F2D1641C039AC4F111031444D7
:100BE000119A012A03D0012208430DD10AE00843DB
:100BF00004D000204FF0110B119072E7A3EB0B050E
:100C00006D1E0DE05B4504DD4FF0000205F10105AE
:100C100004E003DA4FF00002A5F10105002AECD050
:100C200002981199C0E90231C0E9004579E7000056
:100C3000000014400000F03F300000000000F043CE
:100C40000000E03F30380A2801D201207047002020
:100C5000704700002DE9FF4F95B09B468946064638
:100C600000250FE2252877D100242746F84A0121E4
:100C7000059400E0044316F8013F203B01FA03F01D
:100C80001042F7D130782A2811D06FF02F03307836
:100C9000A0F13002092A16D8059A44F0020402EBAA
:100CA000820203EB42021044761C0590EFE759F8EC
:100CB000042B0592002A03DA504244F400540590B4
:100CC00044F00204761C30782E2816D116F8010F55
:100CD00044F004042A280DD06FF02F023078A0F1E0
:100CE0003003092B09D807EB870302EB4303C7182E
:100CF000761CF3E759F8047B761C30786C280FD00B
:100D000006DC4C2817D068280DD06A2814D104E0DE
:100D1000742810D07A280FD10DE044F400140AE0B2
:100D200044F4801401E044F440147278824202D109
:100D300004F58014761C761C307866280BD013DC02
:100D4000582877D009DC002875D04528F6D04628E9
:100D5000F4D047281AD19DE118E0632835D06428E3
:100D600079D0652812D195E1702873D008DC672806
:100D7000F1D069286FD06E280DD06F2806D1B5E06C
:100D800073282CD0752875D0782874D05A461799B6
:100D900090476D1C75E1C4F30250022809D0032866
:100DA0000DD0D9F8001004280DD00D6009F1040908
:100DB00067E1D9F80010EA17C1E90052F6E7D9F85F
:100DC00000100D80F2E70D70F0E719F8041B8DF8A4
:100DD000001000208DF80100EA46012003E059F8D8
:100DE00004AB4FF0FF3061074FF0000102D40DE07B
:100DF00008F101018846B9420FDA8045F8DB1AF89C
:100E000008100029F4D108E008F101018846814268
:100E1000FADB1AF808100029F6D105985B46A0EB1A
:100E2000080721463846179A00F094FA284400EB48
:100E3000080507E04DE029E10DE01AF8010B5A46DC
:100E400017999047B8F10108F7D25B46214638461A
:100E5000179A13E142E00A220092C4F302524FF0C3
:100E6000000A022A08D059F804CB032A4FEAEC7191
:100E70000AD00DE029E02AE009F1070121F007027C
:100E8000F2E802C1914609E00FFA8CFC4FEAEC71DE
:100E9000042A03D14FFA8CFC4FEAEC71002907DADF
:100EA0000A460021DCF1000C61EB02012D2202E078
:100EB000220504D52B228DF80420012203E0E2074D
:100EC00001D02022F7E7904659E00A2102E01022E3
:100ED0000DE010214FF0000A00910BE010224FF0BE
:100EE000000A44F004040827009203E008224FF0AF
:100EF000000A0092C4F30252022A05D059F804CB2A
:100F00000021032A08D009E009F1070121F00702B6
:100F1000F2E802C1914605E01FFA8CFC042A01D1D7
:100F20000CF0FF0C4FF00008220728D5702806D0DF
:100F3000009B83F0100353EA0A0305D00EE0402221
:100F40008DF80420012208E05CEA010206D030227C
:100F50008DF804208DF8050002229046009B83F056
:100F6000080353EA0A030AD15CEA010201D16207CD
:100F700005D530228DF804204FF001087F1E582837
:100F800004D034A003900EA802900DE036A0F9E73B
:100F900053466046009AEFF719F984460398825C3D
:100FA0000298401E029002705CEA0100F0D10298A3
:100FB00006A9081A00F1200A600702D524F480343B
:100FC00000E00127574502DDA7EB0A0000E0002002
:100FD00000EB0A01009005984144401A0590E00397
:100FE00006D45B462146179A059800F0B3F90544EC
:100FF000002706E001A85A46C05D179990476D1C6E
:101000007F1C4745F6DBE0030CD55B462146179A6B
:10101000059800F09FF9054404E030205A461799DE
:1010200090476D1C0099481E00900029F5DC08E0EF
:10103000029802995A460078491C029117999047E4
:101040006D1CBAF10001AAF1010AF1DC65E10000B2
:10105000092801003031323334353637383961628E
:101060006364656600000000303132333435363752
:1010700038394142434445460000000000F058F929
:101080000544761C307800287FF4ECAD19B0284672
:10109000BDE8F08F620700D4062709F1070222F0AD
:1010A000070CFCE80223E14603F000485FEA080C65
:1010B00002D00FF2702C0DE05FEA045C02D50FF253
:1010C000682C07E05FEAC47C02D00FF2602C01E0DC
:1010D000AFF2700C4FF0FF3823F00043CDF850C052
:1010E00065280CD006DC452809D046281DD04728A5
:1010F0003DD13DE0662818D067287ED138E0002138
:10110000112F01DB112000E0781CCDE9000106A9B8
:101110000EA8FFF7D5FCDDE90F010E9A039100211F
:10112000009207F1010A04914DE04FF00040009752
:10113000CDE9011006A90EA8FFF7C2FCDDE90F02F8
:1011400003920E9B11990022DDF80CA000930492EB
:1011500011B9791C00EB010AB7EB0A0004D4C0F105
:10116000FF3007F1010A0490AAEB0700019044E068
:10117000012F00DA01270021112F01DD112000E0ED
:101180003846CDE9000106A90EA8FFF799FCDDE974
:101190000F010E9A0391002104910092BA46210793
:1011A0000CD40399514500DA8A46BAF1010F05DDE6
:1011B000009AAAF10101515C302908D0B84202DA44
:1011C00010F1040F06DA0121CDE9011015E0AAF1B2
:1011D0000101E9E7002805DC049901440491AAEB28
:1011E000000102E0411C514500DD8A460499401A85
:1011F000401C01904FF000400290200704D4019859
:10120000504501DBCDF8048000208DF84F00029896
:101210000DF14F07B0F1004F25D02B200E90029812
:101220004FF0020800280CDA404202902D200E9068
:1012300007E00A210298EFF7B1FA3031029007F87F
:10124000011DB8F10001A8F10108F2DC02980028A4
:10125000EFD1791E0E980870307800F0200040F031
:10126000450007F8020D12A8C01B00F107081498EA
:10127000007800B1012000EB0A01019801EBE07158
:1012800005984144401A401E0590E00306D45B4691
:101290002146179A059800F05DF8054414980078E7
:1012A00018B15A46179990476D1CE00324D55B4648
:1012B0002146179A059800F04DF805441CE0049863
:1012C000002807DBDDE90301884203DD0098405C6C
:1012D000179901E0179930205A469047049805F174
:1012E0000105401C04900198401E019004D12E205D
:1012F0005A46179990476D1CBAF10001AAF1010AEC
:10130000DDDC05E017F8010B5A46179990476D1C74
:10131000B8F10001A8F10108F4DC5B462146179AF8
:101320000598ABE62D0000002B0000002000000017
:101330002DE9F041044600251E461746880404D4D2
:1013400005E039462020B0476D1C641EF9D52846BB
:10135000BDE8F0812DE9F041044600251E46904687
:10136000C80301D5302700E02027880404D505E014
:1013700041463846B0476D1C641EF9D52846BDE885
:10138000F0814A68002A06D00A68531C0B6010706E
:101390004868401E486070470A68531C0B60107014
:1013A000704710B503464FF47A7003FB00F42046F3
:1013B00000F001F810BD002100BF40E000BF00BFF9
:1013C00000BF00BF00BF00BF00BF00BF00BF00BF25
:1013D00000BF00BF00BF00BF00BF00BF00BF00BF15
:1013E00000BF00BF00BF00BF00BF00BF00BF00BF05
:1013F00000BF00BF00BF00BF00BF00BF00BF00BFF5
:1014000000BF00BF00BF00BF00BF00BF00BF00BFE4
:1014100000BF00BF00BF00BF00BF00BF00BF00BFD4
:1014200000BF00BF00BF00BF00BF00BF00BF00BFC4
:1014300000BF00BF00BF00BF00BF00BF491C81420A
:10144000BCD370472DE9F84F04464FF00009CA4657
:1014500025786079824931F810806078401E814992
:10146000C6B20863042D01D0072D01D1012000E090
:101470000020834620787B490873E07938B9084614
:10148000806940F4800088614FEAE80805E075480B
:10149000806920F4800073498861207A714948731B
:1014A00008468069217A4FF4403202EA014108433C
:1014B0006C498861084600218269042000F0F5FB30
:1014C000424642F604012E2000F0DCFB3046FFF7D6
:1014D00028FA6548405D00EB800064494318052206
:1014E00007212B2000F0F9FB614800EB0B030122E0
:1014F0000B21282000F0F1FB5B48405D5D4951F86D
:1015000020200C21282000F0D0FBE0795A4901EB83
:101510008000A17930F811200221272000F0B2FBD1
:10152000564830F816200421272000F0ABFBE07964
:1015300028B964220621272000F0A4FB1EE0A07831
:1015400004280DD11020009010220621272000F041
:1015500099FB6B4601222621272000F0BEFB0DE0FF
:101560002820009020220621272000F08BFB6B46CC
:1015700001222621272000F0B0FB00BF404800EBED
:101580000610E17850F821200821272000F08DFB7B
:10159000B4F8090018B941F24100A4F80900B4F800
:1015A00009202021272000F06DFB36480C2102681D
:1015B000232000F07AFB3348001D30F81620042168
:1015C000232000F05FFBA07958B1E0792E49431841
:1015D00001220021212000F080FB4FF003094FF091
:1015E000010A05F00F00F02101EA051108436178B6
:1015F0004FF4402202EA81410843910001EA095177
:1016000008434FF4003101EA4A41084321794FF081
:10161000F86202EA815108436179520102EAC1612C
:1016200040EA01073A4600211F2000F03EFBA07867
:101630006178084300040B49086108460069E179B4
:101640004FF4004242EA4131084306490861084626
:1016500000210269082000F028FB0020BDE8F88F77
:10166000AC2A030884E40020542A030880060020E2
:101670009E0600205C2A03087C2A0308882A0308A7
:101680008C2A0308742A0308A006002038B50446F3
:101690000D460848808B0443224600212C2000F090
:1016A000F1FA00956B46012206212C2000F015FB73
:1016B00038BD000084E4002010B5FFF720F910BD0C
:1016C00070B505460421362000F054F9044615B1E2
:1016D00044F4006401E024F400642246042136202E
:1016E00000F0E3FA70BD000038B540200090002102
:1016F0000E2000F03FF90446002211460E2000F0B3
:10170000D4FA6B46012200210D2000F0E6FA084AC7
:1017100000210F2000F0C9FA00F098FA22460021BB
:101720000E2000F0C2FA0020024981F82C0038BDDA
:10173000F8FF272484E400202DE9FC41054604201D
:10174000019000264FF00008002078494875086392
:101750000021764880F825100020744981F82C007B
:1017600088834863886300F021F9704908600EE0BF
:101770004FF480106E49886140F2A460FFF71BFEB1
:1017800010206B49886100F011F9684908606748CA
:1017900000686849884204D03846791CCFB20A28CC
:1017A000E6DB0A2F03DD00206349A1F85800002082
:1017B000FFF7D3F800F0FAF85C4908605F4800785A
:1017C000242805DD5D48007824385D49086011E073
:1017D0005A480078062190FBF1F201FB12005749AC
:1017E0000978062291FBF2F1C1F1060140EA4110AD
:1017F000534908605248007800065149098840EA78
:1018000001404F49096840EA01204D4909680843F1
:101810004C4908600846002102681E2000F045FA85
:1018200000F0C4F84149086001AB012200212420E6
:1018300000F053FA1E20FFF71CF986B2300A3B492C
:1018400088730420FFF715F9804600F0AFF8374998
:10185000086008F0FF0070B1022000906B46012282
:1018600012212D2000F039FA3048808B40F480504E
:101870002E49888300BF00F099F82C4908600620A3
:10188000FFF7F7F8294948600720FFF7F2F82749E2
:10189000886006F01F0008750846007D08B9102012
:1018A00008752249087D00F071FA05F0010040B189
:1018B000FFF7C5F81D48808B40F400601B49888302
:1018C0000DE00521362000F03FF804464FF6FF50AA
:1018D000044022460521362000F0D4F900BF012043
:1018E000FFF73BF80021042000F044F80F4988611D
:1018F000012000F0EBF80021262000F03BF8044620
:1019000044F4A03444F4A02422460021262000F010
:10191000CCF900222621362000F0B4F900F046F878
:10192000024908600020BDE8FC81000084E400203A
:10193000000002403001CADE982400207506002015
:10194000780600207C060020F8B504460D464FF6C8
:10195000FF76A9B2A0B26B46022200F02DF807462E
:1019600037B99DF800009DF8011000EB012086B208
:101970003046F8BD2DE9F84305460E464FF0FF37D7
:10198000B1B2A8B26B46042200F016F88046B8F156
:10199000000F08D1032404E01DF8040000EB072722
:1019A000641E002CF8DA3846BDE8F88310B5002133
:1019B0000846FFF7DFFF10BD2DE9F84306460C4649
:1019C0001746984600252CB9F2B228466D1C0DF832
:1019D00000201BE0F0B240F0400228466D1C0DF8DC
:1019E00000207F2C05DCE2B228466D1C0DF800209B
:1019F0000CE0E0B240F0800228466D1C0DF800209B
:101A0000C4F3C71228466D1C0DF80020A8B2434647
:101A10003A46694600F03EFCBDE8F88370B50446DE
:101A20000D46164623462A4631461120FFF7C4FFCD
:101A300070BD10B504462346052200211520FFF78E
:101A4000BBFF10BD38B504460020009000F0FEF842
:101A50004FF480750CB145F400752A4600210D2025
:101A600000F010F9B4B16B46012203210F20FFF7FB
:101A7000A3FF9DF8000000F0080058B1FFF734FE06
:101A80004FF480752A4600210D2000F0FBF84FF03E
:101A9000FF3038BD0020FCE710B504462246012186
:101AA0000A2000F002F910BD70B504460E46002170
:101AB0000E20FFF75FFF05460EB1254300E0A5436A
:101AC0002A4600210E2000F0F0F870BD70B50546E2
:101AD00000212620FFF74EFF044624F47C2405F065
:101AE000010008B144F4802405F0020008B144F478
:101AF000A03422460021262000F0D7F870BD70B532
:101B0000054600211A20FFF735FF04466FF3130442
:101B1000C5F313000443224600211A2000F0C5F843
:101B200070BD10B50446224641F604012E2000F097
:101B3000A9F810BD38B504466B46012203210420E4
:101B4000FFF73AFF002C16DD224600210C2000F0A2
:101B500099F89DF8000040F0100000900F4880694F
:101B600040F080500D4988616B460122032104201A
:101B700000F0B3F810E09DF8000020F01000009095
:101B80000648806920F08050044988616B46012234
:101B90000321042000F0A1F838BD000084E40020F7
:101BA00010B5044622460021182000F06BF810BD45
:101BB000F8B50446002500200090002604F002003D
:101BC00058B1802000906B46012200210D2000F0CA
:101BD00084F801201C4981F82C0004F0010028B38E
:101BE0009DF8000040F0060000906B4601220021A5
:101BF0000D2000F072F803210F20FFF7A5FE064626
